:020000040802F0
:10000000D8F40020A9010208BDAC02081D9F020817
:10001000E1AA0208D1180208D9050308000000006F
:10002000000000000000000000000000FDC4020805
:10003000BF1D02080000000029B20208C5DC02084A
:10004000C3010208C3010208C3010208C301020878
:10005000C3010208C3010208DD420208F34202089C
:10006000C3010208C3010208C3010208C301020858
:10007000C3010208C3010208C3010208C301020848
:10008000451C0208551C0208C301020800000000BC
:10009000000000000000000000000000FD42020817
:1000A000C3010208C3010208C3010208C301020818
:1000B000C3010208D5DF0208C3010208C301020818
:1000C000C3010208C3010208C3010208C3010208F8
:1000D000C3010208B1F60208C1F6020800000000E0
:1000E000E7420208C3010208C30102080000000041
:1000F000000000000000000000000000C301020832
:1001000000000000C3010208C3010208C301020885
:1001100000000000000000000000000000000000DF
:10012000651C0208751C0208851C0208C301020830
:10013000C3010208000000000000000000000000F1
:10014000000000000000000000000000C3010208E1
:10015000C3010208951C0208A51C0208D1F602087A
:10016000C3010208C30102080000000000000000F3
:10017000000000000000000000000000000000007F
:1001800000000000C30102080000000000000000A1
:10019000C3010208DFF80CD000F06AFC00480047F9
:1001A0001D1E0308D8F40020064880470648004773
:1001B000FEE7FEE7FEE7FEE7FEE7FEE7FEE7FEE717
:1001C000FEE7FEE7B5DD0208950102082DE9F05FC4
:1001D0000546002092469B468846064681464024B6
:1001E0001BE0284641464746224600F020F8534689
:1001F0005A46C01A914110D311461846224600F0C3
:10020000E3FA2D1A67EB01084F4622460120002130
:1002100000F0DAFA17EB00094E41201EA4F10104A8
:10022000DFDC484631462A464346BDE8F09F202A97
:1002300004DB203A21FA02F00021704721FA02F390
:10024000D040C2F12002914008431946704740EA6D
:1002500001039B0703D009E008C9121F08C0042A44
:10026000FAD203E011F8013B00F8013B521EF9D22B
:100270007047D2B201E000F8012B491EFBD2704753
:100280000022F6E710B513460A4604461946FFF762
:10029000F0FF204610BD421E12F8013F002BFBD19B
:1002A00011F8013B02F8013B002BF9D1704730B542
:1002B00005462A460B4612F8010B13F8014B08B10C
:1002C000A042F8D01CB1002802D06D1CF1E72846EE
:1002D00030BDCAB2401E10F8011F8A4202D0002968
:1002E000F9D100207047421C10F8011B0029FBD1F6
:1002F000801A704710B5002200E0521C835C8C5CB1
:10030000A34201D1002BF8D1D8B2E1B2401A10BDFE
:1003100030B504460020034600E05B1C934203D244
:10032000E05CCD5C401BF8D030BD034611F8012BDA
:1003300000F8012B002AF9D11846704730B5054660
:100340000020034600E05B1C934205D2EC5CC85CD5
:10035000201A01D1002CF6D130BD70B5064610F040
:10036000A7FA046805460A220021304600F09CFAEC
:100370002C6070BD2DE9FE4F804681EA0300C00F5E
:100380000C46009021F0004123F00045B8EB02003C
:10039000A94105D24046214690461C460B460246DE
:1003A00023F00040104347D0270DC7F30A00C3F3E2
:1003B0000A510290401A019040286BDAC3F31300EF
:1003C00040F4801B0098924620B10023D2EB030A30
:1003D00063EB0B0B01985946C0F14002504600F008
:1003E000F3F906460D4650465946019A00F0FBF9CE
:1003F00010EB08006141002487EA115284EAE77398
:100400001A4340D0009A62B3019A012A4FEA075278
:1004100015DC001B61EB02014FF0004202EA0752BB
:10042000CDE90042001C41F5801132462B4600F018
:10043000B9FA03B0BDE8F08F40462146F9E7001B4A
:1004400061EB0201001C41F5801300185B4120188C
:10045000A2F5001747EB030140EAD570B6196D41CC
:1004600011E06D084FEA360645EAC0754FEA0752BB
:10047000001B61EB0201001C41F5801149084FEAA5
:1004800030000019514132462B4603B0BDE8F04F11
:1004900000F079BA0098012240000023D0EB02025C
:1004A00063EBE073009821464FEAE074B8EB00007C
:1004B00061EB0401E9E783F000435BE781F0004171
:1004C00058E72DE9FE4F81EA030404F0004421F0CF
:1004D000004100944FF0000B23F0004350EA010468
:1004E0005ED052EA03045BD0C3F30A54C1F30A5549
:1004F0002C44A4F2F3340194A0FB0254C1F3130181
:1005000041F48011C3F3130343F4801301FB02444D
:1005100000FB034E840A970A44EA815447EA835752
:10052000A4FB076802958D0A05FB07854FEA932C0B
:1005300004FB0C542705029D4FEA065847EA16377C
:10054000B5EB08056EEB070C870E920E47EA811794
:1005500042EA8312A7FB0201B6EB0B0164EB000435
:100560002B0D43EA0C335E1844EB1C50DA4651461F
:10057000E7FB0201C5F313044FEA0B3343EA1453BC
:100580004FEA0432019C43EA0603A4F10C040294EE
:10059000009CCDE900B400F005FA03B0BDE8F08F8F
:1005A00000200146F9E72DE9F04D81EA030404F04B
:1005B000004B21F0004514464FF0000A23F00041A3
:1005C00050EA050220D054EA01021DD0C5F30A57B3
:1005D0000246C5F31303C1F31300C1F30A5640F4F6
:1005E000801543F48013A7EB0608101BD64608F2CB
:1005F000FD3873EB050002D308F1010801E0921801
:100600005B41B8F1000F03DA00200146BDE8F08D30
:1006100000204FF48011064684460EE0171B73EB52
:10062000050705D3121B63EB050306434CEA010CD7
:1006300049084FEA300092185B4150EA0107EDD1BA
:1006400052EA030012D082EA040083EA050108435B
:1006500005D0101BAB4106D20122002306E0002288
:100660004FF0004302E06FF0010253101AEB060056
:100670004CEB085110EB0A0041EB0B01BDE8F04DCB
:1006800000F081B90EB540F2334102910021CDE96D
:1006900000110A460B4600F085F903B000BD70B5A5
:1006A000C1F30A5201F000450024C1F3130140F2E6
:1006B000FF3341F480119A4201DA002070BD40F20C
:1006C00033439A42A2F2334203DC5242FFF7AFFDBA
:1006D00000E090402C43F1D0404270BD00F0004259
:1006E00030F000400AD0C10D01F56071C0F3160072
:1006F00042EA0151C20840071143704700200146F9
:100700007047000030B5041E71F1000404DB4FF0A7
:100710000044404264EB0101141E73F1000405DB48
:100720001C464FF00043524263EB04038B4208BF68
:10073000824230BD30B5041E71F1000404DB4FF07D
:100740000044404264EB0101141E73F1000405DB18
:100750001C464FF00043524263EB0403994208BF2A
:10076000904230BD01F0004330B421F0004150EA26
:10077000010206D00A0DA2F56072C1F31301002A2E
:1007800002DC30BC00207047440F44EAC104C100C1
:10079000E01830BC00EBC25000F0BEB830B50B46DC
:1007A000014600202022012409E021FA02F59D42A1
:1007B00005D303FA02F5491B04FA02F52844151E75
:1007C000A2F10102F1DC30BD202A04DB203A00FA5C
:1007D00002F1002070479140C2F1200320FA03F398
:1007E000194390407047202A06DBCB17203A41FA84
:1007F00002F043EAE07306E041FA02F3D040C2F1AE
:100800002002914008431946704700000FB40023AE
:1008100000B589B00CA900910B996FF00042CB6034
:100820001E4B06931E4B07930423CDE901321D4A4C
:10083000089202466B46002000F0CEF909B05DF840
:1008400014FB70B586B006464FF0FF300091CDE93D
:100850000101002015460C4604903246694604A862
:10086000FFF7D4FF02460498211825B108B10846C5
:1008700000E020462860049800280DD0002A02DD00
:100880000098884208D0081B0094CDE90104324644
:10089000694604A8FFF7BAFF06B070BD110E020842
:1008A0002F0E02089D0A02082DE9F04791460F46D7
:1008B00080460446002614F8015B2DB100F0EAF8EA
:1008C0000068405DC007F6D12B2D02D02D2D18D029
:1008D000641E4A463946204600F0BAFA27B1396804
:1008E000A14201D1C7F8008071054FF002040BD579
:1008F0004042002803DD0FF0DBFF0460A007BDE8E5
:10090000F08746F48066E4E70028F8DA0FF0D0FFBD
:1009100004606FF00040F2E70029A8BF7047401C58
:10092000490008BF20F00100704710B4B0FA80FC05
:1009300000FA0CF050EA010404BF10BC704749B142
:10094000CCF1200421FA04F411FA0CF118BF0121B2
:1009500021430843A3EB0C01CB1D4FEA00614FEA92
:10096000102042BF002010BC704700EBC350104461
:100970000029A4BF10BC7047401C490008BF20F0EC
:10098000010010BC704710B5141E73F1000408DAA2
:10099000401C41F1000192185B411A4301D120F043
:1009A000010010BD2DE9F04D92469B4611B1B1FA00
:1009B00081F202E0B0FA80F220329046FFF704FFA5
:1009C00004460F4640EA0A0041EA0B0153465A46E4
:1009D000084313D0114653EA010019D0C8F1400270
:1009E0005046FFF724FC05460E46504659464246FF
:1009F000FFF7EAFE084305D0012004E0204639460F
:100A0000BDE8F08D0020054346EAE0762C433743ED
:100A10000A986305E40AA0EB08000022FD0A44EAF4
:100A200047540A3002D500200146E9E701051019B4
:100A30006941DDE9084500196941BDE8F04DA2E7CB
:100A4000C1F30A52C1F3130140F2FF3341F48011A4
:100A50009A4202DA00200146704740F233439A423C
:100A6000A2F2334202DC5242FFF7E1BBFFF7ACBE19
:100A7000064C074D06E0E06840F0010394E80700EB
:100A800098471034AC42F6D3FFF788FB3839030897
:100A90005839030800487047982B030810B50446DE
:100AA000FFF7F8FF0068005D00F0010010BD0000D6
:100AB0002DE9FF4F087883B09946FF2805D0491CDF
:100AC0002D2804D00024002008E000200BE00124A1
:100AD000F9E700EB800003EB4000491C0B78FF2B8B
:100AE000F7D104B1404200230293147819461D4601
:100AF0002D2C01D02B2C04D1521C2D2C13D00024D2
:100B00000294AA461478FF2C0FD00A25A3FB05787F
:100B100001FB05814FF0000C03FB0C11521CE31983
:100B20004AEB0101EEE70124EAE7814453EA0100C0
:100B300002D019F5C87F06DA03980021C0E9001138
:100B400007B0BDE8F08F0025AE4E2F46DFF8B88223
:100B5000184600F0DAF9CDE90001B9F1000002DA37
:100B6000C9F1000400E004460023A74A1AEB030B76
:100B700042EB045A12E0E00707D02A4633463846D3
:100B80004146FFF79EFC074688462A4633461046F4
:100B90001946FFF796FC05460E466410002CEAD174
:100BA000DDE90001B9F1000F5A46534606DAFFF7B6
:100BB000FAFC3A464346FFF7F6FC05E0FFF781FCF6
:100BC0003A464346FFF77DFC029A0AB181F00041A4
:100BD000039AC2E90001B3E72DE9FF4F1F468DB02C
:100BE000D7E901464FF0FF382E2045464FF0000967
:100BF0000B90B9696D1C0E988847396A8246884700
:100C00000028F6D1BAF1FF3F0AD024F4D064002EB8
:100C100011DDBAF12B0F08D0BAF12D0F0BD102E084
:100C2000404611B08DE744F48064B9696D1C0E989C
:100C300088478246761E6946600501D52D2000E072
:100C40002B208DF8000001F1010B0DF1200809E0C7
:100C5000B9696D1C0E98884782460F9844F4007459
:100C6000761E0560002E02DDBAF1300FF0D00B9930
:100C70008A453ED144F0800406E00F99681CA9F132
:100C8000010944F400740860B9696D1C761E0E9861
:100C9000884782463028F0D02BE00B998A4505D151
:100CA000200603D444F08004761E18E050460FF06E
:100CB000D5FF08B30DF11301761E44F400748B4583
:100CC00008D2AAF130000BF8010B200607D5A9F1D4
:100CD000010003E0200602D409F101008146A005CD
:100CE00002D50F99681C0860B9696D1C0E98884779
:100CF0008246002ED1DC53E0002E51DDBAF1650FA3
:100D000002D0BAF1450F4BD1A00549D5B9696D1C88
:100D100024F44074761E0E9888478246002E0CDD1F
:100D20002B2804D0BAF12D0F07D144F48074B9698F
:100D30006D1C0E9888478246761EE00501D52D2150
:100D400000E02B2108F8011BCDF82C8021E00DF1EB
:100D50002901761E44F4007488450CD2AAF13000B3
:100D600010F0FF0088F8000002D10B99884509D9DE
:100D700008F1010806E0E00501D5244801E042F24F
:100D80000F708146B9696D1C0E98884782460F988E
:100D90000560002E04DD50460FF060FF0028D6D11C
:100DA000F9690E988847FF208BF8000088F800004A
:100DB0000020069007904B466A4608A906A8FFF750
:100DC00077FEA00502D46FF001002AE714F0240F8B
:100DD0000AD0E00714D1DDE906123868031D3B6034
:100DE0000068C0E900120BE0DDE90601FFF7BAFC7C
:100DF0000146E00704D13868021D3A6000680160CE
:100E000028460EE7000014400000F03FF1D8FFFF35
:100E1000426842B1016811F8013B23B1521EC0E99A
:100E20000012184670470121C160881E7047426851
:100E30005AB1C368016843B983688B4205D0491E23
:100E4000521CC0E90012002070474FF0FF3070477D
:100E50002DE9F05F82460078002715468B460AF19F
:100E60000104B946302801D09DB113E014F8010BFC
:100E70000127782803D0582801D045B10AE00DB1E8
:100E8000102D07D10027102514F8010B02E00825CA
:100E900000E00A250026B0460EE005FB080005FB31
:100EA00006F1012701EB10461FFA80F8B6F5803FE6
:100EB00000D3B94614F8010B294600F018F80028B1
:100EC000EBDABBF1000F05D00FB1641E00E0544611
:100ED000CBF80040B9F1000F06D00FF0E9FC022179
:100EE0000160C81EBDE8F09F48EA0640FAE73A28CC
:100EF00000D2303820F02002412A01D3A2F137007D
:100F0000884201D34FF0FF3070470EB540F23342B4
:100F100002920022CDE900221346FFF743FD03B001
:100F200000BD70B58C1810F8015B15F0070301D1F6
:100F300010F8013B2A1106D110F8012B03E010F83C
:100F4000016B01F8016B5B1EF9D12B0705D400235F
:100F5000521E0DD401F8013BFAE710F8013BCB1A01
:100F6000921C03E013F8015B01F8015B521EF9D5F6
:100F7000A142D8D3002070BD70B50546AC6B206C83
:100F800000F0500050BB206C40F4007020642068DA
:100F9000806800F04050E8B9A069D8B92068C06AFC
:100FA00000F4700020B12068806800F4806088B987
:100FB0002068406820F0200021684860206C20F400
:100FC00080702064206C00F4805018B9206C40F0D0
:100FD00001002064204604F011F903E0A06BC16C0D
:100FE0002846884770BD70B50546AC6B402020642C
:100FF000606C40F004006064204604F001F970BDAC
:1010000070B50446A56B284604F0F9F870BD0000E1
:10101000014600220023022901DB00207047002244
:1010200006E0064800EB820030F811000344521C31
:10103000642AF6D36420B3FBF0F0EFE7F4E200207B
:1010400010B5C82202490348006804F06DF910BDCC
:10105000F4E200204006002054494A6822F440325D
:101060004A604A6843681A434A600268526822F438
:10107000807203685A6002685368026943EA022278
:1010800003685A600268526822F0407203685A602E
:101090000268526883681A4303685A60026892685B
:1010A00022F4006203689A6002689268C3681A4377
:1010B00003689A603E4B826A9A4218D0026892682E
:1010C00022F0706203689A6002689268836A1A4329
:1010D00003689A600268926822F0405203689A603E
:1010E00002689268C36A1A4303689A600BE0026858
:1010F000926822F0706203689A600268926822F037
:10110000405203689A600268926822F00202036803
:101110009A6002689368826943EA420203689A60AF
:10112000026AA2B10268526842F4006203685A601F
:101130000268526822F4604203685A600268536889
:10114000426A521E43EA423203685A6005E002686E
:10115000526822F4006203685A600268D26A22F47C
:1011600070020368DA620268D36A828B521E43EA15
:1011700002520368DA620268926822F4007203681D
:101180009A6002689368026B43EA422203689A609D
:101190000268926822F4806203689A600268936829
:1011A000426943EA822203689A6070470023014043
:1011B0000100000F01490860704700004006002050
:1011C00010B500200E49088000F04EFC09F094F89C
:1011D00008F004FA06F09EFF09F098F803F0A2FC6C
:1011E0000EF078F90748B0F85600012801D10CF04C
:1011F00055FE0AF043F80AF019F80FF0CDFA10BDC9
:101200001E0000209824002008B500200AF08EFE61
:1012100010F0CAFF0AF0E6FA00F0EEFB0BF024FC37
:10122000FFF70EFF00F054F809F04CF81248B0F840
:101230005600012802D10CF01FFE08E00E48B0F85D
:101240005600022803D109F025FE09F039FD03F00C
:10125000A3FA0EF031F911F0A3F8084808F088F964
:101260000020074B4FF47A72012100900348006878
:1012700008F00AFA08BD00009824002000000020B1
:10128000C5B1020810B5FFF79BFF0E4800780E4964
:10129000097888420ED00C4800780A490870084640
:1012A000007810B10EF046FA04E00020074908600B
:1012B00010F00EFA0348007808B111F08FF808F02A
:1012C000C3FF10BD2E0000202D000020640600206A
:1012D00010B5012010F06FFE0D4908700846007827
:1012E000132802D110F0A0FE10E00A4809F05AF8C5
:1012F000084800780649087008460078332802D16B
:1013000009F01EF802E000200349C88710BD000064
:10131000540600205506002098240020F8B500212E
:101320000F2010F033FB7F49086000217E4810F049
:10133000C7FB7C48008800F4804000287ED04FF432
:10134000804200210F2010F0BCFC0021102010F082
:101350001DFB764908700846007875490870002220
:1013600072480178734810F065FB73487149B1F811
:101370000110018071486F49B1F8051001806D4876
:1013800000786F49097888427ED16A48407A2028DF
:10139000FAD16848C0786B490870664800796A4994
:1013A00008706448807A6949087064486149B1F8F6
:1013B000051001806548007842005E490B316448A1
:1013C000FEF745FF61480078420060480078400021
:1013D0000B30584BC1185F48FEF739FF5B48007867
:1013E0000B2101EB8000534901445B4809880180CF
:1013F00000205A490880022059490870002519E048
:10140000534830F8150057490968884210D15648AA
:1014100090ED000B51EC100BFFF741F940B2464242
:101420004C4830F915103246444800880AF010FC48
:10143000681CC5B245480078854200E060E0DFDB0B
:101440003E48008800F09CFA4849088048480088D7
:10145000B0F5967F1CDB084600884549098888421C
:1014600013D14348008841490880344802884048E5
:1014700001880088401C3E4B18803E4820F811200F
:1014800001203D49087003E039E000203A49087026
:101490002E4800783949097888420BDD2B480078BE
:1014A0003649087029480078420022490B313448F7
:1014B000FEF7CDFE002414E00B2000EB44001D4994
:1014C000084400880090BDF8000026490968884259
:1014D00005D100202B490870204600F057F8601C09
:1014E000C4B21A4800788442E6DB18480078844287
:1014F0000BD1012023490870204600F047F804E092
:10150000214A00210F2010F0DCFB10F0F9F8012136
:10151000054810F0D5FA002010F018FB002010F05C
:101520009DFAF8BD5002002000D023245C02002068
:101530005D020020104400206402002066020020AA
:10154000D70100206E0200206F02002071020020EF
:10155000EC490020444C0020740200200A000020C6
:101560001A020020CC010020E802002078020020AE
:10157000760200209C4E00205F02002072020020B4
:101580003C450020600200200090272410B504464E
:101590006D4800686D4908806D4804706D486E495B
:1015A0000988A0F801106D490988C1816749098837
:1015B00001826B4800786749C87108466949098803
:1015C000A0F8051010F014FC674A03C267480078C1
:1015D000A04222D107F0FCFF642190FBF1F201FB55
:1015E0001200634908806148007800EB800040F2F7
:1015F0009E2101EB800004EB4401C1EBC41100EB20
:10160000C1000004C117584B0CCB80185941000A87
:1016100040EA01605749086018E05448007800EB40
:10162000800040F29E2101EB800004EB4401C1EBFD
:10163000C41100EBC1000004C1174B4B0CCB801848
:101640005941000A40EA01604A4908604948006877
:1016500010F02EFA45490978491C091B01EB41029B
:10166000C2EBC1110A2202EBC10010F054FA41484A
:10167000006820F001000021090241EA1061000227
:101680003D4A03C238480CC832481A3010F034FEC4
:1016900039480CC82F481E3010F02EFE0020374964
:1016A00088812C48898941843548007878B135484B
:1016B0003549364A128841F82200084633490988DC
:1016C00000EB810123480968C0F80A1008E02E48A1
:1016D0002E49098800EB81011E480968C0F80A10EC
:1016E0002B4800781B4908702A480078887421200C
:1016F00048720846C574C07C00F00F00C874002210
:101700003C2010F02AFB00213C2010F039FB012086
:1017100010F05AFA204908700020204908701E482D
:10172000007880B904E01D480078052800DD09E054
:1017300000210F2010F02AF91949086000F08000FC
:101740000028F0D000BF10BD240400407A02002021
:101750006B020020A6440020CC0100201C000020C9
:10176000EA010020660200208002002071020020B1
:101770004203002054020020400200209824002050
:101780005F020020FFFF01004C5300207802002080
:10179000D7010020680200206102002020060020FE
:1017A000500200200148008870470000A405002076
:1017B00010B500F003F8002010BD000010B5264859
:1017C000FFF7F8FC254900200AF028FE0021084612
:1017D0000AF006FD2023224A002108460AF06AFC8E
:1017E0002023204A032100200AF064FC40231D4AE4
:1017F000012100200AF05EFC80231A4A0221002009
:101800000AF058FC184900200EF064FC174901202A
:101810000EF060FC164902200EF05CFC4FF4806272
:101820000F49002001F0F4F801220D49022001F0D7
:10183000EFF84FF480520A49012001F0E9F8402204
:101840000C49002003F064F94FF48052054901204F
:1018500003F05EF9002010BDC0E4002068E5002020
:10186000000402400000024038E60020B8E60020F4
:1018700078E600200008024010B5114800880028D2
:1018800002DD01200F4908800E480088B8B10C48DD
:10189000008800280CDD0A480088401E084908809E
:1018A0000120094908700C21084805F0E9FD06E00F
:1018B0000020054908700C21044805F001FE10BD08
:1018C000040000200600002009000020C0E50020E0
:1018D00000BFFEE710B504460021024809F012F9E6
:1018E00010BD0000A9D5020810B502460B46002025
:1018F000002103E0545C0444A0B2491C9942F9D38E
:10190000C443A0B210BD00002DE9F04104460D46CD
:1019100016460748006838B106483246294603682B
:101920002046034F3F68B8470020BDE8F081000023
:10193000680500206C05002010B5002007490870DC
:101940000749086009F0ECFD00224FF4805105487A
:1019500004F04CFA00F008F810BD00001602002058
:10196000680600200000024010B50021034810F076
:10197000A7F80FF0C5FE0FF0ABFE10BD00D023247A
:1019800031B500240AE00A4800EB4401022268460F
:10199000FEF7BEFC00B905E0601C84B20548008873
:1019A0008442F0DB00BF002003490855204638BDC3
:1019B0009C4E002076020020205200200EB500210F
:1019C000084A0948CDE901210090A0F2E220B0F8D0
:1019D000A01200F2C22300F2A22200F5207009F04A
:1019E000F9F90EBD29AD02087A27002001480078D8
:1019F000704700007D03002000B587B01C216846B9
:101A0000FEF73EFC00208DF8010002208DF800005A
:101A10000F4801904FF480700290C0000490402065
:101A20000590694600200EF0F5F80A480A49C1F809
:101A300090050A48C1F89C050948C1F8980509486D
:101A4000C1F89405084607F071FC07B000BD00001E
:101A5000F46D0020C71B020854680020B91B02085F
:101A6000011C0208151C02081CB5FFF7BFFF10B9C6
:101A700007F0CEFB97E0FFF7B9FF01282FD1002038
:101A800001900090694602200EF0B0F820E09DF829
:101A90000400032812D14448006850B107F098FDB3
:101AA00041490968401AC8280BD9002000F0C2F843
:101AB00007E007F08DFD3C49086002E000203A494C
:101AC00008604FF47A73012201A9009806F037F9F3
:101AD00001A900200DF0CCFF0028D8D063E0FFF76B
:101AE00085FF02282FD10020019000906946022036
:101AF0000EF07CF820E09DF80400032815D12B4857
:101B0000006868B107F064FD28490968401AC828D0
:101B10000ED9012026490870002000F08BF807E05C
:101B200007F056FD2149086002E000201F490860C7
:101B30009DF804000EF052FD01A900200DF098FF61
:101B40000028D8D02FE0FFF751FF03282BD1002029
:101B50000190002420E09DF80400032815D11548C9
:101B6000006868B107F034FD12490968401AC828B6
:101B70000ED901200E490870002000F05BF807E044
:101B800007F026FD0B49086002E0002009490860C3
:101B90009DF804000EF022FD01A900200DF068FF61
:101BA0000028D8D000BF1CBD800300208403002083
:101BB0007E0300208803002010B504462146002043
:101BC0000DF056FF10BD0FB410B5ADF5027D85A820
:101BD00081904FF4007101A8819B849A0EF052FE0F
:101BE0000020819001A8FEF77EFB0446224601A951
:101BF00000200EF029FB0DF5027D10BC5DF814FBF2
:101C000031B500240122694600200EF01DFB044678
:101C1000204638BD70B5044600252046FEF763FB1C
:101C200006463246214600200EF00EFB05462846A9
:101C300070BD00000146024801700020704700009E
:101C40007D03002010B5024803F058FC10BD0000D1
:101C5000B8E7002010B5024803F050FC10BD0000AA
:101C600018E8002010B5024803F048FC10BD000041
:101C700008E5002010B5024803F040FC10BD00004C
:101C800078E8002010B5024803F038FC10BD0000D1
:101C9000F8E6002010B5024803F030FC10BD00004B
:101CA000D8E8002010B5024803F028FC10BD000061
:101CB00058E700200146087810381823B0FBF3F2EB
:101CC0000848805CC865032A05D908686FF30900D5
:101CD000001D886503E008686FF309008865886D5A
:101CE00070470000F62A0308014600208A6A8B69C3
:101CF000CBB932B1012A0DD0022A03D0032A10D168
:101D00000EE000BFCB6A03F08073B3F1807F00D197
:101D1000012007E0CB6AB3F1C07F00D1012001E0D0
:101D200000E000BF34E08B69B3F5005F1AD132B137
:101D3000012A07D0022A03D0032A11D10AE000BFEA
:101D400001200EE0CB6A03F08073B3F1807F00D1F5
:101D5000012006E0CB6AB3F1C07F00D1012000E092
:101D600000BF15E032B1012A05D0022A04D0032AAF
:101D70000CD103E000BF00BF012008E0CB6A03F0F4
:101D80008073B3F1807F00D1012000E000BF00BF6D
:101D9000704730B50468246824F4802405682C60FA
:101DA000046863608468402C04D10468A2600468FD
:101DB000E16003E00468A1600468E26030BD704740
:101DC00001201A4948720220194948720320194912
:101DD000487204201849487214481849097801705B
:101DE000144816490978017011481449097801709E
:101DF0000E4813490988A0F805100E4810490988B3
:101E0000A0F805100A480E490988A0F801100A48F0
:101E10000B490988A0F801100A4809490988A0F867
:101E2000011007490988A0F80510704784090020AF
:101E3000E2090020A609002098090020D70100200F
:101E4000CC010020F809002010B509F0A3FF3820CC
:101E50000BF02AFF01200FF07BFC08200BF024FF81
:101E60000FF0B0FD0F4908600F48007818B10F4817
:101E70000FF0F4FA02E00E480FF0F0FA01210D48DD
:101E80000FF01EFE48F283000FF057FE00200FF007
:101E900093FE4FF47A700FF059FE00200FF0DEFD34
:101EA00010BD0000C4000020770100204400002085
:101EB0003900002000D023242DE9F04391B00746DB
:101EC0000D4614463C22934902A8FEF7C0F9D7F804
:101ED0000880D8F83400D0F800902846362D73D00A
:101EE00013DC04283FD007DCC0B1012832D002281F
:101EF00037D0032869D135E00E2867D00F2867D086
:101F0000152876D03528F5D1C6E0373808285CD2B8
:101F1000DFE800F0C4C5C6C7C8C9CACB00207E49E7
:101F200008607E4908607C48006800EB400002AB16
:101F300053F820207848006800EB400003EB800055
:101F40004168404606F02EF874480068401C73490A
:101F50000860DBE0404606F047F8484607F0F2FA32
:101F6000D4E000BF00BF042D37D16B48006800EB00
:101F7000400002A901EB8000007A00F0040030B3B9
:101F800000206649086064480068401C6249086097
:101F900008460068052805D300226149384606F046
:101FA00031FC10E05C48006800EB400002AB53F8E5
:101FB00020205948006800EB400003EB8000416896
:101FC000404605F0EFFFA1E067E09DE052E000E051
:101FD0008EE0012011B0BDE8F0834F48006800EBAF
:101FE000400002A901EB80008068022D02D101218E
:101FF00001E06EE00221084018B300204749086064
:1020000045480068401C44490860084600680528A7
:1020100005D300224249384606F0F4FB29E03E4849
:10202000006800EB400002AB53F820203A480068FB
:1020300000EB400003EB80004168404605F0B2FF32
:1020400017E036480068401C3449086008460068BC
:10205000032805D300223349384606F0D3FB08E0B5
:102060000E203B4642F2107200210090484606F0D6
:10207000ADFB4BE02848006800EB400002AB53F892
:1020800020202548006800EB400003EB80004168F9
:10209000404605F087FF39E000BF00BF00BF00BF2A
:1020A00000BF00BF00BF00BF00BF26461A4800683F
:1020B00010B101280AD104E0D6E9000108F0A4FD1E
:1020C00005E0D6E9000108F0B7FD00E000BF00BF61
:1020D0001CE026466B4614A2D6E9000107F00AFC74
:1020E000012800D012E0DDE9000108F07BFD0DE0E1
:1020F000002008F017FD012805D100220D490E48E7
:1021000006F080FB02E001E0012063E700BF002051
:1021100060E70000BC2903080C0500201005002022
:102120005C290308FC2803082B434349443A202533
:10213000700D0A00EC2803088CC300202DE9F84339
:1021400004460D469046A668706B0768032D78D04C
:1021500005DC5DB1012D23D0022D6FD127E0042DC8
:1021600070D00E2D6CD00F2DF7D1B3E04FF461205D
:10217000614908600846016801200DF0CFFE00208B
:102180005E4908705E4908605E4908600E2023467B
:102190004FF47A7200210090384606F017FBA8E051
:1021A000304605F021FF384607F0CCF9A1E053484E
:1021B0000078012812D14FF461204F490860084689
:1021C000016801200DF0AAFE0E2023464FF47A721A
:1021D00000210090384606F0F9FA8AE000204949CB
:1021E000086047480068401C454908600846006888
:1021F000032818D340480068B0F5E13F09D1012019
:102200003E49087040A241F28831304605F0CAFECE
:1022100012E00321002008F099FC00223F492046EB
:1022200006F0F0FA08E00E2023464FF47A720021FF
:102230000090384606F0CAFA5BE002E056E001E0A2
:1022400033E056E02F480068401C2E49086000200B
:102250002B4908602B480068052812D14FF4E13063
:10226000254908600846016801200DF057FE0E2040
:1022700023464FF47A7200210090384606F0A6FA01
:1022800012E0204800680A2805D900222449204687
:1022900006F0B8FA08E00E2023464FF47A720021C7
:1022A0000090384606F092FA23E01448007801289E
:1022B00009D10321002008F049FC002217492046DB
:1022C00006F0A0FA15E017A241F28831304605F079
:1022D00069FE0EE0002008F025FC012805D100224F
:1022E0001249134806F08EFA03E002E00120BDE82F
:1022F000F88300BF0020FAE7000500200405002055
:10230000F8040020FC04002041542B4950523D3970
:1023100032313630303B26570D0A00002C29030895
:10232000FC280308415445300D0A0000EC2803083E
:102330008CC300202DE9F04105460E461446AF68D7
:1023400036B1012E16D0022E18D0032E1ED116E063
:10235000A046FFF727FA104908801049D8F8040072
:1023600008600D4803880EA241F28831384605F016
:1023700019FE0EE0384605F037FE0AE000BF0022E5
:1023800006480168284606F03DFA02E00120BDE853
:10239000F08100BF0020FAE7AC0500201006002005
:1023A00041542B434C564C3D25750D0A000000004E
:1023B0002DE9F84305460E461446AF6836B1012EA6
:1023C0001ED0022E20D0032E26D11EE0A0460120D2
:1023D000144908701449D8F80400086013480068CC
:1023E000006800901148006811A241F288314368EA
:1023F000384605F0D7FD0D4800680BF0A1FF0EE050
:10240000384605F0F1FD0AE000BF002206480168E9
:10241000284606F0F7F902E00120BDE8F88300BF86
:102420000020FAE7AA05002014060020B4050020C9
:1024300041542B514C544F4E453D312C252E2A737F
:102440000D0A00002DE9F04105460E461446AF681E
:1024500036B1012E14D0022E1BD0032E21D119E04B
:10246000A0461349D8F80400086012A241F288314E
:10247000384605F097FD4FF480201249086013E0BC
:1024800000201149087011490870384605F0ACFD6C
:102490000AE000BF002206480168284606F0B2F9AB
:1024A00002E00120BDE8F08100BF0020FAE7000053
:1024B0001806002041542B514C544F4E453D300DD1
:1024C0000A000000180C0240AA050020AB050020FD
:1024D0002DE9F84305460E461446AF6836B1012E85
:1024E0001ED0022E20D0032E26D11EE0A0460120B1
:1024F000144908701449D8F80400086013480068AB
:10250000006800901148006811A241F288314368C8
:10251000384605F047FD0D4800680BF065FF0EE0FA
:10252000384605F061FD0AE000BF00220648016858
:10253000284606F067F902E00120BDE8F88300BFF5
:102540000020FAE7A805002008060020B0050020BA
:1025500041542B515454533D322C22252E2A7322A0
:102560000D0A00002DE9F04105460E461446AF68FD
:1025700036B1012E14D0022E1BD0032E21D119E02A
:10258000A0461349D8F80400086012A241F288312D
:10259000384605F007FD4FF480201149086013E02C
:1025A00000201049087010490870384605F01CFDDD
:1025B0000AE000BF002206480168284606F022F91A
:1025C00002E00120BDE8F08100BF0020FAE7000032
:1025D0000C06002041542B515454533D300D0A0039
:1025E000180C0240A8050020A905002010B50446DB
:1025F000FFF7D8F81D490988884204D0204600F02A
:1026000043F8002010BD1A48007858B90BF0A8FE16
:10261000184908600846006868B1204600F086F84E
:102620000020EFE714480078012804D1204600F08C
:1026300093F80020E6E71148007858B90BF046FE01
:102640000F4908600846006868B1204600F03AF873
:102650000020D7E70B480078012804D1204600F07D
:1026600047F80020CEE74FF0FF30CBE7AC05002065
:10267000A8050020B0050020A9050020AA0500201B
:10268000B4050020AB0500201CB5044600200090D6
:10269000E06B40680190E06B406840680449486026
:1026A000002088606A46E06B06F0ACF800201CBD94
:1026B000D805002001200249087000207047000062
:1026C000AB0500201CB5044600200090E06B40687C
:1026D0000190E06B406840680449486000208860D1
:1026E0006A46E06B06F08EF800201CBDE80500206D
:1026F0001CB5044600200090E06B40680190E06B40
:102700004068406804494860002088606A46E06B81
:1027100006F078F800201CBDF805002001200249D1
:102720000870002070470000A90500201CB5044671
:1027300000200090E06B40680190E06B40684068CA
:1027400004494860002088606A46E06B06F05AF849
:1027500000201CBDB80500201CB5044600200090D8
:10276000E06B40680190E06B406840680449486055
:10277000002088606A46E06B06F044F800201CBD2B
:10278000C80500202DE9F84305460E461446D5F845
:102790000880022E18D003DC3EB1012E2CD10FE0B0
:1027A000032E12D00A2E27D116E027461549786845
:1027B000086015A241F28831404605F0F3FB1EE0A7
:1027C000404605F011FC1AE000BF00220D480168E8
:1027D000284606F017F812E00020009027466B46C6
:1027E0000CA2D7E9000107F085F8022800D006E026
:1027F000009808F04DFA02E00120BDE8F88300BF20
:102800000020FAE77804002041542B4353510D0A6D
:10281000000000002B4353513A2025642C252A0D3B
:102820000A0000001CB5044600200090E06B4068E0
:102830000190E06B4068406804494860002088606F
:102840006A46E06B05F0DEFF00201CBD6804002036
:1028500010B5044608F014FA012802D12046FFF70B
:10286000E1FF4FF0FF3010BD2DE9F04104460D4669
:102870001746A66835B1012D0BD0022D0DD0032DC2
:1028800016D10BE00DA241F28831304605F08AFBEB
:1028900011E0304605F0A8FB0DE000BF022108461C
:1028A00008F054F900220849204605F0ABFF02E089
:1028B0000120BDE8F08100BF0020FAE741542B431E
:1028C00046554E3D300D0A004C2903087FB5E0B057
:1028D00005460E46144622464FF4C0716846639B77
:1028E0000DF0D0FF684605F0DBFD002064B070BD40
:1028F00000B595B000208DF8390002208DF8380021
:1029000025480F904FF42060109024481190042027
:102910001290102013900EA901200DF07BF918B130
:102920004FF0FF3015B000BD1D4806F021FE10B17C
:102930004FF0FF30F6E71B4803901B480490382007
:1029400005901A4806901A4807901A4808901A48A5
:1029500009904FF4C0600A9018480B904FF4C06083
:102960000C900F480D9003A9154805F069FB10B1B4
:102970004FF0FF30D6E701201149124B12A2CDE9EA
:1029800000101349074805F0DFFE1249054805F01D
:1029900015FF0020C6E70000F4AC00207C040020F6
:1029A000800400208CC3002010260308A93D0208E3
:1029B000893F0208213E0208F4B60020F4BC002042
:1029C000F4C20020D02703084543363030530000BE
:1029D000CC280308CD28020810B50548006928B1A5
:1029E000034A918A1069012203F000FA002010BD09
:1029F00074C3002010B50548006928B1034A918AC4
:102A00001069002203F0F2F9002010BD74C3002009
:102A10000346044840F8331000EBC30082800020D6
:102A20007047000074C3002010B50548006828B145
:102A3000034A91881068002203F0D8F9002010BDE5
:102A400074C3002010B50548006828B1034A918876
:102A50001068012203F0CAF9002010BD74C30020E1
:102A60002DE9F04105460E461446D5F8088036B1EA
:102A7000012E0ED0022E10D0092E26D11DE00020EE
:102A80001549086015A241F28831404605F08AFADE
:102A90001EE0404605F0A8FA1AE00F480068012839
:102AA00005D100221049284605F0ACFE04E00022C2
:102AB0000E49284605F0A6FE0AE02746064B0CA262
:102AC000D7E9000106F016FF02E00120BDE8F08121
:102AD00000BF0020FAE700003005002041542B43DE
:102AE000474154543F0D0A009C2903085C29030800
:102AF0002B43474154543A20256400002DE9F0430C
:102B000093B005460C469146002720210BA8FDF7FF
:102B1000B7FBAE68706BD0F8008024228D4902A804
:102B2000FDF795FB07F0E6FF074605228AA1384628
:102B3000FDF704FC28B1052289A13846FDF7FEFB0C
:102B400028B989A220210BA806F0C7FF22E00522A0
:102B500087A13846FDF7F2FB28B987A220210BA8F0
:102B600006F0BBFF16E0052285A13846FDF7E6FB1F
:102B700028B97DA220210BA806F0AFFF0AE00522AC
:102B800081A13846FDF7DAFB20B981A220210BA8EC
:102B900006F0A3FF032C31D005DC5CB1012C25D05D
:102BA000022C7DD129E0042C29D00E2C79D00F2CB9
:102BB000F7D1C8E000207849086078490860764875
:102BC000006800EB400002AB53F820207248006818
:102BD00000EB400003EB80004168304605F0E2F96D
:102BE0006E480068401C6D490860AFE0304605F053
:102BF000FBF9404606F0A6FCA8E000BF00BF042C8D
:102C000033D16548006800EB400002A901EB800069
:102C1000007A00F0040020B30020604908605E489C
:102C20000068401C5C49086008460068032805D31A
:102C300000225B49284605F0E5FD11E05648006892
:102C400000EB400002AB53F820205348006800EB33
:102C5000400003EB80000BAB4168304605F0A2F961
:102C600074E0012013B0BDE8F083022C0AD14A4879
:102C7000006800EB400002A901EB8000007A00F040
:102C8000010060B9032C32D14348006800EB4000DA
:102C900002A901EB8000007A00F0020038B301E0E5
:102CA00052E03DE000203D4908603B480068401C80
:102CB0003949086008460068032805D300223849CE
:102CC000284605F09FFD2AE03348006800EB4000ED
:102CD00002AB53F820203048006800EB400003EBC3
:102CE00080000BAB4168304605F05CF917E02B48DB
:102CF0000068401C2949086008460068032805D37D
:102D000000222849284605F07DFD08E00E202B46CC
:102D100042F2107200210090404605F057FD15E088
:102D20001D48006800EB400002AB53F820201A4811
:102D3000006800EB400003EB80000BAB41683046BD
:102D400005F030F902E001E001208BE700BF002030
:102D500088E70000F82903083436303030000000DE
:102D60003436303032000000434D4E4554000000F0
:102D70003436303031000000554E494E4554000085
:102D80003436303036000000343630303300000046
:102D900043544E4554000000280500202C05002017
:102DA0008C290308CC2803082DE9F04104460D4680
:102DB0001746A66825B1012D03D00F2D15D101E0CE
:102DC00016E015E00C480078012808D100200A49D7
:102DD000087000220949204605F014FD08E030463D
:102DE00001F06CF800B903E002E00120BDE8F081D9
:102DF00000BF0020FAE70000980400205C290308C7
:102E0000F8B507460D4614460F2D0FD005DC4DB121
:102E1000012D08D0042D24D109E01A2D0DD0272D25
:102E20001FD11AE01FE00AF073FC1CE01BE0002237
:102E30000E49384605F0E6FC15E0264600200090D5
:102E40006B460BA2D6E9000106F054FD012800D024
:102E500009E000980AF080FD05E001200A490870A9
:102E600001E00120F8BD00BF0020FBE7DC280308DB
:102E70002B51495552433A2022636C6F736564228B
:102E80002C25640D0A000000980400202DE9F04173
:102E900004460D461746A66825B1012D03D00F2D17
:102EA00006D101E007E006E0304600F0E3FF02E073
:102EB0000120BDE8F08100BF0020FAE770B50546AB
:102EC0000C46164624B1012C03D0042C08D101E095
:102ED00008E007E000220549284605F093FC01E0E0
:102EE000012070BD00BF0020FBE70000DC280308C4
:102EF0002DE9F04104460D461746A66835B1012D6F
:102F00000BD0022D0DD0032D16D10BE00DA241F2F6
:102F10008831304605F046F811E0304605F064F897
:102F20000DE000BF0321022007F010FE0022084937
:102F3000204605F067FC02E00120BDE8F08100BFFB
:102F40000020FAE741542B4346554E3D310D0A000F
:102F50005C29030870B505460C46164624B1012CC1
:102F600009D00F2C1CD107E0FFF75EFD02210020E5
:102F700007F0ECFD16E015E0002007F0D3FD012876
:102F800003D10221002007F0E1FD002007F0D4FD6D
:102F9000012804D100220549284605F033FC01E050
:102FA000012070BD00BF0020FBE70000FC280308E3
:102FB0002DE9F84305460E469046AC68606B0768FD
:102FC00026B1012E1AD00E2E60D11BE00020E06247
:102FD00000BF2046216988470028FAD00020E0621F
:102FE0002D490870FFF720FD0E202B4640F6B83221
:102FF00000210090384605F0E9FB4AE0384606F02B
:10300000A1FA46E02448007830B1012813D0022804
:1030100025D0032838D131E001201F490870FFF77F
:1030200011FD0E202B464FF47A7200210090384695
:1030300005F0CCFB28E0022017490870FFF7CCFC14
:103040004FF4612101200CF069FF0E202B464FF454
:103050007A7200210090384605F0B8FB14E0032096
:103060000D490870FFF7C6FC0E202B464FF448723E
:1030700000210090384605F0A9FB05E00022074931
:10308000284605F0BFFB00BF00BF02E00120BDE8FD
:10309000F88300BF0020FAE7DC0400200C290308B5
:1030A000F8B507460D461446142D13D005DC4DB176
:1030B000012D08D0042D31D106E0332D1AD0342D46
:1030C0002CD121E02CE02BE000221749384605F0F6
:1030D00099FB25E02646002000906B4613A2D6E916
:1030E000000106F007FC012800D019E000980AF062
:1030F0000DFC15E0264612A13068FDF7FBF800B183
:103100000EE0FFF70BFB0BE0264610A13068FDF741
:10311000F1F800B104E0FFF7CDFA01E00120F8BDBD
:1031200000BF0020FBE70000DC2803082B514955B5
:1031300052433A202272656376222C2564000000F7
:103140002B515454533A20300D0A00002B514C544B
:103150004F4E453A20300D0A00000000034611B1E1
:10316000012902D100E002E001E00120704700BF28
:103170000020FBE72DE9F04105460C461646AF68F6
:10318000052C1FD2DFE804F0030E1213140007F021
:10319000B5FC804643460EA241F28831384604F021
:1031A00001FF12E0384604F01FFF0EE000BF00BF31
:1031B000304607F013FD084800224168284605F014
:1031C00021FB02E00120BDE8F08100BF0020FAE70A
:1031D00025730D0A00000000A00400202DE9F8432B
:1031E00004460E461546A768786BD0F80090072E67
:1031F00074D005DC5EB1012E1AD0022E6FD11EE014
:10320000082E6DD00E2E6CD00F2EF7D1C5E0002009
:103210006849087068490860684908600120684981
:10322000087068A241F28831384604F0BBFEBEE067
:10323000384604F0D9FE484606F084F9B7E05D4808
:103240000078A8BB00205E4908705C48006801282F
:1032500003D05A480068052811D10120554908704B
:1032600000205549086055490860012054490870FC
:1032700057A241F28831384604F094FE4EE04E48A1
:103280000068401C4C49086008460068642805D95D
:1032900000225249204605F0B5FA88E00E20234668
:1032A0004FF4FA6200210090484605F08FFA35E0AD
:1032B000FFE740480078012830D1002040490870DD
:1032C0003E480068012803D03C480068052809D121
:1032D00043480068401C424908600BE01FE063E07F
:1032E0002BE039E000203E49086033480068401C6C
:1032F000314908603A480068032805D3002239495B
:10330000204605F07FFA08E00E2023464FF4FA62CB
:1033100000210090484605F059FA00BF47E0A84652
:103320002448007840B9254B2FA2D8E9000106F0C7
:10333000E1FA022800D03AE039E0A8461D480078BA
:10334000012808D11D4B2CA2D8E9000106F0D2FAC1
:10335000022800D02BE02AE01648007860B900204F
:103360001649086001201649087027A241F28831E9
:10337000384604F017FE0FE00E48007801280BD104
:1033800000200E49086001200D49087010A241F28A
:103390008831384604F006FE09E00948007810B983
:1033A000384600F067FD02E00120BDE8F88300BF69
:1033B0000020FAE7140500201C0500201805002055
:1033C0002405002041542B43455245473F0D0A0038
:1033D00041542B43475245473F0D0A00DC28030860
:1033E000200500207C2903082B43455245473A20FD
:1033F000252A2C25640000002B43475245473A20DC
:10340000252A2C256400000041542B435245473F98
:103410000D0A00002DE9F04104460D461646A76846
:1034200035B1012D0ED0022D11D0032D19D10DE093
:103430000F4806600FA243F698210368384604F04F
:10344000B1FD11E0384604F0CFFD0DE000BF0848A3
:1034500000680AF081FA00220B49204605F0D2F9F3
:1034600002E00120BDE8F08100BF0020FAE7000083
:103470004005002041542B5149434C4F53453D25B5
:10348000642C31300D0A00009C2903082DE9FE4F01
:1034900005460E461446AF68786BD0F80090032EB0
:1034A0003CD005DC4EB1012E30D0022E74D134E078
:1034B0000E2E72D0162EF9D14BE0464804600068FB
:1034C0000AF0D4F98046434800680AF0BDF9824604
:1034D000404800680AF0FAF9012801D13EA000E056
:1034E0003EA08346CDE901A800903A483CA241F2B3
:1034F00088310368384604F055FD0E202B46414ABA
:1035000000210090484605F061F95FE0384604F07C
:103510006BFD484606F016F858E057E02D48006865
:103520000AF03EFA38480068401C374908600846EF
:103530000068032807D3002008600022334928468A
:1035400005F060F904E000223149284605F05AF9F7
:103550003CE0A04600200290019001A8009002AB40
:103560002CA2D8E9000106F0C5F9022800D02DE010
:1035700018480068029988421ED1019870B900204D
:1035800021490860134800680AF028FA00222049FF
:10359000284605F037F90FE015E00EE00D48006809
:1035A0000AF0FEF918480068401C1749086000221C
:1035B0001749284605F026F908E000221449284654
:1035C00005F020F902E00120BDE8FE8F00BF0020D9
:1035D000FAE70000380500205443500055445000DD
:1035E00041542B51494F50454E3D312C25642C22DE
:1035F0002573222C222573222C25752C302C300D7E
:103600000A00000020BF02003C050020CC2803086F
:103610009C2903082B51494F50454E3A2025642CD4
:1036200025640D0A000000002DE9FC4106460F4606
:103630001446D6F80880022F25D003DC3FB1012FB5
:1036400057D10EE0032F10D01B2F52D121E02C4870
:1036500004602CA241F288310368404604F0A2FCC9
:103660004AE0404604F0C0FC46E0254800680AF005
:1036700061F9234800680AF06FF9002226493046B4
:1036800005F0C0F838E000222349304605F0BAF8CA
:1036900032E0002001902546009001AB1FA2D5E941
:1036A000000106F027F9012804D0154800680AF047
:1036B00041F921E0019820B9114800680AF03AF96F
:1036C0001AE06B4618A2D5E9000106F013F90228AA
:1036D00004D00B4800680AF02DF90DE00848DDE938
:1036E000001200680AF026FA054800680AF0B0F9EE
:1036F00002E00120BDE8FC8100BF0020FAE70000E5
:103700004405002041542B514952443D25642C313D
:103710003032340D0A0000009C2903082B51495215
:10372000443A2025640D0A002B514952443A202581
:103730002A0D0A25650000002DE9F04385B00546F5
:103740000E461446AF68786BD0F80090032E50D028
:1037500005DC4EB1012E1CD0022E74D120E00E2EBD
:103760007DD0172EF9D153E045480460002045492B
:10377000087005F02DFF4449414A126841F82200C3
:103780003F4842A241F288310368384604F00AFCFF
:1037900072E0384604F028FC484605F0D3FE6BE0A2
:1037A0003848007801280AD100203D49344A12687F
:1037B000885400223B49284605F024F818E005F01B
:1037C00007FF39492E4A126851F82210401A37492A
:1037D000884208D32A4800680AF0BEF80020304921
:1037E000274A1268885400222E49284605F00AF814
:1037F00042E000202A49224A126888542048006882
:103800000AF0AAF800222749284604F0FBFF33E01B
:103810000020049003900290A04602A803A9CDE9DD
:10382000001004AB22A2D8E9000106F063F80328D7
:103830000BD0134800680AF08FF800221949284677
:1038400004F0E0FF18E013E009E0029818B9012045
:103850000C49087002E000200A4908700CE0084892
:103860000AA241F288310368384604F09BFB03E06A
:10387000012005B0BDE8F08300BF0020F9E700009B
:103880005005002054050020BCC3002041542B519A
:103890004953454E443D25642C300D0A000000007C
:1038A000340500209C290308C8C30020905F010054
:1038B0002B514953454E443A2025642C25642C2530
:1038C000640D0A002DE9F84305460E461746D5F863
:1038D00008800024032E33D005DC5EB1012E27D0F2
:1038E000022E77D12BE0102E34D0182E4AD0192E6C
:1038F0007BD170E040480760006809F0C7FF0446CC
:1039000004B975E0204606F08AF93C49086008468B
:10391000006800B96CE0394800684068009036489B
:1039200037A241F288310368404604F03BFB5FE078
:10393000002032490860404604F056FB58E057E04A
:103940002D4800680AF008F800223249284604F0A1
:1039500059FF4DE004F0CEFB012807D1274A126839
:103960005168264A1268106804F040FE2348006837
:1039700043682248006844F620610268404604F02B
:103980003BFB35E01C48006809F080FF044604B9A1
:103990002EE01A480168204606F019F901211E4858
:1039A000154A1268815405F013FE1C49124A126828
:1039B00041F8220008461049096850F821001849CA
:1039C0000D4A126841F8220000221249284604F0EC
:1039D00019FF0DE009E00848006809F0BDFF00226A
:1039E0000C49284604F00EFF02E00120BDE8F883F0
:1039F00000BF0020FAE70000480500204C05002029
:103A000041542B514953454E443D25642C25750D99
:103A10000A0000009C29030834050020BCC30020D4
:103A2000C8C300202DE9F0410446002600250027E8
:103A300005F0CEFD804600BF35E0284609F036FF90
:103A400003280BD1042128460AF01CF92A462D49E7
:103A5000E06B04F0D7FE0020BDE8F081284609F0B5
:103A600025FF042806D12A462749E06B04F0CAFE48
:103A70000020F1E7284609F019FF052806D12A465B
:103A80002049E06B04F0BEFE0020E5E7284609F07F
:103A90002DFF012806D12A461C49E06B04F0B2FE36
:103AA0000020D9E76D1C032DC7DB19480068401CB6
:103AB000032190FBF1F201FB120500261DE02846D0
:103AC00009F0F4FE062811D1284609F0DFFE07466A
:103AD00067B1384606F0A3F840B10D4805602A46A4
:103AE0000C49E06B04F08EFE0020B5E7681C032152
:103AF00090FBF1F201FB1205761C032EDFDB4FF089
:103B0000FF30A9E72C2A03081C2A03083C2A0308D3
:103B1000580500204C2A03082DE9F0432DED028BB7
:103B200091B004460D469146A668706B07689FEDFC
:103B3000370AB0EE408A042D58D005DC4DB1012D76
:103B400011D0022D58D14FE00E2D4ED0322D53D131
:103B500010E00E20234642F21072002100903846F9
:103B600004F034FE4EE0304604F03EFA384605F0EC
:103B7000E9FC47E007F0E0FCBCEEC00A244880ED19
:103B8000000A24488088000B4FF47A7110FB01F082
:103B900020498988C1F3032101EBC10202EB011125
:103BA00000EB81001B490979C1F3031101EB81018D
:103BB00000EB41001749097901F00F01084416494B
:103BC000086013480368084614A1026802A80CF0B4
:103BD00045FE1949086002A8FCF785FB804641466E
:103BE00002A80AF0D3FB0DE000BF00BF002213497A
:103BF000204604F007FE05E0012011B0BDEC028B69
:103C0000BDE8F08300BF0020F7E7000000000000DF
:103C1000E404002098240020F0040020C9E8B1B892
:103C2000B1E0BAC52564CAA3D3E0B5E7C1BFB0D936
:103C3000B7D6D6AE25640000EC0400201C2903088A
:103C40002DE9F84304460D469046A668706B076858
:103C5000102D6FD2DFE805F008141B252F6E6E6E55
:103C60006E6E6E6E5D6E3D6100203549087035499F
:103C7000086035A241F28831304604F093F95BE0E8
:103C8000304604F0B1F9384605F05CFC54E00E20F3
:103C9000234640F6B83200210090384604F096FDE5
:103CA0004AE00E2023464FF47A72002100903846F5
:103CB00004F08CFD40E022480078012805D1002264
:103CC0002449204604F09EFD02E00120BDE8F8836F
:103CD00032E01B480078012805D100221D4920460A
:103CE00004F090FD14E0174800680A280BD215482C
:103CF0000068401C1349086013A241F28831304625
:103D000004F050F904E000221349204604F07AFD43
:103D100012E001200A4908700EE0002006F002FFC0
:103D2000012805D100220D490D4804F06BFD03E088
:103D300002E0FFE70120C9E700BF0020C6E700005E
:103D4000050500200805002041542B4350494E3FF3
:103D50000D0A00003C2903084C290308EC2803083D
:103D60008CC3002010B50446022006F0DBFE0128BB
:103D700012D100200A490860E06B40684860E06B9F
:103D80004068406807494860002088600022E06B76
:103D900004F038FD002010BD4FF0FF30FBE70000BD
:103DA000A0040020BC04002070B505460C46214646
:103DB00001200BF05DFE70BD0648416805E0064835
:103DC000814201D10120704749680029F7D10020C4
:103DD000F9E700008CC300208C29030810B50446C5
:103DE000022006F0A9FE012812D100200A4908602D
:103DF000E06B40684860E06B406840680749486095
:103E0000002088600022E06B04F0FCFC002010BD64
:103E10004FF0FF30FBE70000A0040020CC0400209E
:103E200070B506460D461446285D68B944B1601E5B
:103E3000285C0A2804D1294606A004F079FB03E097
:103E4000294608A004F074FB2246294601200CF004
:103E5000FBF970BD5B41542053656E645D20257392
:103E6000000000005B41542053656E645D202573A3
:103E70000D0A000010B50446204600F067F808B9A6
:103E8000002010BD2046FEF7B1FB08B90020F8E77E
:103E9000204600F003FA08B90020F2E72046FFF7B9
:103EA00061FF08B90020ECE72046FFF797FF08B94B
:103EB0000020E6E74FF0FF30E3E7000070B505466D
:103EC00005F086FB0446284600F040F808B90020BB
:103ED00070BD2846FEF78AFB08B90020F8E728469F
:103EE000FFF7A0FD08B90020F2E72846FEF7B0FC76
:103EF00008B90020ECE712480068201A42F210715D
:103F0000884208D90E48046000220E490E4804F089
:103F100079FC0020DCE7284600F0C0F908B9002051
:103F2000D6E72846FFF71EFF08B90020D0E728464D
:103F3000FFF754FF08B90020CAE74FF0FF30C7E78A
:103F40009C040020AC2903088CC3002010B5044653
:103F5000002006F0F1FD012803D10321002006F026
:103F6000F5FD002006F0DEFD012806D100220449FF
:103F7000044804F047FC002010BD4FF0FF30FBE781
:103F8000EC2803088CC300207FB504460020039072
:103F90002CB1E06818B1606A08B1A06A18B94FF096
:103FA000FF3004B070BD14E103A92046E2689047D9
:103FB00010B14FF0FF30F4E79DF80C10E26A501C8E
:103FC000E062606A81540020E26A616A8854E06AB3
:103FD00007280CD1072290A0616AFCF799F930B943
:103FE00001208F49087001F007FF8E490860E06AE0
:103FF00007280CD107228CA0616AFCF789F930B937
:1040000002208749087001F0F7FE86490860E06ADF
:104010000A280CD10A2286A0616AFCF779F930B926
:1040200003207F49087001F0E7FE7E4908607C4864
:104030000078012807D07A480078022803D0784811
:104040000078032809D101F0D7FE76490968401AA3
:1040500040F2DC51884200D9C1E071480078012863
:104060001FD176A1606AFCF722F90546C5B1002090
:10407000029002AB72A2E16A606A05F03BFC012883
:1040800000D0ACE0029800B9A9E0606A281A801C50
:10409000029908446D4908600A206149087000BF10
:1040A00097E05F480078022829D164A1606AFCF794
:1040B000FEF8054615B366480068B0F1FF3F0ED123
:1040C0000020029002AB63A2E16A606A05F012FC74
:1040D000012800D083E05E490298086000BF5C4878
:1040E000006800B97BE0606A281A801C584909689A
:1040F0000844564908600A204949087069E0484860
:104100000078032825D1002002904CA1606AFCF7BA
:10411000CEF801900198D8B101A8009002AB50A24E
:10412000E16A606A05F0E6FB052800D057E0606AA6
:104130000199081A001D02990844444908600A20A0
:10414000374908704149E06A0968884200D146E071
:104150003FE0334800780A2805D13C49E06A096805
:10416000884236D13BE09DF80C000D2803D1012098
:1041700084F830000AE09DF80C000A2806D194F873
:104180003000012802D1022084F8300094F8300079
:10419000022816D1E06A022804D10020E06284F8E7
:1041A00030000EE0002084F830001D4800780A2816
:1041B00006D100201A490870E06284F8300000E05F
:1041C0000DE0E06A012804D1606A00783E2800D141
:1041D00005E0D4E90A01401E8142FFF4E5AE00BFCC
:1041E000E16A606A05F06CFB012810D1E06A50B109
:1041F000E06A401E616A085C0A2804D11FA0616A57
:1042000004F096F903E021A0616A04F091F900201E
:104210000349087000BFC4E62B514952443A2000BC
:104220008C04002094040020434F4E4E454354001C
:104230002B514D54524543563A2000000D0A0000C0
:104240002B514952443A202564000000900400207C
:1042500088040020434F4E4E4543542025640000FF
:104260002B514D54524543563A20252A2C252A2CB1
:10427000252A2C25752C2565000000005B41542063
:10428000526563765D202573000000005B41542079
:10429000526563765D2025730D0A000010B5044653
:1042A00006F094FC012812D100200A490860E06B56
:1042B00040684860E06B40684068074948600020FB
:1042C00088600022E06B04F09DFA002010BD4FF0E2
:1042D000FF30FBE7A0040020AC04002010B5012053
:1042E00001F084FC10BD10B54FF4805001F07EFC4D
:1042F00010BD10B5022001F079FC10BD10B54FF4CF
:10430000007001F073FC10BD70B586B004460D4618
:10431000002000900190022005900120029020468C
:1043200006F096F803906119481E06F091F80646CB
:10433000204606F08DF8301A401C0490694601A80A
:1043400001F0D6FA18B14FF0FF3006B070BD002072
:10435000FBE7000010B5002201B909E0012901D1F5
:104360000A0205E0022901D10A0201E04FF440727D
:104370000E4B1B6823F440730C4C236023461B68D0
:104380001343236023461B6823F0F803236023466E
:104390001B68022444EAC0042343044C23602346E0
:1043A0001B6843F48033236010BD0000103C0240C2
:1043B0001C48006800F40070B0B11A48006820F48E
:1043C00000701849086000BF0846006840F40060AB
:1043D00008600846006820F40060086000BF0846D6
:1043E000006840F4007008600E48006800F48060C7
:1043F000B0B10C48006820F480600A49086000BF32
:104400000846006840F4805008600846006820F4C0
:104410008050086000BF0846006840F48060086073
:1044200070470000003C02400A4A126822F44072C1
:10443000084B1A601A46126842F004021A601A46C3
:1044400012684FF4803343EA00231A43014B1A6089
:1044500070470000103C0240074A126822F4407284
:10446000054B1A601A4612681A601A46126842F022
:1044700001021A6001707047103C024010B50949F2
:10448000096821F44071074C21602146096841F414
:10449000407121602146096841F0010121600260FC
:1044A000436010BD103C0240084A126822F440727A
:1044B000064B1A601A46126842F480721A601A4655
:1044C000126842F001021A6001807047103C0240FD
:1044D000084A126822F44072064B1A601A461268A3
:1044E00042F400721A601A46126842F001021A6021
:1044F00001607047103C02402A48006800F010003C
:1045000040B12948C06940F010002749C861102017
:10451000244908602348006800F0200040B1224888
:10452000C06940F008002049C86120201D4908608A
:104530001C48006800F0400040B11B48C06940F0D2
:1045400004001949C86140201649086015480068F0
:1045500000F0800040B11448C06940F002001249E8
:10456000C86180200F4908600E48006800F4807020
:1045700048B10D48C06940F001000B49C8614FF4D3
:104580008070084908600748006800F0020040B1E8
:104590000548C06940F020000349C8610220014974
:1045A000086070470C3C024038E9002070B50446B2
:1045B000002500201449C86101F01EFC054609E0F1
:1045C000601C38B124B101F017FC401BA04201D996
:1045D000032070BD0D48006800F480300028EFD142
:1045E0000A48006800F0010010B101200749086086
:1045F0000648006800F4F97018B1FFF77DFF01204C
:10460000E7E70020E5E7000038E900200C3C024025
:104610002DE9F84307460D4614460026B046002013
:10462000009024E0042C0CD24FF0FF3000900026C4
:1046300003E0A85D0DF80600761CA642F9D3A0465B
:1046400003E0286800904FF00408F3200A4908604E
:10465000002339460220009A01F0A0F918B14FF06A
:10466000FF30BDE8F88347444544A4EB0804002C20
:10467000D8D10020F5E700000C3C02400FB4F8B59B
:1046800004460D4600261CB9701EF8BC5DF814FBEC
:10469000E06A08B90020F8E709A80090E76A29460F
:1046A0002046009B089AB8470646002000903046F6
:1046B000EBE7F0B504460D461E4600210027002317
:1046C000214600BF10E042F8331002EBC300476000
:1046D00002EBC3075B1C6868D1F804C0604502D1D7
:1046E00037600020F0BD49680029ECD1481EF9E789
:1046F0002DE9F0410546002700264FF6FF7000EA3D
:104700001547AEB20848046809E02088B84205D1D0
:1047100000223146204603F0B1FF02E06469002C1C
:10472000F3D100BFBDE8F081C80600202DE9F041BB
:1047300086B006460F464FF000080025002402A868
:1047400004AB12A239460090304605F0D3F8022897
:1047500003D0601E06B0BDE8F081DDE9020105F07E
:1047600060F800F0FF0804980578012403E004983D
:10477000005D4540641C0598A042F8D8454502D02C
:104780004FF0FF30E6E70020E4E700002425702A20
:1047900025700D0A0000000010B588B000F024FA62
:1047A00000F0D4FB00208DF805008DF804002248AD
:1047B00002904FF480600390204804904FF42060F2
:1047C00005900220069001A90BF024FAB0211C48A4
:1047D00005F006F81BA20A211948401C05F07DF9D6
:1047E0001749086219A20A2115480B3005F075F91E
:1047F0001349486217A20A211148153005F06DF9D6
:104800000F4988620120154908701548B0F8540016
:104810001349B1F8521040EA0124B4F5612F02D8CF
:10482000B4F5165F01D24FF4E134214602200BF0BB
:1048300075FB08B010BD0000F46E0020F47200207B
:10484000047D002024474E4747410000244750473D
:10485000535600002447424753560000920300205D
:104860009824002030B58FB004460D46282104A8B6
:10487000FBF706FD29462046FFF758FF18B14FF019
:10488000FF300FB030BD23482349244A244BCDE9E3
:104890000021029023A22946204605F02BF80F287C
:1048A00002D04FF0FF30ECE71A490868FBF755FDDE
:1048B000284908701849086800210CF009F82648B2
:1048C00080ED000B1549086800210CF001F8234821
:1048D00080ED000B0F490868FBF73FFD1D4908708C
:1048E000084600781E4908600846006838B10C4840
:1048F00000681C4902680A608088888007E01421EB
:104900001848FBF7BDFC174817A109780170002073
:10491000B7E700001C040020040400200C04002061
:104920002404002024252A2C25702C25702C252ACF
:104930002C25702C252A2C25702C252A2C252A2C58
:10494000252A2C252A2C252A2C252A2C252A2C25DB
:104950002A2A000090030020F0030020F803002022
:1049600000040020B47D00203000000070B596B037
:1049700004460D4628210CA8FBF782FC0AA808A9CA
:1049800006AA04ABCDE9002102903D4A2946204603
:1049900004F0B0FF15281AD13A480088001D3949A3
:1049A00008800498FBF7D9FC06460698FBF7D5FC6F
:1049B00006440898FBF7D1FC06440A98FBF7CDFCA7
:1049C00030443149098808442F49088054E008A838
:1049D00006A904AB2DA2CDE900102946204604F01B
:1049E00089FF112816D127480088C01C2549088056
:1049F0000498FBF7B2FC06460698FBF7AEFC0644AB
:104A00000898FBF7AAFC30441F49098808441E494E
:104A1000088031E006A804AB2AA22946009020466F
:104A200004F068FF0D2812D116480088801C154933
:104A300008800498FBF791FC06460698FBF78DFC6E
:104A400030441149098808440F49088014E004AB38
:104A500027A22946204604F04DFF09280CD1094819
:104A60000088401C074908800498FBF776FC06493B
:104A70000988084404490880002016B070BD000071
:104A8000202D03082E0400202C04002024252A2C8D
:104A9000252A2C252A2C252A2C252A2C252A2C258A
:104AA0002A2C25702C252A2C252A2C252A2C2570E9
:104AB0002C252A2C252A2C252A2C25702C252A2A1F
:104AC0000000000024252A2C252A2C252A2C252A02
:104AD0002C252A2C252A2C252A2C25702C252A2CFD
:104AE000252A2C252A2C25702C252A2A0000000096
:104AF00024252A2C252A2C252A2C252A2C252A2C2B
:104B0000252A2C252A2C25702C252A2A0000000075
:104B1000034B43F8301003EBC0039A80704700004A
:104B2000F47C00200EB500200290019000906946B0
:104B30000BF05CF82DE0FCF759FF012803D0FCF7DF
:104B400055FF022806D14FF47A73012201A900987B
:104B500003F0F5F89DF8040000F09AF89DF80410B1
:104B6000194802680068401C174B186017488154A8
:104B700018460068B0F5007F07D31846016813484F
:104B800006F0C6F800201049086004F021FD104925
:104B9000086001A902200AF06BFF02900028CAD029
:104BA0000948006870B104F013FD09490968401A0A
:104BB000322807D904480168044806F0A9F8002003
:104BC000014908600EBD000038040020C87D0020A7
:104BD0003C04002010B5034A91899068002201F03E
:104BE00005F910BDF47C002010B5034A9189906846
:104BF000012201F0FBF810BDF47C002010B5044642
:104C00001D480470012C06D0022C0FD0052C18D0A2
:104C10000A2C2CD120E00E22184902200BF014FBA4
:104C20001522174902200BF00FFB21E00E22154937
:104C300002200BF009FB1522114902200BF004FBA6
:104C400016E00E22104902200BF0FEFA15220C4944
:104C500002200BF0F9FA0BE00E220C4902200BF0B7
:104C6000F3FA1522064902200BF0EEFA00E000BF2D
:104C700000BF002010BD000091030020B103002000
:104C80009C030020BF030020CD030020DB03002095
:104C900030B589B004469F4AD2E900109268CDE948
:104CA000070206919B4A0C3207CA03AB07C3994A15
:104CB000183207CA8DE807009748007830B10128FC
:104CC00019D0022851D003287DD169E0242C11D1BC
:104CD0000120914908700020C1F8AC000846D0F8C6
:104CE000AC10D0F8AC00401C8B4AC2F8AC0002F10A
:104CF0002C0044540AE18848D0F8AC10D0F8AC003D
:104D0000401C854AC2F8AC0002F12C0044542C38F7
:104D1000D0F8AC001146096A884225D31046411CE0
:104D2000026A2C30FBF7F4FA18B902207A490870AD
:104D30001AE0794800F10B01426A2C30FBF7E8FADF
:104D400018B90220744908700EE0734800F115018B
:104D5000826A2C30FBF7DCFA18B902206E49087021
:104D600002E000206C490870D0E06B48D0F8AC102D
:104D7000D0F8AC00401C684AC2F8AC0002F12C002C
:104D800044542C38D0F8AC007F2803D300201146BF
:104D90000870BBE00D2C02D103205F490870B5E01C
:104DA0005D48D0F8AC10D0F8AC00401C5A4AC2F8AC
:104DB000AC0002F12C0044540A2C6FD15748007803
:104DC00040B9574800E0A0E0B0F8700055490978B4
:104DD000884207D0002051490870514991F870006D
:104DE000FFF70CFF4C4800F11501826A2C30FBF7ED
:104DF0008FFA28B94848D0F8AC102C30FFF7B6FD30
:104E00004548411C026A2C30FBF782FA00286CD11D
:104E10004148D0F8AC102C30FFF724FD00223E486A
:104E2000D0F8AC00801E3C492C310A543E48007832
:104E300078B100203C4908703C4908603C48036850
:104E40003C480268084601683B48006807F0D8FB08
:104E50004BE0012034490870384800683849097827
:104E600088420DD036480078042808D103A8FBF703
:104E70003AFA0546294603A809F088FA00BF00BFA0
:104E80002F48007806281CD2DFE800F003090D1B2C
:104E900012174FF408402549086017E031E08820D8
:104EA0002249086012E04FF08810204908600DE0A8
:104EB0004FF408001D49086008E022481B490860BB
:104EC00004E0204888301949086000BF00BF184836
:104ED000036818480268154801681748006807F019
:104EE0008FFB174800781549086004F071FB1649DC
:104EF0000968401AB0F57A7F03D304F069FB1249C0
:104F0000086000200449087000E000BF00BF09B03D
:104F100030BD0000DC250308047D00209203002042
:104F2000982400209103002034040020680600200B
:104F3000700600206C06002064060020300400206B
:104F400090030020008888009403002010B50C4ACC
:104F500091881068012200F049FF0A2000F0B4FC9B
:104F6000074A91881068002200F040FF0A2000F0F4
:104F7000ABFC034A91881068012200F037FF10BD96
:104F8000F47C00202DE9F04F95B004468846154684
:104F900099460020009082462E46CB4600271CB141
:104FA000B8F1000F00D025B94FF0FF3015B0BDE8C3
:104FB000F08F4AE000203870142301AA3B213046CC
:104FC00004F0A2FD00900098122838D926A101987B
:104FD000FBF790F900B138E0BAF1000F14D1B246F6
:104FE00020212046029A04F078FD202104F12000BF
:104FF000039A04F072FD0C98FBF7AFF908B1012099
:1050000000E0002084F8400041460398FBF772F965
:10501000A8B920212046029A04F05FFD202104F166
:105020002000049A04F059FD0C98FBF796F908B19A
:10503000012000E0002084F840000020B6E7B81C02
:10504000801BABEB000BBE1C00BF5A4607A13046CD
:1050500004F09DFD071EADD1BAF1000F01D1401E35
:10506000A4E70020A2E70000535452000D0A0000FC
:1050700038B502460020009000BF92F83C0001289D
:1050800001D1022038BD012082F83C0000BF086831
:10509000092816D91068C0680C780A3C04EB44054E
:1050A0000724AC40A0431468E0600C780A3C04EB91
:1050B00044048868A0401468E46820431468E060F1
:1050C00013E0106800690C7804EB44050724AC4039
:1050D000A043146820610C7804EB44048868A04065
:1050E000146824692043146820614868072817D28F
:1050F0001068406B0C79641E04EB84051F24AC40DF
:10510000A04314686063088880B20C79641E04EBC5
:105110008404A0401468646B20431468606331E029
:1051200048680D2817D21068006B0C79E41F04EB57
:1051300084051F24AC40A04314682063088880B213
:105140000C79E41F04EB8404A0401468246B204312
:105150001468206316E01068C06A0C790D3C04EBFB
:1051600084051F24AC40A0431468E062088880B224
:105170000C790D3C04EB8404A0401468E46A2043DD
:105180001468E062194B1A4C1068A04206D10868F6
:10519000122803D1586840F480005860144C1068FD
:1051A000A0421CD10868102802D00868112816D126
:1051B000586840F400005860086810280FD10D4866
:1051C00000680D4CB0FBF4F000EB80004000009054
:1051D00002E00098401E009000980028F9D100BF1E
:1051E000002082F83C0000BF00BF4BE700230140D5
:1051F00000200140C406002040420F007047704765
:105200007047000070B5044600250CB9012070BD40
:105210001549A06A884200D000BF206C30B9002038
:10522000606484F83C00204600F020F8206C00F018
:10523000100088B9206C20F4885040F002002064EF
:105240002046FBF709FF00206064206C20F002007C
:1052500040F00100206400E0012500BF002084F838
:105260003C0000BF2846D2E70100000F10B586B011
:1052700004462149206888423CD100BF00200090AC
:105280001E48006840F480701C49086008460068A9
:1052900000F48070009000BF00BF02200190032046
:1052A00002900020039001A9154800F0ADFC1548BC
:1052B0001549086000204860002113488160C160E2
:1052C0004FF48061016149004161890081614911A8
:1052D000C1614FF4403101620021416200F02EFAB9
:1052E00018B17E2109A00BF08FFA00BF0648A06319
:1052F000846300BF06B010BD002001404438024066
:10530000000002401064024008E500202E2E2F53BA
:1053100072632F73746D3332663478785F68616CB2
:105320005F6D73702E630000F8B504460D46164697
:105330000020009000BF94F83C00012801D1022019
:10534000F8BD012084F83C0000BF2068806800F0B0
:105350000100A0B92068806840F0010021688860E1
:105360003C4800683C49B0FBF1F000EB4000009085
:1053700002E00098401E009000980028F9D12068B3
:10538000806800F00100002862D0206C40F20161CA
:10539000884340F4807020642068406800F4806096
:1053A00028B1206C20F4005040F480502064206C20
:1053B00000F4805020B1606C20F00600606401E0D1
:1053C0000020606400BF002084F83C0000BF234F31
:1053D0002348A16BC8632348A16B08642248A16BD2
:1053E000C8646FF02200216808602068406840F0BF
:1053F0008060216848602068806840F4807021687F
:105400008860226802F14C0133462A46A06B00F006
:105410000BFA786800F01F0058B92068806800F027
:10542000405028B92068806840F08040216888603A
:105430000EE00E49206888420AD12068806800F09A
:10544000405028B92068806840F08040216888601A
:10545000002075E7C406002040420F0000230140F1
:10546000790F020801100208E70F0208002001402E
:10547000014691F83500022803D0802048650120BC
:105480007047052081F835000868006820F00100A9
:105490000A6810600020F3E770B504460CB90120DB
:1054A00070BD94F83500022800D1F9E72068006843
:1054B00020F0010021680860002021680860216850
:1054C0004860216888602168C860216808612120DF
:1054D000216848612046FCF7EDFB054694F85C1016
:1054E0003F208840A8600020606584F8350000BF38
:1054F00084F8340000BF00BFD2E70000F8B50446CE
:10550000002000908C4800684FF41651B0FBF1F772
:10551000A56D2E6894F85C1008208840304098B142
:105520002068006800F0040070B12068006820F076
:1055300004002168086094F85C1008208840A86086
:10554000606D40F00100606594F85C1001208840B7
:10555000304068B12068406900F0800040B194F8A4
:105560005C1001208840A860606D40F0020060651A
:1055700094F85C1004208840304068B120680068CE
:1055800000F0020040B194F85C1004208840A8604C
:10559000606D40F00400606594F85C101020884055
:1055A000304078B32068006800F0080050B394F8E9
:1055B0005C1010208840A8602068006800F48020FB
:1055C00080B12068006800F4002028B9206CC8B1C0
:1055D0002046216C884715E0A06C98B12046A16C4C
:1055E00088470FE02068006800F4807028B92068C0
:1055F000006820F0080021680860206C10B1204687
:10560000216C884794F85C102020884030400028A6
:1056100065D02068006800F0100000285FD094F882
:105620005C1020208840A86094F83500052828D117
:105630002068006820F01600216808602068406932
:1056400020F0800021684861206C08B9A06C28B166
:105650002068006820F008002168086094F85C1059
:105660003F208840A86000BF002084F8340000BFBD
:10567000012084F83500206D10B12046216D884747
:10568000F8BD2068006800F4802080B120680068C0
:1056900000F4002028B9606C10B12046616C884786
:1056A0001DE0E06BD8B12046E16B884717E0206829
:1056B000006800F4807068B92068006820F010006D
:1056C0002168086000BF002084F8340000BF01207A
:1056D00084F83500E06B10B12046E16B8847606DBF
:1056E00038B3606D00F00100F0B1052084F835009A
:1056F0002068006820F001002168086000BF009861
:10570000401C0090B84200D905E02068006800F015
:1057100001000028F3D100BF00BF002084F834004E
:1057200000BF012084F83500E06C10B12046E16C28
:10573000884700BFA4E70000C40600202DE9F0411F
:105740000446002500F058FB074614B90120BDE8C7
:10575000F081606A00B100BF00BF002084F834000F
:1057600000BF022084F835002068006820F00100A6
:10577000216808600AE000F03FFBC01B052805D93E
:1057800020206065032084F83500E0E72068006889
:1057900000F001000028EED120680568214805408E
:1057A000D4E901010843E1680843216908436169BC
:1057B0000843A1690843E1690843216A0843054396
:1057C000606A042803D1D4E90B010843054320682B
:1057D00005602068456925F00705606A0543606A31
:1057E00004280DD1A06A0543E06A48B12046FCF7C1
:1057F0007BFA28B140206065012084F83500A6E7D7
:10580000206845612046FCF755FA064694F85C107E
:105810003F208840B06000206065012084F835009A
:10582000002094E73F8010F02DE9F04704460D4634
:1058300016461F464FF00008D4F8589000BF94F861
:105840003400012802D10220BDE8F087012084F84D
:10585000340000BF94F8350001282BD1022084F8D1
:105860003500002060653B46324629462046FCF75D
:1058700090FA94F85C103F208840C9F8080020682E
:10588000006840F01600216808602068406940F018
:10589000800021684861206C28B12068006840F0D1
:1058A0000800216808602068006840F00100216855
:1058B000086006E000BF002084F8340000BF4FF00D
:1058C00002084046C0E7000070B5044600F094FAB4
:1058D00006462546681C10B104480078054400BF00
:1058E00000F08AFA801BA842FAD370BDC0060020DF
:1058F0002DE9F04104460E460127002500BF25484A
:10590000007E012802D10220BDE8F081012021495A
:10591000087600BF4CF25030FEF748FE0746002FD5
:1059200031D1401E3060206801280FD1207C616891
:10593000FEF77AFD4CF25030FEF738FE0746164867
:10594000006820F00400144908601AE0A56812E01D
:10595000217C2846FEF7FEFC4CF25030FEF726FE76
:1059600007460D48006820F0FA000B4908600FB1A7
:10597000356005E06D1CD4E902100844A842E7D860
:1059800000BFFEF715FD00BF00200249087600BFEA
:105990003846B9E738E90020103C02402DE9F041D3
:1059A00006460F4614461D464FF0010800BF1F482B
:1059B000007E012802D10220BDE8F08101201B49B0
:1059C000087600BF4CF25030FEF7F0FD8046B8F18B
:1059D000000F23D126B9E1B23846FEF73DFD12E0B3
:1059E000012E04D1A1B23846FEF75EFD0BE0022E77
:1059F00004D121463846FEF76BFD04E022462B46D3
:105A00003846FEF73BFD4CF25030FEF7CFFD8046A6
:105A10000748006820F001000549086000BF002029
:105A20000249087600BF4046C6E7000038E900207A
:105A3000103C024000200949096801F0004159B1B9
:105A40000749064A0C3A1160064911600349096882
:105A500001F0004101B1012070470000103C0240FC
:105A600023016745AB89EFCDF0B50C460025002238
:105A70000023002181E0012606FA01F504EA05026F
:105A8000AA4279D106684FEA410C032707FA0CF7BE
:105A9000BE430660CF0800F1200656F827604F0786
:105AA0004FEAD76C0F2707FA0CF7BE434FEAD10C29
:105AB00000F1200747F82C6086684FEA410C032765
:105AC00007FA0CF7BE438660476801268E40B7434D
:105AD0004760C6684FEA410C032707FA0CF7BE433C
:105AE000C660284E8F0856F827308E07370F0F26CE
:105AF000BE403340244EB04201D1002614E0234E74
:105B0000B04201D101260FE0214EB04201D1022660
:105B10000AE0204EB04201D1032605E01E4EB042FD
:105B200001D1042600E007268F073F0FBE409E42AA
:105B300022D18E07370F0F2606FA07F3114E8F0872
:105B400056F827609E430F4F4FEA910C47F82C60A0
:105B5000124E36689643114F3E603E1D366896439E
:105B60003F1D3E603E1D366896433F1D3E603E1D14
:105B7000366896433F1D3E60491C1029FFF47BAFF9
:105B8000F0BD00000838014000000240000402405F
:105B900000080240000C024000100240003C01409E
:105BA00010B50446B4F5805F01D105F03FFB012C30
:105BB00004D19FED0B0A0B4880ED000AB4F5007F7D
:105BC00004D10948007808B9FBF7A8FBB4F5007FB9
:105BD00005D105480078012801D109F0D7FE10BD94
:105BE000000000001C0600207701002010B50446CC
:105BF00004480068204020B1024804602046FFF7B6
:105C0000CFFF10BD143C0140F8B503460A460025FD
:105C1000002400200021CDE0012606FA01F51668D7
:105C200006EA0504AC4273D15668022E02D05668CB
:105C3000122E13D1CF0803F1200656F827004E0785
:105C4000F70E0F26BE40B0434F07FF0E1669BE4049
:105C50003043CF0803F1200646F8270018684F00AC
:105C60000326BE40B043167906F003064F00BE403F
:105C7000304318605668012E08D05668022E05D0B1
:105C80005668112E02D05668122E13D198684F0014
:105C90000326BE40B0434F00D668BE4030439860F4
:105CA000586801268E40B0431679C6F300168E4020
:105CB00030435860D8684F000326BE40B0434F00C1
:105CC0009668BE403043D860566806F08056B6F1FC
:105CD000805F6ED100BF00260096384E366846F4CD
:105CE0008046364F3E603E46366806F48046009653
:105CF00000BF00BF324E8F0856F827008E07370FBF
:105D00000F26BE40B0432F4EB34202D1002615E00D
:105D10004FE02D4EB34201D101260FE02B4EB3428E
:105D200001D102260AE02A4EB34201D1032605E042
:105D3000284EB34201D1042600E007268F073F0F0B
:105D4000BE4030431E4E8F0846F82700224E306872
:105D5000A043566806F48036B6F5803F00D1204354
:105D60001D4E3060361D3068A043566806F400367C
:105D7000B6F5003F00D12043174E361D3060361D6A
:105D80003068A043566806F48016B6F5801F00D12F
:105D90002043114E08363060361D3068A0435668E7
:105DA00006F40016B6F5001F00D120430A4E0C364B
:105DB0003060491C1029FFF42FAFF8BD4438024071
:105DC0000838014000000240000402400008024080
:105DD000000C024000100240003C014002461369E2
:105DE0000B400BB1012000E0002070470AB1816137
:105DF00001E00B04836170470148006870470000B0
:105E0000B80600200348006803490978084401499E
:105E100008607047B8060020C006002010B50D4885
:105E2000006840F400700B4908600846006840F4C0
:105E3000806008600846006840F4807008600320B5
:105E400000F0B6F8002000F007F800F02BF8002072
:105E500010BD0000003C024070B504460E480078BA
:105E60004FF47A71B1FBF0F00C490968B1FBF0F521
:105E7000284600F090FF08B1012070BD102C07D219
:105E800000222146501E00F054F80548046001E04D
:105E90000120F2E70020F0E7C0060020C406002041
:105EA000BC06002010B5032000F082F80022114645
:105EB0006FF00B0000F03DF8002211466FF00A0071
:105EC00000F037F8002211466FF0090000F031F8B9
:105ED00000221146501F00F02CF800221146101F1E
:105EE00000F027F800221146901E00F022F8002250
:105EF0001146501E00F01DF810BD000000BF00F05C
:105F00001F0201219140034A430942F8231000BFB8
:105F10007047000080E100E000BF00F01F02012197
:105F200091404209920002F1E022C2F8001100BF44
:105F300070472DE9F05F80460D461646002704F0B5
:105F4000DDFF074639462A46334601F00700C0F117
:105F5000070ABAF1040F02D94FF0040A01E0C0F1B8
:105F6000070AD14600F1040ABAF1070F02D24FF036
:105F7000000A01E0A0F1030AD4464FF0010A0AFA30
:105F800009FAAAF1010A0AEA020A0AFA0CFA4FF01F
:105F9000010B0BFA0CFBABF1010B0BEA030B4AEA0A
:105FA0000B042146404604F0B1FFBDE8F09F00001D
:105FB00000BF00F00702064B19684FF6FF031940B7
:105FC000044B0B4343EA0221014B196000BF7047A9
:105FD0000CED00E00000FA050D4A126822F0030201
:105FE00002430B4B1A600B4A126842F00402094B41
:105FF0001A60012901D130BF02E040BF20BF20BF9D
:10600000044A126822F00402024B1A607047000032
:106010000070004010ED00E070B504460D460CB96C
:10602000012070BD5848006800F00F00A84209D256
:1060300055490D700846006800F00F00A84201D0D5
:106040000120EEE7207800F0020002281DD1207820
:1060500000F00400042805D14C48006840F4E050EA
:106060004A490860207800F00800082805D1474810
:10607000006840F46040454908604448006820F0EA
:10608000F000A168084341490860207800F0010051
:10609000A8B36068012807D13C4808380068C0F3FD
:1060A0004040B8B90120BCE76068022802D06068AF
:1060B000032807D1354808380068C0F3406048B964
:1060C0000120AEE7314808380068C0F3400008B945
:1060D0000120A6E72D48006820F00300616808430E
:1060E0002A490860FFF788FE064609E0FFF784FEAC
:1060F000801B41F28831884202D9032091E707E0F2
:106100002248006800F00C006168B0EB810FEDD10F
:106110001D48006800F00F00A84209D91A490D7007
:106120000846006800F00F00A84201D0012078E77F
:10613000207800F00400042807D11448006820F4F7
:10614000E050E168084311490860207800F0080039
:10615000082808D10D48006820F46040216940EA11
:10616000C1000A49086000F03DF808490968C1F318
:106170000311074A515CC840064908600020FFF738
:106180006BFE00204DE70000003C02400838024052
:10619000FE2A0308C406002001480068704700007A
:1061A000C406002000B5FFF7F7FF04490968C1F3F2
:1061B0008221034A515CC84000BD000008380240FB
:1061C0000E2B030800B5FFF7E7FF04490968C1F388
:1061D0004231034A515CC84000BD0000083802400B
:1061E0000E2B03082DE9F047002400250026A146C8
:1061F0002548006800F00C0020B1042805D00828CC
:106200003AD105E0DFF8849039E0DFF8849036E099
:106210001D48001F006800F03F041B48001F006875
:1062200000F4800078B11A481749091F0968C1F3C2
:106230008811A0FB01700146224600233846F9F779
:10624000C5FF05460EE011480F49091F0968C1F353
:106250008811A0FB01700146224600233846F9F759
:10626000B5FF05460848001F0068C0F30140401C08
:106270004600B5FBF6F902E0DFF8109000BF00BF62
:106280004846BDE8F0870000083802400024F400CA
:1062900000127A00F8B504460CB90120F8BD207848
:1062A00000F00100002874D0F948006800F00C00EC
:1062B00004280DD0F648006800F00C00082813D11F
:1062C000F348001F006800F48000B0F5800F0BD188
:1062D000EF4808380068C0F34040002859D0606893
:1062E000002856D10120D9E700BF6068B0F5803F93
:1062F00008D1E7480838006840F48030E44908399C
:1063000008601EE06068B0F5A02F0DD1E0480838A5
:10631000006840F48020DE490839086008460068BB
:1063200040F4803008600CE0D9480838006820F458
:106330008030D749083908600846006820F480207A
:10634000086000BF606890B1FFF756FD054606E0A3
:10635000FFF752FD401B642801D903209EE7CC487B
:1063600008380068C0F340400028F1D011E0FFF782
:1063700043FD054606E0FFF73FFD401B642801D9B9
:1063800003208BE7C24808380068C0F3404000286B
:10639000F1D1207800F0020002285FD1BC480068EB
:1063A00000F00C0058B1BA48006800F00C00082852
:1063B0001CD1B748001F006800F48000B0B9B44891
:1063C00008380068C0F3400020B1E068012801D01F
:1063D000012063E7AE480838006820F0F800216922
:1063E00040EAC100AA490839086037E0E06800B314
:1063F0000120A8490860FFF7FFFC054606E0FFF70B
:10640000FBFC401B022801D9032047E7A0480838BD
:106410000068C0F340000028F1D09D4808380068AB
:1064200020F0F800216940EAC10099490839086064
:1064300014E0002097490860FFF7DEFC054606E0FF
:10644000FFF7DAFC401B022801D9032026E7904819
:1064500008380068C0F340000028F1D1207800F02F
:10646000080008282CD16069A8B101208A49086079
:10647000FFF7C2FC054606E0FFF7BEFC401B022802
:1064800001D903200AE782486C300068C0F340005D
:106490000028F1D014E000207F490860FFF7ACFC31
:1064A000054606E0FFF7A8FC401B022801D903209F
:1064B000F4E677486C300068C0F340000028F1D162
:1064C000207800F00400042870D10026704838308D
:1064D000006800F0805090B900BF002000906C4828
:1064E0003830006840F0805069493831086008460B
:1064F000006800F08050009000BF00BF0126674890
:10650000006800F48070B0B96448006840F480709E
:1065100062490860FFF770FC054606E0FFF76CFC77
:10652000401B022801D90320B8E65C48006800F44B
:1065300080700028F2D000BFA068012808D154481C
:106540006830006840F001005149683108601DE082
:10655000A06805280DD14E486830006840F004005E
:106560004B49683108600846006840F00100086047
:106570000CE047486830006820F001004449683169
:1065800008600846006820F00400086000BFA068AA
:10659000A8B1FFF731FC054609E0FFF72DFC401BD1
:1065A00041F28831884202D9032077E626E0384854
:1065B00068300068C0F340000028EED013E0FFF719
:1065C0001BFC054608E0FFF717FC401B41F2883131
:1065D000884201D9032061E62D4868300068C0F385
:1065E00040000028EFD1012E07D12948383000683B
:1065F00020F0805026493831086000BFA069B8B348
:106600002348006800F00C0008285ED0A06902282A
:1066100046D100201F490866FFF7EEFB054606E05D
:10662000FFF7EAFB401B022801D9032036E6184891
:1066300008380068C0F340600028F1D1D4E90701B0
:106640000843616A40EA81110122A06AC2EB50004E
:1066500041EA00412C20005D41EA00600C49091F1D
:10666000086001200B490866FFF7C6FB054607E0F6
:106670002DE0FFF7C1FB401B022801D903200DE6E6
:10668000034808380068C0F340600028F1D01EE0DD
:106690000838024000004742800E47420070004028
:1066A00000200C490866FFF7A7FB054606E0FFF748
:1066B000A3FB401B022801D90320EFE50648006830
:1066C000C0F340600028F2D101E00120E6E500209F
:1066D000E4E5000000004742003802404FF0E020AF
:1066E000006940F002004FF0E0210861704710B5EA
:1066F00004460CB9012010BD022084F85100206826
:10670000006820F0400021680860204600F050F842
:106710000020606584F8510000BF84F8500000BF7D
:1067200000BFE8E710B504460CB9012010BD606A4F
:1067300000B900BF0021A16294F8510028B90020DF
:1067400084F85000204600F04BF8022084F85100F5
:106750002068006820F0400021680860D4E9010149
:106760000843E16808432169084361690843218BB4
:1067700001F400710843E1690843216A0843A16AF2
:106780000843216808600421A06901EA1040616A99
:106790000843216848602068C06920F400602168CF
:1067A000C86100206065012084F851000020BDE729
:1067B00010B5044607492068884209D10648006898
:1067C00020F4805004490860E0210448FFF74CF9A8
:1067D00010BD00000030014044380240000002407B
:1067E00010B586B004461249206888421DD100BF0A
:1067F000002000900F48006840F480500D49086068
:106800000846006800F48050009000BF00BFE02000
:1068100001900220029000200390032004900520A4
:10682000059001A90448FFF7EFF906B010BD00007C
:106830000030014044380240000002402DE9F84396
:1068400004460D4617461E464FF00008C1466068D4
:10685000B0F5827F0DD1A06858B9042084F85100AA
:106860003B462A4629462046009600F070F9BDE8CE
:10687000F88300BF94F85000012801D10220F6E708
:10688000012084F8500000BFFFF7B6FA804694F864
:106890005100012802D04FF002097BE005B117B981
:1068A0004FF0010976E0042084F851000020606573
:1068B000A563A787E7872063A086E08620646064DD
:1068C000A068B0F5004F05D12068006820F4804032
:1068D000216808602068006800F04000402805D06A
:1068E0002068006840F0400021680860E068E8B96E
:1068F00018E02068806800F0010038B12068007B53
:1069000028706D1CE08F401EE0870BE03EB1701CCC
:1069100040B1FFF771FAA0EB0800B04202D34FF08C
:10692000030937E0E08F0028E3D11CE018E020687D
:10693000806800F0010038B12068C0682880AD1C74
:10694000E08F401EE0870BE03EB1701C40B1FFF7C6
:1069500053FAA0EB0800B04202D34FF0030919E04C
:10696000E08F0028E3D16068B0F5827F0DD1A06888
:10697000B0F5004F03D0A068B0F5806F05D1206856
:10698000006820F0400021680860606D08B14FF099
:10699000010900BF012084F8510000BF002084F8E5
:1069A000500000BF484662E72DE9F84304460D4613
:1069B00017461E464FF00008C14600BF94F850002D
:1069C000012802D10220BDE8F883012084F850009C
:1069D00000BFFFF711FA804694F85100012802D059
:1069E0004FF00209A9E005B117B94FF00109A4E081
:1069F000032084F85100002060652563A786E786A0
:106A0000A063A087E08760642064A068B0F5004FB1
:106A100005D12068006840F4804021680860206843
:106A2000006800F04000402805D02068006840F071
:106A3000400021680860E068B0F5006F2AD1606806
:106A400010B1E08E012806D128882168C860AD1CED
:106A5000E08E401EE08619E02068806800F00200A9
:106A6000022807D128882168C860AD1CE08E401E2E
:106A7000E0860BE03EB1701C40B1FFF7BDF9A0EB22
:106A80000800B04202D34FF0030956E0E08E002820
:106A9000E2D129E0606810B1E08E012806D12878A3
:106AA000216808736D1CE08E401EE08619E02068A6
:106AB000806800F00200022807D128782168087356
:106AC0006D1CE08E401EE0860BE03EB1701C40B1B4
:106AD000FFF792F9A0EB0800B04202D34FF0030990
:106AE0002BE0E08E0028E2D133460122022120462D
:106AF000CDF8008005F09AFC10B14FF003091CE0BE
:106B000042463146204605F059FC20B14FF00109BC
:106B10002020606511E0A06850B900BF00200090FF
:106B20002068C068009020688068009000BF00BFA7
:106B3000606D08B14FF0010900BF012084F85100D9
:106B400000BF002084F8500000BF48463BE72DE915
:106B5000FE4F04460D4616461F46DDF830804FF0C6
:106B6000000A0020029081464FF0010B019000BF07
:106B700094F85000012802D10220BDE8FE8F0120C8
:106B800084F8500000BFFFF737F9814694F851A010
:106B900060680290BAF1010F0BD00298B0F5827FC5
:106BA00004D1A06810B9BAF1040F02D002200190FC
:106BB000D2E00DB106B117B901200190CCE094F8F4
:106BC0005100012802D1052084F8510000206065A1
:106BD000A663E787A7872563E786A78620646064A6
:106BE0002068006800F04000402805D02068006858
:106BF00040F0400021680860E068B0F5006F43D1C4
:106C0000606810B1E08E012806D128882168C8602C
:106C1000AD1CE08E401EE0862FE0BBF1000F10D0CF
:106C2000E08E70B12068806800F00200022808D170
:106C300028882168C860AD1CE08E401EE0864FF0B9
:106C4000000BE08F68B12068806800F0010040B15F
:106C50002068C0683080B61CE08F401EE0874FF08F
:106C6000010B08F1010040B1FFF7C6F8A0EB0900E5
:106C7000404502D3032001906EE0E08E0028CCD185
:106C8000E08F0028C9D142E0606810B1E08E012891
:106C900006D12878216808736D1CE08E401EE086BE
:106CA0002FE0BBF1000F10D0E08E70B1206880683B
:106CB00000F00200022808D115F8010B21680873C2
:106CC000E08E401EE0864FF0000BE08F68B1206838
:106CD000806800F0010040B12068C06806F8010B30
:106CE000E08F401EE0874FF0010B08F1010040B13A
:106CF000FFF782F8A0EB0900404502D30320019082
:106D00002AE0E08E0028CCD1E08F0028C9D143468C
:106D1000012202212046CDF8009005F087FB10B13A
:106D20000320019018E04A464146204605F046FB04
:106D300020B101200190202060650DE0A06850B9CD
:106D400000BF002000902068C06800902068806824
:106D5000009000BF00BF00BF012084F8510000BFB9
:106D6000002084F8500000BF019806E7042808D1ED
:106D70004FF0E021096941F004014FF0E022116178
:106D800007E04FF0E021096921F004014FF0E02213
:106D900011617047704770B504462546681EB0F112
:106DA000807F01D301200FE0681E4FF0E021486191
:106DB0000F214FF0FF3004F0A9F800204FF0E02140
:106DC000886107200861002070BD10B5FFF7E2FF61
:106DD00010BD4FF0E020006920F002004FF0E021EC
:106DE000086170477047704710B50346002200BF26
:106DF00093F83800012801D1022010BD012083F84A
:106E0000380000BF22F0FF00CC6840EA040222F400
:106E100040708C6840EA040222F480604C6840EACA
:106E2000040222F400600C6840EA040222F480505C
:106E30000C6940EA040222F400504C6940EA040262
:106E400022F480408C6940EA040222F400408C69FC
:106E500040EA04021868426400BF002083F838004A
:106E600000BF00BFC9E7024600BF92F83800012802
:106E700001D102207047012082F8380000BF0220B3
:106E800082F839001068406820F07000136858607C
:106E9000106840680B681843136858601068806871
:106EA00020F0800013689860106880684B68184371
:106EB00013689860012082F8390000BF002082F832
:106EC000380000BF00BFD5E710B50446022084F8A3
:106ED000390000BF2068006A41F21111084050B922
:106EE0002068006A8910084028B92068006820F0EE
:106EF00001002168086000BF204600F023F8002050
:106F000084F8390000BF84F8380000BF10BD10B508
:106F100004460CB9012010BD94F8390028B90020AE
:106F200084F83800204600F021F8022084F8390067
:106F3000211D206807F056F8012084F83900002050
:106F4000E9E7000010B5044606492068884208D1E8
:106F50000548006820F00200034908601D20FEF784
:106F6000CDFF10BD000400404038024038B5044653
:106F70000E492068884217D100BF002000900C48BD
:106F8000006840F002000A4908600846006800F006
:106F90000200009000BF00BF002211461D20FEF736
:106FA000C8FF1D20FEF7B8FF38BD000000040040F8
:106FB0004038024001460868C06840F001000A6895
:106FC000D0600868006840F001000A681060002086
:106FD000704701460868C06820F001000A68D06068
:106FE00000BF0868006A41F21112104050B90868E9
:106FF000006A9210104028B90868006820F001006B
:107000000A68106000BF002070472DE9F041044677
:107010000D46002600BF94F83800012802D1022056
:10702000BDE8F081012084F8380000BF022084F818
:1070300039002068866826F0770626F47F462068A7
:107040008660286850283BD00CDC202860D004DC07
:10705000002853D0102865D155E030285DD0402855
:1070600060D141E0602835D070280DD0B0F5805F48
:1070700003D0B0F5005F55D115E02068806820F09E
:107080000700216888604EE0D5E902136A6820682D
:1070900007F00EF82068866826F0770646F0770637
:1070A000206886603FE0D5E902136A68206806F030
:1070B000FFFF2068806840F480402168886032E0EB
:1070C000EA686968206807F0D5F85021206806F062
:1070D000FBFF28E0EA686968206807F0E0F86021B3
:1070E000206806F0F1FF1EE0EA686968206807F092
:1070F000C1F84021206806F0E7FF14E00021206875
:1071000006F0E2FF0FE01021206806F0DDFF0AE044
:107110002021206806F0D8FF05E03021206806F025
:10712000D3FF00E000BF00BF012084F8390000BF9A
:10713000002084F8380000BF00BF71E7704710B529
:10714000044620680069C0F34000D8B12068C068D8
:10715000C0F34000B0B16FF0020021680861012067
:1071600020762068806900F0030018B12046FFF700
:10717000E5FF05E0204600F0C7F8204600F07EF964
:107180000020207620680069C0F38000D8B1206814
:10719000C068C0F38000B0B16FF0040021680861DE
:1071A000022020762068806900F4407018B12046E3
:1071B000FFF7C4FF05E0204600F0A6F8204600F0E7
:1071C0005DF90020207620680069C0F3C000D8B1C6
:1071D0002068C068C0F3C000B0B16FF0080021683B
:1071E0000861042020762068C06900F0030018B10F
:1071F0002046FFF7A3FF05E0204600F085F8204673
:1072000000F03CF90020207620680069C0F30010EF
:10721000D8B12068C068C0F30010B0B16FF01000A2
:1072200021680861082020762068C06900F4407059
:1072300018B12046FFF782FF05E0204600F064F811
:10724000204600F01BF9002020762068006900F03D
:10725000010058B12068C06800F0010030B16FF043
:10726000010021680861204600F068F92068006983
:10727000C0F3C01058B12068C068C0F3C01030B16E
:107280006FF08000216808612046FFF7ABFD2068A1
:107290000069C0F3801058B12068C068C0F3801046
:1072A00030B16FF0400021680861204600F0D2F94B
:1072B00020680069C0F3401058B12068C068C0F36E
:1072C000401030B16FF02000216808612046FFF7C0
:1072D0008AFD10BD10B586B0044609492068884271
:1072E0000CD1C01401900220029000200390049061
:1072F0000120059001A90348FEF786FC06B010BDE9
:107300000000014000000240704770B504460D4681
:10731000164600BF94F83800012801D1022070BD44
:10732000012084F8380000BF022084F8390036B10B
:10733000042E1BD0082E31D00C2E5ED145E02946FC
:10734000206806F0CBFE2068806940F008002168C4
:1073500088612068806920F00400216888612068C5
:107360008069296908432168886147E029462068C7
:1073700006F0E6FE2068806940F4006021688861BC
:107380002068806920F480602168886120688069B5
:10739000296940EA0120216888612FE02946206898
:1073A00006F006FF2068C06940F008002168C86147
:1073B0002068C06920F004002168C8612068C069A5
:1073C000296908432168C86118E02946206806F049
:1073D00025FF2068C06940F400602168C86120680A
:1073E000C06920F480602168C8612068C06929698B
:1073F00040EA01202168C86100E000BF00BF012011
:1074000084F8390000BF002084F8380000BF00BFB6
:1074100085E710B504460CB9012010BD94F8390079
:1074200028B9002084F83800204600F00DF802202A
:1074300084F83900211D206806F0D4FD012084F86D
:1074400039000020E9E7000008B50A4A01689142C6
:107450000FD100BF002100910749096841F00101E7
:10746000054A11601146096801F00101009100BF51
:1074700000BF08BD000001404438024070470000D2
:1074800030B504460D4601222946206806F002FE6A
:107490000A492068884201D1012000E0002028B17B
:1074A0002068406C40F4004021684864206800680F
:1074B00040F0010021680860002030BD000001405C
:1074C00030B504460D4600222946206806F0E2FD4C
:1074D00019492068884201D1012000E0002090B1C4
:1074E00000BF2068006A41F21111084050B92068BD
:1074F000006A8910084028B92068406C20F40040D8
:107500002168486400BF00BF2068006A41F2111181
:10751000084050B92068006A8910084028B92068DE
:10752000006820F001002168086000BF012084F895
:107530003900002030BD00000000014010B50446B5
:1075400035480088401C3449088034480078401C85
:107550003249087030480088B0F57A7F51DB00204E
:107560002D4908802E480088401C2D4908802D4850
:1075700090ED000AF7EE000A30EE200A80ED000AD6
:10758000012029490870264800880A2821DDFAF7D9
:107590002DFA03281DD000BF00BF00BF00BF00BFF1
:1075A000BFF34F8F00BF00BF00BF2048006800F44A
:1075B000E0601F490843001D1C49086000BF00BF70
:1075C00000BFBFF34F8F00BF00BF00BF00BF00BFB1
:1075D000FDE71848B0F8580098B94FF40071164804
:1075E000FEF7FCFB68B1FAF701FA032809D013484B
:1075F000036813480268134801681348006804F0E0
:10760000FFFF0548008811490968884202D101201E
:107610000F49087010BD00001C000020200600204B
:107620001E0000201C060020200000200CED00E0C1
:107630000000FA0598240020000402407006002093
:107640006C06002068060020640600203C01002033
:10765000D9010020704710B504460CB9012010BDB7
:10766000242084F83900204600F0F2F80020E0637E
:1076700084F8390084F83A0000BF84F8380000BF6D
:1076800000BFECE710B50446204608F043FD10BDEE
:107690002DE9F0470446206805682068C668206820
:1076A00047694FF00008C14605F00F08B8F1000F18
:1076B0000AD105F0200038B106F0200020B12046A4
:1076C00006F0B4FFBDE8F087B8F1000F6DD007F009
:1076D000010018B906F49070002866D005F001008A
:1076E00030B106F4807018B1E06B40F00100E06347
:1076F00005F0040030B107F0010018B1E06B40F074
:107700000200E06305F0020030B107F0010018B19B
:10771000E06B40F00400E06305F0080030B107F0D2
:10772000010018B1E06B40F00800E063E06B68B363
:1077300005F0200028B106F0200010B1204606F028
:1077400075FF20684069C0F38019E06B00F0080005
:1077500010B9B9F1000F22D0204606F03DFF206895
:10776000406900F04000B0B12068406920F040005E
:1077700021684861606B50B11748616B0865606BA8
:10778000FDF776FE10B1606B016D88470CE0204676
:10779000FFF778FF08E02046FFF774FF04E020467B
:1077A000FFF770FF0020E0638CE705F0800030B148
:1077B00006F0800018B1204607F03AF982E705F09C
:1077C000400030B106F0400018B1204606F014FF2A
:1077D00078E700BF76E70000DDE4020810B5044654
:1077E0000CB9012010BDA06900B100E000BF94F801
:1077F000390028B9002084F83800204600F082F8CB
:10780000242084F839002068C06820F400502168E2
:10781000C860204606F058FF2068006920F49040B8
:10782000216808612068406920F02A0021684861C9
:107830002068C06840F400502168C8600020E06300
:10784000202084F8390084F83A000020CAE70000BC
:1078500010B5044625492068884214D124480068A0
:1078600020F01000224908604FF4C0612148FEF763
:10787000FBF8606BFDF710FE206BFDF70DFE252079
:10788000FEF73CFB30E01C492068884215D11848BF
:10789000001F006820F400301549091F08600C2102
:1078A0001448FEF7E1F8606BFDF7F6FD206BFDF77D
:1078B000F3FD2620FEF722FB16E0104920688842DF
:1078C00012D10B48006820F0200009490860C0214F
:1078D0000B48FEF7C9F8606BFDF7DEFD206BFDF786
:1078E000DBFD4720FEF70AFB10BD00000010014041
:1078F00044380240000002400044004000140140AF
:107900000008024010B586B00446AA4920688842A3
:107910006CD100BF00200090A748006840F0100024
:10792000A54908600846006800F01000009000BFFC
:1079300000BF4FF4C060019002200290012003902C
:10794000032004900720059001A99C48FEF75CF9EC
:107950009B489C4908604FF00060486000219948AE
:107960008160C1604FF480610161002141618161EA
:107970004FF48071C161002101624162FDF7DEFEBA
:1079800020B140F2651190A008F03EFF00BF8D4885
:107990006063846300BF8A487830924908604FF082
:1079A0000060486040218F4881600021C1604FF431
:1079B00080610161002141618161C16101624162B7
:1079C000FDF7BCFE20B140F277117FA008F01CFF4C
:1079D00000BF84482063846300BF0022012125206A
:1079E000FEF7A7FA2520FEF797FAE0E07E49206827
:1079F00088426DD100BF002000906F48001F0068D2
:107A000040F400306C49091F08600846006800F423
:107A10000030009000BF00BF0C20019002200290B7
:107A200001200390032004900720059001A96348DA
:107A3000FEF7EAF86D486E4908604FF00060486054
:107A400000216B488160C1604FF4806101610021B9
:107A5000416181614FF48071C16100210162416225
:107A6000FDF76CFE20B14FF4D27157A008F0CCFEA8
:107A700000BF5F486063846300BF5C4818305D49A5
:107A800008604FF00060486040215A488160002142
:107A9000C1604FF480610161002141618161C16178
:107AA00001624162FDF74AFE20B14FF4DB7146A04E
:107AB00008F0AAFE00BF4F482063846300BF002285
:107AC00001212620FEF735FA2620FEF725FA6EE082
:107AD0004949206888426AD100BF0020009036489A
:107AE000006840F02000344908600846006800F053
:107AF0002000009000BF00BFC02001900220029033
:107B000001200390032004900820059001A93B4820
:107B1000FEF77AF82A481838394908608005486025
:107B2000002137488160C1604FF48061016100210C
:107B3000416181614FF48071C16100210162416244
:107B4000FDF7FCFD20B140F2E3111FA008F05CFE40
:107B500000BF2B486063846300BF19486030294927
:107B600008604FF020604860402126488160002175
:107B7000C1604FF480610161002141618161C16197
:107B800001624162FDF7DAFD20B140F2F5110EA06D
:107B900008F03AFE00BF1B482063846300BF002248
:107BA00001214720FEF7C5F94720FEF7B5F906B0D9
:107BB00010BD0000001001404438024000000240A7
:107BC00040640240F8E600202E2E2F5372632F737C
:107BD000746D3332663478785F68616C5F6D737092
:107BE0002E63000058E700200044004088600240F7
:107BF000B8E7002018E80020001401400008024007
:107C000078E80020D8E8002077B581B00446154612
:107C100094F83A00202850D1029800B115B90120FB
:107C200004B070BD00BF94F83800012801D10220D3
:107C3000F6E7012084F8380000BF0298A062A5850D
:107C40000020E063222084F83A001D48616BC8637D
:107C50001C48616B08641C48616BC8640020616B40
:107C6000086502AE32682368191D2B46606BFDF76C
:107C7000DBFD00BF002000902068006800902068B5
:107C80004068009000BF00BF00BF002084F83800AB
:107C900000BF2068C06840F480702168C860206818
:107CA000406940F00100216848612068406940F067
:107CB0004000216848610020B2E70220B0E70000E0
:107CC00041E5020887E50208F1E4020810B5034621
:107CD00093F83A00202829D101B10AB9012010BD3A
:107CE00000BF93F83800012801D10220F7E70120F6
:107CF00083F8380000BF99629A85DA850020D8633E
:107D0000222083F83A0000BF002083F8380000BF2B
:107D10001868406940F001001C6860611868C0681C
:107D200040F490701C68E0600020D8E70220D6E79D
:107D300010B50446204608F027FA10BD70472DE91B
:107D4000F84304460D4616461F464FF0000994F8C6
:107D5000390020285CD105B116B90120BDE8F883AF
:107D600000BF94F83800012801D10220F6E7012075
:107D700084F8380000BF0020E063212084F8390037
:107D8000FEF73AF88146A684E6842BE0E08C401E9C
:107D9000E084A068B0F5805F16D14B4600228021B8
:107DA0002046009706F078FE08B10320D6E7A846E3
:107DB000B8F80000C0F3080021684860206908B9DD
:107DC000AD1C0FE06D1C0DE04B46002280212046CB
:107DD000009706F061FE08B10320BFE715F8010B1C
:107DE00021684860E08C0028D0D14B460022402119
:107DF0002046009706F050FE08B10320AEE7202091
:107E000084F8390000BF002084F8380000BFA5E7DF
:107E10000220A3E7F7B50446154694F83900202858
:107E20003DD1019800B10DB90120FEBD00BF94F80D
:107E30003800012801D10220F7E7012084F838003A
:107E400000BF01982062A584E5840020E063212022
:107E500084F839001348216BC8631348216B086408
:107E60001248216BC8640020216B086501AE2368AD
:107E70001A1D31682B46206BFDF7D6FC6FF04000D1
:107E80002168086000BF002084F8380000BF206827
:107E9000406940F08000216848610020C5E7022069
:107EA000C3E7000095E50208CBE50208F1E402080B
:107EB00010B5034693F83900202823D101B10AB93F
:107EC000012010BD00BF93F83800012801D1022025
:107ED000F7E7012083F8380000BF19629A84DA843A
:107EE0000020D863212083F8390000BF002083F8E8
:107EF000380000BF1868C06840F080001C68E0606F
:107F00000020DEE70220DCE710B50446204608F03A
:107F100071FA10BD70472DE9FE4304460025A846BE
:107F200000260020029000270CB1606808B9BDE867
:107F3000FE83A068402800D9F9E700252CE0204600
:107F400000F0DEF82E464FF000081DE0606A825D0A
:107F500002AB4146204600F07CF90746022F0DD1C6
:107F6000606A0090E06A01906068029A00EBC200CB
:107F70006A464168204600F0A1F808E007B906E02B
:107F800000BF761C08F10108E06AB042DED800BFED
:107F9000022F00D103E06D1CE06AA842CFD800BFD9
:107FA00000BFC4E70FB438B504460D4607A80090DB
:107FB000D4E90601009B069A08F064FC20620020C8
:107FC000009008480078012803D1216AA06900F0D8
:107FD00047FB29462046236AA26900F00DF838BC09
:107FE0005DF814FBEC06002010B50446A06B01F010
:107FF000A9FA002010BD0000F8B504460D4616464B
:108000001F463A46314620466369984750B9204694
:10801000FFF7EAFF0094084B2A460021A06B01F00D
:1080200033FB06E00094054B01220021A06B01F018
:108030002BFB0020F8BD000081810208718102083D
:1080400070B504460D468021204601F0C9FB286822
:10805000E06368686060A868A060E868E06028691C
:10806000206168696061A869A061E869E061002039
:108070002062286A6062686AA0620020E06284F878
:108080003000A86A606304F1380001F071FA10B1A1
:108090004FF0FF3070BD204600F002F8FAE7000014
:1080A000014611B94FF0FF3070470348006808607F
:1080B000014801600020F7E7E806002070B504469B
:1080C0000D461646022D06D0032D05D0042D04D0F2
:1080D000052D07D102E000BF00BF00BF2046FFF71B
:1080E00083FF00E000BF00BF32462946E06B00F08E
:1080F000C5FA70BD0148007870470000EC0600200A
:1081000010B504460122402104F14000F8F7B1F80F
:1081100010BD000010B50024124804681EE020467F
:1081200021698847C8B910480078012810D1E16A50
:10813000606A01F0C5FB012803D1606A00F0B0F964
:1081400006E0E16A606A00F051FA08A000F0A8F9C0
:108150002046FFF7E0FE0020E0622468002CDED11C
:1081600010BD0000E8060020EC0600200D0A00000B
:1081700010B50446002205212046FFF79FFF10BDE1
:1081800010B50446002204212046FFF797FF10BDDA
:1081900070B504460D46204600F02FF8012801D1A5
:1081A000801E70BD2068401CE168B0FBF1F201FB4D
:1081B0001200206026692368A16803FB061032467E
:1081C0002946F8F744F80020EBE710B58160C2605B
:1081D0000361012444600024046010BD0146086866
:1081E000401CCA68B0FBF2F302FB13004A689042DD
:1081F00001D1012070470020FCE701460868801C7F
:10820000CA68B0FBF2F302FB13004A68904201D146
:10821000012070470020FCE770B504460D4620465B
:10822000FFF7DCFF012801D1801E70BD2669D4E96B
:10823000013003FB060132462846F8F708F860686B
:10824000401CE168B0FBF1F201FB1200606000200D
:10825000EBE7F0B504460D46002600211BE004F1D3
:108260004000405C012815D1606850F83100405D45
:10827000904204D0002704F1400047540AE0761CE5
:10828000606850F83170681C385C18B903B1196027
:108290000220F0BD491CA0688842E0D80EB9002039
:1082A000F7E70120F5E700002DE9F04104460D460F
:1082B0009C46002700210023344E15B9481EBDE816
:1082C000F0810320B5FBF0F800FB185020B9032023
:1082D000B5FBF0F0870004E00320B5FBF0F0401C94
:1082E0008700781C844502D24FF0FF30E7E700207A
:1082F000D055002100232AE0E05C06EBA0000078C6
:108300005054E05C80074FEA9068581C205C48EAB3
:10831000201016F80080481C02F80080581C205CD1
:1083200000074FEA9068981C205C48EAA01016F8F5
:108330000080881C02F80080981C205C00F03F0040
:1083400016F80080C81C02F80080DB1C091DB81E4E
:108350008842D1D80320B5FBF0F800FB1850012863
:1083600002D002280FD108E04FF03D08881E02F825
:108370000080481E02F8008005E04FF03D08481ECE
:1083800002F8008000BF00BF002098E7F43803081F
:1083900010B5024612B94FF0FF3010BD00BF106893
:1083A0008842FCD31068401A106050680844D368B3
:1083B000B0FBF3F403FB140050600020EDE710B5B0
:1083C000024612B94FF0FF3010BD1068084410602B
:1083D00000BFD36810689842FBD890680844D368FF
:1083E000B0FBF3F403FB140090600020ECE7F0B561
:1083F0000446002522B11BB1E6682068B04202D3D2
:108400004FF0FF30F0BD2668E068801B884202D242
:108410004FF0FF30F6E7A0680844E668B0420BD999
:10842000D4E90260851B2668E068801B4E19B042C3
:1084300002D24FF0FF30E5E7A0682844E668B0FBC1
:10844000F6F706FB17001060681818600020D9E7DF
:10845000014648687047014688687047024612B96D
:108460004FF0FF3070470020506090601060D16086
:1084700000BFF7E7014609B901207047086808B94D
:108480000120FAE70020F8E7014609B9012070470A
:108490000A68C868904201D10120F8E70020F6E799
:1084A0000FB410B5ADF5027DF9F7A0FA28B10020A0
:1084B0000DF5027D10BC5DF814FB002485A88190A9
:1084C0004FF4007101A8819B849A08F0DBF90446FF
:1084D00000208190B4F5007F01D340F2FF142246C2
:1084E00001A9002007F0B0FE0020E1E70FB410B5AD
:1084F000ADF5027D002485A881904FF4007101A89C
:10850000819B849A08F0BEF9044600208190B4F55E
:10851000007F01D340F2FF14224601A9002007F09A
:1085200093FE00200DF5027D10BC5DF814FB0000E9
:108530000FB430B5ADF5097DF9F758FA28B1002030
:108540000DF5097D30BC5DF814FB0024FDF754FCEB
:108550004FF47A71B0FBF1F201FB12059DF81E0099
:108560009DF81D109DF81C20CDE90405CDE90221E0
:108570009DF81B009DF81A10CDE90010BDF81830C9
:1085800011A24FF4007108A801F0A7FA0446224690
:1085900008A9002007F058FE8DA888904FF40071BC
:1085A00008A8889B8C9A08F06DF9044600208890F2
:1085B000B4F5007F01D340F2FF14224608A9002041
:1085C00007F042FE0020BBE7253034752D25303200
:1085D000752D2530327520253032753A25303275AB
:1085E0003A253032752E253033752000F0B591B024
:1085F00006460C46F9F7FAF910B1002011B0F0BDAB
:10860000002515480078012801D00020F6E700BFBA
:10861000102C01D9102500E02546402101A8F7F7CC
:108620002FFE0120402301AA29460090304601F088
:108630008BF80AA101A8F7F72EFE01A8F7F753FE61
:1086400007463A4601A9002007F0FEFD641B2E44B0
:10865000002CDDD10020D1E77C0300200D0A0000B2
:1086600070B504460D46F9F7C1F908B1002070BD98
:108670002A462146002007F0E7FDF8E72DE9FC41F6
:1086800004460D4617464FF0000800266088012872
:108690001FD1206950B960680068CDE900051AA2B1
:1086A00000212046E368FBF7E9FF12E0206950F85B
:1086B000250000782D280CD0206950F8250061682D
:1086C0000968CDE9001018A200212046E368FBF7F5
:1086D000D5FF66683A4629462046F36898478046A3
:1086E0000BE0706840B170683A462946C36820467E
:1086F00098478046766800E002E0B8F1010FF0D0BC
:1087000000BFBDE8FC81000046534D3A252D38736B
:108710002053544154453A252D323873204556454F
:108720004E543A25750D0A0046534D3A252D38739F
:108730002053544154453A252D323873204556452F
:108740004E543A25730D0A002DE9F04704460E46B3
:1087500017469846DDE9089A00250CB9BDE8F08770
:1087600030212046F7F78CFDC4F80890C4F810803B
:108770006660E7600021A16261620E480088208087
:10878000A4F802A00C48006860610B480460094826
:108790000088401C07490880656806E06560002283
:1087A00011462046FFF76AFFAD68002DF6D100BFE5
:1087B000D4E70000CC060020C8060020024612B90B
:1087C0004FF0FF307047D1620020FBE72DE9F843FE
:1087D00005460E4617461C46DDF820904FF000086F
:1087E0002188484661F31F408046054B3A46314692
:1087F0002846CDF8008000F047FFBDE8F883000070
:10880000F14602082DE9F04196B005460E4617469E
:10881000D5F80480002400201590444629E06C60BF
:10882000002201212846FFF729FFA64205D13A463A
:1088300000212846FFF722FF1DE0502101A8F7F78D
:108840001FFD15AB01AA21463046FBF732FF78B970
:108850000AE01598006868603A4600212846FFF74C
:108860000DFF15984068159015980028F1D102E089
:108870006468002CD3D100BFB46806E06C603A464F
:1088800000212846FFF7FAFEA468002CF6D116B0A6
:10889000BDE8F081016E05E000F17C024B1CD35C69
:1088A0005354491CC26D8A42F6D8704710B5C26D48
:1088B000511E05E000F17C02545C4B1CD454491E4F
:1088C000026E8A42F6DD10BD70B505460C46A879E9
:1088D00010B101282ED100E000BF432C1BD004DCD6
:1088E000412C0CD0422C22D10FE0442C19D07E2CEC
:1088F0001DD100220821284600F028FB18E00022A4
:108900000321284600F022FB12E000220421284621
:1089100000F01CFB0CE000220621284600F016FBAC
:1089200006E000220521284600F010FB00E000BF11
:1089300000BF2CE0432C1BD004DC412C0CD0422C7B
:1089400022D10FE0442C19D07E2C1DD10022082109
:10895000284600F07FF818E000220321284600F0A6
:1089600079F812E000220421284600F073F80CE0A8
:1089700000220621284600F06DF806E000220521BD
:10898000284600F067F800E000BF00BF00BF00BF4E
:1089900070BD70B504460D46432D45D008DC1B2D37
:1089A0000DD0332D24D0412D3CD0422D4CD13AE076
:1089B000442D3AD05B2D10D07E2D45D123E0207977
:1089C00010B1042804D100E000BF0120207102E0B2
:1089D0000020207100BF00BF39E02079012802D1BA
:1089E0000220207102E00020207100BF00BF2EE0B5
:1089F0002079022802D10320207102E0002020719A
:108A000000BF00BF23E02079032806D12946204675
:108A1000FFF75AFF0420207102E00020207100BF00
:108A200000BF14E000BF00BF00BF2079022806D1BC
:108A300029462046FFF748FF0420207102E000206D
:108A4000207100BF00BF02E00020207100BF00BF06
:108A5000207970BD2DE9F04104460D461746092DD9
:108A600002D00020A066E0660A2D6FD2DFE805F094
:108A70006E0540CDFDFCFBFAF9F8607910B10128D4
:108A800033D100E000BFE06D63282BD23846D4F824
:108A9000981588472046FFF709FF04F17C00216EF6
:108AA0004754206E401C2066E06D401CE065266E39
:108AB0004FF0000808E004F17C02905DD4F89815AE
:108AC0008847761C08F10108E06DB042F3D803E056
:108AD0000820D4F898158847B8F10000A8F10108DB
:108AE000F6D100BF0020607100E000BF00BF28E2A7
:108AF000E06D20B9FEA0D4F89415884721E2607992
:108B000010B1012866D122E0002104F17C00E26D61
:108B10008154616F01EBC10202EB011204F5A271F5
:108B200001EB8200C839F7F700FC606F401C6067FA
:108B3000606F0A2801DB00206067A06F401CA067FF
:108B4000A06F0A2801D30A20A06744E0F8E100BF23
:108B500000BF206F00EBC00202EB001204F5A27010
:108B600000EB8201642204F22C50F7F770FB266FB1
:108B700019E0701C0A21B0FBF1F201FB120808EBAE
:108B8000C80202EB081304F5A27202EB830106EBA4
:108B9000C60202EB061304F5A27202EB8300642204
:108BA000F7F755FB4646606F09300A2190FBF1F25A
:108BB00001FB1200B042DCD106EBC60101EB06124C
:108BC00004F5A27101EB8200642204F22C51F7F744
:108BD0003EFB00E000BF00BFC6A0D4F89415884754
:108BE000204600F0A9FC04F17C0000F007FC002006
:108BF00000F0A2FC00202066E065606F0A3020676C
:108C0000BDA0D4F8941588479BE1607910B1012884
:108C100053D100E000BFA06F00B94FE0A06F0A2859
:108C200003D1D4E91C0188420ED1A06F0A2841D09B
:108C3000606F0A30A16F401A0A21B0FBF1F201FB0C
:108C40001200216F884235D0206F09300A21B0FB15
:108C5000F1F201FB12002067206F00EBC00205E07B
:108C600008E1CCE08EE07EE072E029E002EB001249
:108C700004F5A27000EB8201C838F7F756FB04F147
:108C80007C00F7F730FBE065E06D20669BA0D4F830
:108C900094158847226F02EBC20303EB021304F51D
:108CA000A27202EB8300D4F89415884794A0D4F8FC
:108CB000941588470120607100E000BF00BF40E1CB
:108CC000607910B1012840D100E000BFA06F00B969
:108CD0003CE0606F09300A2190FBF1F201FB1200C9
:108CE000216F88422ED0206F401C0A21B0FBF1F288
:108CF00001FB12002067206F00EBC00202EB0012A4
:108D000004F5A27000EB8201C838F7F70EFB04F1FE
:108D10007C00F7F7E8FAE065E06D206677A0D4F80C
:108D200094158847226F02EBC20303EB021304F58C
:108D3000A27202EB8300D4F89415884770A0D4F88F
:108D4000941588470120607100E000BF00BFF8E083
:108D5000206E002806DD206E401E20660820D4F814
:108D600098158847EDE0D4E91710884209D204F13C
:108D70007C02236ED05CD4F898158847206E401C86
:108D80002066DEE0607910B1012835D100E000BF37
:108D9000E06D70B3206E00282BDD0820D4F8981504
:108DA0008847266E4FF0010808E004F17C02905DD0
:108DB000D4F898158847761C08F10108E06DB04298
:108DC000F3D82020D4F89815884703E00820D4F879
:108DD00098158847B8F10000A8F10108F6D1206E77
:108DE000401E20662046FFF755FDE06D401EE06501
:108DF00000BF0020607100E000BF00BFA1E060790B
:108E000010B1012833D100E000BFE06D60B3206EE7
:108E1000002829DDD4E91701884225D0206E461CA0
:108E20004FF0010808E004F17C02905DD4F8981539
:108E30008847761C08F10108E06DB042F3D8202085
:108E4000D4F89815884703E00820D4F89815884787
:108E5000B8F10000A8F10108F6D12046FFF71AFD8D
:108E6000E06D401EE06500BF0020607100E000BFC3
:108E700000BF66E0607910B101285ED100E000BF5C
:108E8000E06D98B3E06E50B90120E06604F17C011A
:108E900004F1E000E26DF7F7DAF9E06D60663CE0BE
:108EA000A06E00F0F1FA064604F1E001626EF7F7F9
:108EB00045FAE0B913A0D4F894158847A06E00F0E5
:108EC000E3FA0646D4F894158847A06E00F0DCFA61
:108ED0000646314604F17C00F7F727FA04F17C00DE
:108EE000F7F701FAE065E06D20660FE022E011E09F
:108EF0000D0A3E000D0A00003E0000000D3E00007D
:108F00001B5B4A000D1B5B4A3E000000A06E401C2C
:108F1000A06607E0A06E401CA06600F0AFFAA16E4C
:108F20008842BDD800BF00F0A9FAA16E884201D8DE
:108F30000020A0660020607100E000BF00BF00E0DC
:108F400000BF00BFBDE8F081002070472DE9F0416F
:108F500004460E461746092E7DD2DFE806F07C0552
:108F6000457C7C9BA6BDF800E06D63283BD2A079D0
:108F7000012804D12A20D4F89815884703E0384600
:108F8000D4F8981588472046FFF790FC04F17C0040
:108F9000216E4754206E401C2066E06D401CE06549
:108FA000256E4FF0000810E0A079012804D12A2096
:108FB000D4F89815884705E004F17C02505DD4F898
:108FC000981588476D1C08F10108E06DA842EBD8A0
:108FD00003E00820D4F898158847B8F10000A8F1FC
:108FE0000108F6D1ECE0EBE0E06D30B9A07920B9F2
:108FF00075A0D4F894158847E2E0A07910B1012853
:1090000045D115E0002104F17C00E26D815472A08D
:10901000D4F8941588470120A07100202066E065EF
:1090200004F17C02102104F10C0000F056FD2FE049
:10903000002104F17C00E26D81540020E06504F120
:109040007C02402104F11C0000F047FD04F11C01EA
:1090500004F10C0000E0B2E000F070F950B962A039
:10906000D4F8941588470220A07100202066E0659E
:1090700060710BE060A0D4F89415884752A0D4F832
:10908000941588470020A0712066E06500E000BFCD
:1090900000BF95E0206E002806DD206E401E206691
:1090A0000820D4F8981588478AE0D4E91710884238
:1090B00011D2A079012804D12A20D4F89815884724
:1090C00006E004F17C02236ED05CD4F89815884742
:1090D000206E401C206673E0E06DB0B3206E002867
:1090E00033DD0820D4F898158847256E4FF0010825
:1090F00010E0A079012804D12A20D4F898158847D7
:1091000005E004F17C02505DD4F8981588476D1C89
:1091100008F10108E06DA842EBD82020D4F898159A
:10912000884703E00820D4F898158847B8F1000074
:10913000A8F10108F6D1206E401E20662046FFF7F8
:10914000A9FBE06D401EE06500BF39E0FFE7E06D80
:10915000A0B3206E002831DDD4E9170188422DD05C
:10916000206E451C4FF0010810E0A079012804D1C1
:109170002A20D4F89815884705E004F17C02505D58
:10918000D4F8981588476D1C08F10108E06DA842D5
:10919000EBD82020D4F89815884703E00820D4F8AD
:1091A00098158847B8F10000A8F10108F6D12046CB
:1091B000FFF770FBE06D401EE06500BF00E000BF00
:1091C00000BFBDE8F08100000D0A757365726E6125
:1091D0006D653A20000000000D0A70617373776FAF
:1091E00072643A20000000000D0A57656C636F6DD1
:1091F00065210D0A3E0000000D0A55736572207648
:109200006572696679206661696C65642E0000008C
:1092100038B5002000900024424804687EE076E0E3
:1092200000F0D6F905469DF800102046FFF7B1FB87
:1092300000B16CE0FFF788FE01280AD1A068281A67
:109240003949884207D9A5600020A071E0652066F1
:1092500001E00220A071A07910B101282BD100E01B
:1092600000BF9DF800000D2806D19DF800200221C6
:109270002046FFF76BFE1DE09DF800000A2819D07C
:109280009DF80000082805D1002207212046FFF79D
:109290005DFE0FE09DF80000092805D1002209219C
:1092A0002046FFF753FE05E09DF8002001212046EF
:1092B000FFF74CFE29E09DF800000D2806D19DF82F
:1092C000002002212046FFF7C5FB1DE09DF80000AD
:1092D0000A2819D09DF80000082805D1002207218E
:1092E0002046FFF7B7FB0FE09DF80000092805D1E5
:1092F000002209212046FFF7ADFB05E09DF8002084
:1093000001212046FFF7A6FB00BF00BF00BF684653
:10931000D4F89C158847002882D02468002C7FF45C
:109320007EAF38BDF006002040771B000249096877
:109330000160014908607047F006002002460020E5
:109340007047000000BFEFF3058000B17047074889
:10935000006820B9012080F3108800BF00BF0348D7
:109360000068401C0149086000BFEFE7D0060020FC
:1093700070B504460D4600F099F850B100F096F82B
:10938000D0F8900528B100F091F8D0F8901502A01F
:109390008847002070BD00001B5B481B5B4A000033
:1093A00030B502460C460021002302B114B94FF03B
:1093B000FF3030BD0021002315E00E4850F8310089
:1093C00080B952F833000B4D45F8310002EBC30071
:1093D000406805EBC105686007480068401C064D01
:1093E00028605B1C491C502901D2A342E5D3002010
:1093F000DFE70000FC060020F8060020F0B595B07D
:109400000446002600E0641C20782028FBD020467B
:10941000F6F769FF10B9002015B0F0BD2046F6F749
:1094200062FF2044461E02E000203070761E307835
:109430002028F9D0142301AA2021204600F064FB43
:109440000746002511E00C4951F835002146F6F792
:1094500051FF48B9084800EBC50001A942683846E9
:10946000904700B905E004E06D1C00F007F8A84241
:10947000E9D800BF0020CFE7FC06002001480068C3
:1094800070470000F8060020014605480068814248
:1094900001D304A07047044850F83100FAE70000F7
:1094A000F806002000000000FC06002001480068CB
:1094B00070470000F40600202DE9F04106460F46F3
:1094C00000252AE0002412E0FFF7F0FF70B1FFF75B
:1094D000EDFFD0F8900548B1FFF7E8FFD0F89025F0
:1094E0002819114B53F8301010A09047641C052C1C
:1094F00004DAFFF7C3FF29198842E5D8FFF7D6FF42
:1095000050B1FFF7D3FFD0F8900528B1FFF7CEFF99
:10951000D0F8901507A088476D1DFFF7AFFFA84250
:10952000D0D80020BDE8F081FC060020252D313682
:10953000730000000D0A0000014908607047000038
:10954000F40600200146202902D34FF0FF30704777
:109550000120C1EBC102054B43F822000020C1EB02
:10956000C10203EB8202D06000BFF0E758E900209F
:1095700070B5054600240DB9601E70BD00240DE0D5
:10958000C4EBC4000C4951F8200030B90120C4EBF1
:10959000C401094A42F8210002E0641C202CEFD3E8
:1095A00000BF202C05D105A0FEF77AFF4FF0FF3059
:1095B000E3E72C600020E0E758E9002074696D655E
:1095C000722049442069732066756C6C0D0A000096
:1095D0000148006870470000D806002010B500243C
:1095E00000BF4AE0C4EBC400254951F8200002281E
:1095F00042D1C4EBC40001EB8000C0682149096876
:10960000081AC4EBC4011E4A02EB810109698842B1
:1096100032D9C4EBC400114601EB8000806928B345
:10962000C4EBC40001EB8000007928B90120C4EB31
:10963000C40142F821000CE00220C4EBC401104A2E
:1096400042F821000F480068C4EBC40102EB81011D
:10965000C860C4EBC4020A4B03EB82025069C4EB3E
:10966000C40203EB82029169884705E00120C4EB44
:10967000C401034A42F82100641C202CB2D310BD5F
:1096800058E90020D8060020F0B50446059D202C9E
:1096900002D34FF0FF30F0BD0220C4EBC406114FDF
:1096A00047F82600C4EBC4003E4606EB800001717B
:1096B0000D480068C4EBC40607EB8606F060C4EBF7
:1096C000C4003E4606EB80000261C4EBC40006EB1A
:1096D00080008361C4EBC40006EB8000456100207C
:1096E000D9E7000058E90020D806002007480068A4
:1096F000401C06490860064802684068521C40F158
:10970000000003490A60486070470000D806002046
:10971000E006002000BFEFF3058000B17047094864
:10972000006820B107480068401E064908600548E7
:10973000006820B9002080F3108800BF00BF00BF80
:10974000ECE70000D00600202DE9F04305460C466A
:109750009846079F0026002399460DB102B114B91F
:109760000020BDE8F083012F01D1032000E002209A
:109770006043401C404501D90020F2E7002618E074
:1097800015F806904FEA191000F019F819465B1CFD
:10979000505409F00F0000F012F819465B1C5054A9
:1097A000012F05D14FF0200C18465B1C02F800C0B9
:1097B000761CA642E4D30020D0541846D1E70146D7
:1097C000092903DC01F13000C0B270470A2905DB2A
:1097D0000F2903DC01F13700C0B2F6E73020F4E7CF
:1097E00070B504460D4629462046F6F749FD70BD82
:1097F0000146302904DB392902DCA1F130000EE0FA
:10980000412904DB462902DCA1F1370007E0612988
:1098100004DB662902DCA1F1570000E00020C0B2A1
:10982000704710B502460B46002406E01078FFF79B
:10983000DFFF00EB0414521C5B1E002BF6D1204608
:1098400010BD00B50246002305E01078FFF7D0FFF9
:1098500000EB0313521C10780028F6D1184600BD07
:1098600070B588B005460C4600200790069005901C
:1098700004902846F6F737FD064604A805A906AA6F
:1098800007ABCDE9002102900AA23146284600F03C
:1098900031F8042803D04FF0FF3008B070BD0798AE
:1098A0002070069860700598A0700498E070002001
:1098B000F3E7000025642E25642E25642E25640020
:1098C00002460B46002100BF10E0505C202803DB5D
:1098D000505C7E2800DC08E0505C0D2802D0505C13
:1098E0000A2800D101E000207047491C9942ECD3BE
:1098F0000120F9E70FB42DE9F84704460020009055
:109900000022202600270CB10B9820B90020BDE8CA
:10991000F8075DF814FB0CA80090D4E041B90B984F
:109920000078252803D10B984078652800D0CFE037
:109930000B980078252874D10B98401C0B900B983D
:1099400010F8016B0B90652E6CD004DC2A2E07D02A
:10995000642E68D113E0702E7AD0782EF9D144E0CD
:1099600008E020780B9B1B78984202D0641C491EAB
:1099700000E001E00029F4D100BF521C92E04FF05A
:10998000000CE046002300252020DDF8009059F867
:10999000045BCDF800901AE02078B8F1000F06D1F2
:1099A0002D2804D14FF0010C4FF001080DE03028B4
:1099B0000ADB392808DC4FF00108A0F1300903EB7D
:1099C000830A09EB4A0300E003E0641C491E0029F6
:1099D000E2D100BFBCF1010F03D16FEA030909F125
:1099E000010305B12B60521C5CE000230025DDF86B
:1099F00000C05CF8045BCDF800C022E0207830287D
:109A000006DB392804DCA0F1300C0CEB031316E064
:109A1000612809DB662807DCA0F1570C0CEB031367
:109A20000DE043E033E03AE0412807DB462805DC5F
:109A3000A0F1370C0CEB031301E009E003E0641C18
:109A4000491E0029DAD100BF05B12B60521C29E064
:109A5000DDF800C05CF8040BCDF800C00025002341
:109A600025460CE094F800C0DDF82C8098F80080C2
:109A7000C44501D05B1C00E003E0641C491E0029C2
:109A8000F0D100BF08B105604360521C0AE0009BA2
:109A900001CB009300B10460521C012702E00127B2
:109AA000002200BF00BF012F0DD111E020780B9BD9
:109AB0001B78984205D1641C0B98401C0B90491EE2
:109AC00001E0002204E00B98007800287FF426AF24
:109AD00000BF00200090104619E70FB4F8B5064605
:109AE0000C46002509A8009021463046009B089AA4
:109AF00006F0C8FE054600200090A54200D3651E72
:109B00002846F8BC5DF814FBF0B504460E461D4629
:109B1000214600230DB104B10AB90020F0BD18465A
:109B20005B1C42F820100AE00878B04206D1002001
:109B30000870481C1F465B1C42F82700491C087827
:109B400008B1AB42F0D31846E8E770B506460025E9
:109B5000002478213046F6F7BCFB044624B958218E
:109B60003046F6F7B6FB04465CB1641C05E020788D
:109B7000FFF73EFE00EB0515641C20780028F6D1A7
:109B800003E03046F6F7E9FB0546284670BD2DE9AF
:109B9000F04106460F4614463846F6F7A4FB054644
:109BA00015B93046BDE8F081A54201D90020F9E79A
:109BB00009E0641E2A4639463046F6F7A9FB08B983
:109BC0003046EFE7761CAC42F3D20020EAE770B5EE
:109BD00004460D4604B115B94FF0FF3070BD0121A8
:109BE00004F11000FEF7D4FB04F12000A968FEF791
:109BF000CFFB0020F2E770B504460D4604B115B95D
:109C00004FF0FF3070BD012104F11000FEF7D7FBCB
:109C100004F12000A968FEF7D2FB0020F2E710B59E
:109C200004460CB9002010BD04F11000FEF722FC20
:109C3000012801D10020F6E704F12000FEF71AFC0C
:109C4000012801D10020EEE704F11000FEF700FC2E
:109C500000EB4000216801EB8000E4E77CB504469E
:109C60000E46002500200190009004B97CBD04F14F
:109C70001000FEF709FC08B10020F7E76B4601AAC7
:109C8000314604F12000FEF7B2FB08B10020EDE7F9
:109C900004F11000FEF7DFFB00EB4000216801EB50
:109CA0008005A0680199084428606E600098A8604B
:109CB0002846DBE72DE9F04104460E4617461D46CF
:109CC0004FF0000805EB4500B7EB800F03D84FF0CD
:109CD000FF30BDE8F08105EB45004FEA80082660C3
:109CE000C4F8048060683044A060A7EB0801E1601C
:109CF000294604F11000FEF7B1FB04F12000E168F1
:109D0000FEF7ACFB0020E4E710B5044621460CA0AA
:109D1000FEF7C6FB1048007868B11048006803F0F1
:109D2000C5FD012804D00D48006803F0D5FC02E011
:109D30000020094908700A480068FFF703FC10BDBD
:109D40004572726F72206F63637572726564204032
:109D500025730D0A000000005C050020600500204E
:109D60006405002038B504460D46354800780228C1
:109D70002BD134480068C82821D12CB932A0FFF774
:109D8000C3FF4FF0FF3038BD002060552B46224600
:109D900036493748FBF7F6F828B136A0FFF7B4FF8D
:109DA0004FF0FF30EFE7042002F040FC3A48008813
:109DB00082B23A493A48006803F0D6FC3DE039A047
:109DC000FFF7A2FF4FF0FF30DDE71D4800780328C2
:109DD00019D11C480068C8280FD1052002F026FCC4
:109DE000002039490860394B4EF660220146009048
:109DF00037480068FFF748FC1FE036A0FFF784FFF4
:109E00004FF0FF30BFE70E480078052815D12CB978
:109E100039A0FFF779FF4FF0FF30B4E700202B4B5C
:109E20004EF660220146009029480068FFF72CFC9E
:109E30002A462146C820F7F767FD0020A3E7000067
:109E40005C050020800500202E2E5C464D4C5C49B0
:109E50006E7465726E65745C4E54524950436C6901
:109E6000656E742E633A33323000000054C4002013
:109E700074C400202E2E5C464D4C5C496E74657295
:109E80006E65745C4E54524950436C69656E742E15
:109E9000633A33323700000070050020D4C300203D
:109EA000600500202E2E5C464D4C5C496E74657238
:109EB0006E65745C4E54524950436C69656E742EE5
:109EC000633A333336000000780500208DE4020841
:109ED000640500202E2E5C464D4C5C496E74657204
:109EE0006E65745C4E54524950436C69656E742EB5
:109EF000633A3335300000002E2E5C464D4C5C49F1
:109F00006E7465726E65745C4E54524950436C6950
:109F1000656E742E633A33353800000005E003A106
:109F200009A006F073FC05F0A9FBF8E72E2E2F53CD
:109F300072632F73746D3332663478785F69742E70
:109F4000633A38350000000025732055525452659D
:109F500073746172740000002DE9F04106460C46EE
:109F6000002514E016F8017B3A111449022303FB83
:109F7000051013A106F072FC07F00F026900491CDE
:109F80000E4BC8180EA106F069FC681CC5B2A542AC
:109F9000E8DB0D20094A02F814000A216000401C89
:109FA0001154F7F723FD022805D16000821C0349F4
:109FB000002006F049F9BDE8F08100005E1C002099
:109FC0002578000010B500224FF400510D48FBF732
:109FD0000DFF00224FF480410A48FBF707FF0A20DB
:109FE00007F0F5F9012251030648FBF7FFFE0A20AE
:109FF00007F0EDF900224FF400510248FBF7F6FE9E
:10A0000010BD00000004024010B500224FF40051C2
:10A010000C48FBF7EBFE012291030A48FBF7E6FE32
:10A020000A2007F0D4F9012251030648FBF7DEFEAF
:10A030000A2007F0CCF900224FF400510148FBF749
:10A04000D5FE10BD0004024070B505460024002670
:10A050001CE000224FF400511148FBF7C7FE0A2014
:10A0600007F0B5F9012251030D48FBF7BFFE60066A
:10A07000040E4FF480410A48FBF7B0FE08B1601CA3
:10A08000C4B2052007F0A3F9701CC6B2082EE0DBAD
:10A0900015B9FFF7B9FF01E0FFF794FF204670BD47
:10A0A0000004024070B5044600224FF400511748E6
:10A0B000FBF79CFE002525E0E00928B10122910371
:10A0C0001248FBF793FE05E000224FF480410F4851
:10A0D000FBF78CFE6006040E0A2007F078F90122D7
:10A0E00051030A48FBF782FE0A2007F070F90022AC
:10A0F0004FF400510548FBF779FE0A2007F067F995
:10A10000681CC5B2082DD7DB70BD000000040240FA
:10A1100010B5012291030C48FBF768FE01225103A0
:10A120000948FBF763FE00224FF480410648FBF725
:10A130005DFE0A2007F04BF900224FF4005102485F
:10A14000FBF754FE10BD00000004024010B50022D1
:10A150004FF400510C48FBF749FE00224FF48041B8
:10A160000948FBF743FE0A2007F031F901225103A9
:10A170000548FBF73BFE012291030348FBF736FE3F
:10A180000A2007F024F910BD0004024010B5002495
:10A19000012291031248FBF729FE062007F017F968
:10A1A000012251030E48FBF721FE062007F00FF9AC
:10A1B00007E0601CC4B2FA2C03DDFFF7C7FF0120E3
:10A1C00010BD4FF480410648FBF708FE0028F0D18F
:10A1D00000224FF400510248FBF708FE0020EFE791
:10A1E0000004024010B51548808A00EE100AB8EE4F
:10A1F000400A1348D0ED000AB4EEE00AF1EE10FA7E
:10A2000003D201200F49087002E000200D490870B8
:10A210000A48408F00EE100AB8EE400A0848D0ED18
:10A22000000AB4EEE00AF1EE10FA05D20348C08F3E
:10A23000012801D107F022FE10BD00009824002063
:10A240001C0600200800002010B50F48B0F8600080
:10A25000012809D100200C49A1F860000BA110A031
:10A2600006F0D4FA05F00AFA0748008845F2AA5128
:10A27000884202D10448C08828B90DA108A006F080
:10A28000C5FA05F0FBF910BD982400202E2E5C4184
:10A29000504C5C7577625F6170702E633A393400A0
:10A2A0002573205552545265737461727400000016
:10A2B0002E2E5C41504C5C7577625F6170702E632E
:10A2C0003A39390010B5F8F713FB10B14FF0FF30F1
:10A2D00010BD04F04DF810B14FF0FF30F8E703F077
:10A2E000FDFF10B14FF0FF30F2E70020F0E710B5AE
:10A2F000F9F762FD10BD000010B500220F210248E1
:10A30000FEF7BCF9002010BD8CC3002010B5FFF78C
:10A31000EEFF012804D14FF40800074908600AE065
:10A320000648007820B14FF408400349086002E075
:10A3300000200149086010BD6C06002016020020B4
:10A3400010B53721202000F079F80321212000F0FA
:10A3500075F84021222000F071F80821232000F038
:10A360006DF8AA21302000F069F801200B49088718
:10A37000084690F83810322000F060F802213320AF
:10A3800000F05CF85F21202000F058F8044800F04D
:10A3900009F80A2007F01BF810BD000098240020DF
:10A3A0005506002010B5044621460F2000F023F882
:10A3B00008B9002010BD0120FCE770B50446002557
:10A3C000FFF7A6FE3220FFF76DFEFFF7DFFEE0B2DB
:10A3D000FFF768FEFFF7DAFEFFF79AFE3320FFF77C
:10A3E00061FEFFF7D3FE0020FFF72EFE0546FFF7C4
:10A3F000ADFE284670BD70B505460C462846FFF7F1
:10A40000DCFF2070012070BD70B504460D46FFF7DB
:10A410007FFE3220FFF746FEFFF7B8FEE0B2FFF7FF
:10A4200041FEFFF7B3FE2846FFF73CFEFFF7AEFE06
:10A43000FFF78CFE0A2006F0CAFF70BD70B5044617
:10A440000D4629462046FFF7DFFF012070BD0000C2
:10A4500001460020174A914203D2B1F1006F00D3A8
:10A4600026E0154A914204D2124A914201D30120BA
:10A470001EE0124A914204D20F4A914201D30220B7
:10A4800016E00F4A914204D20C4A914201D30320B4
:10A490000EE00C4A914204D2094A914201D30420B1
:10A4A00006E0094A914203D2064A914200D30520B0
:10A4B00070470000004000080080000800C000084D
:10A4C0000000010800000208000004081FB51F4832
:10A4D0001F4908604FF48030486000211C488160AB
:10A4E00001210161816100210162C162194981621A
:10A4F0000021C1600221C161012101634161FAF7BC
:10A5000081FE20B140F2051113A006F07DF9012073
:10A51000009001900720029069460D48FAF7A8FDC7
:10A5200020B140F20F110CA006F06EF9112000903E
:10A530000220019069460648FAF79AFD20B14FF4CF
:10A540008C7105A006F060F91FBD000000200140DD
:10A55000C0E400200100000F2E2E2F5372632F6DD8
:10A5600061696E2E6300000008B500BF00200090F6
:10A570002A48006840F480002849086008460068BE
:10A5800000F48000009000BF00BF00BF00200090DA
:10A590000846006840F4001008600846006800F4AF
:10A5A0000010009000BF00BF002211461020FBF7F2
:10A5B000C0FC1020FBF7B0FC002211461120FBF775
:10A5C000B8FC1120FBF7A8FC002211463820FBF74D
:10A5D000B0FC3820FBF7A0FC002211463920FBF725
:10A5E000A8FC3920FBF798FC002211463A20FBF723
:10A5F000A0FC3A20FBF790FC002211464520FBF717
:10A6000098FC4520FBF788FC002211464620FBF70A
:10A6100090FC4620FBF780FC08BD0000303802406B
:10A6200000B587B000BF002001908748006840F067
:10A630000400854908600846006800F004000190A5
:10A6400000BF00BF00BF002001900846006840F036
:10A65000800008600846006800F08000019000BF9C
:10A6600000BF00BF002001900846006840F00100D4
:10A6700008600846006800F00100019000BF00BFBC
:10A6800000BF002001900846006840F0020008600A
:10A690000846006800F00200019000BF00BF00BF44
:10A6A000002001900846006840F008000860084655
:10A6B000006800F00800019000BF00BF012248F2CE
:10A6C00010116248FBF792FB012241F21001604831
:10A6D000FBF78CFB0022A5215E48FBF787FB0122DC
:10A6E00046F248415B48FBF781FB00224FF4807142
:10A6F0005748FBF77BFB00224FF480515348FBF790
:10A7000075FB002204215448FBF770FB4FF4005006
:10A71000029000200390049002A94D48FBF774FAC0
:10A72000012002904D4803900020049002A9474860
:10A73000FBF76AFA49F21010029001200390002002
:10A740000490059002A94148FBF75EFA41F210100F
:10A7500002900120039000200490059002A93C483B
:10A76000FBF752FA40F2ED400290012003900020E6
:10A770000490059002A93748FBF746FA02200290A0
:10A78000364803900120049002A93248FBF73CFAB6
:10A790004FF480500290314803900020049002A9A9
:10A7A0002C48FBF731FA4FF4C0400290112003907F
:10A7B000002004900320059002A92648FBF724FA04
:10A7C0004FF400700290254803900020049002A9E5
:10A7D0001F48FBF719FA0420029001200390002083
:10A7E00004900220059002A91B48FBF70DFA4FF4D4
:10A7F0000470029000200390049002A91548FBF712
:10A8000003FA002201210620FBF793FB0620FBF749
:10A8100083FB002201210720FBF78BFB0720FBF7BE
:10A820007BFB002201211720FBF783FB1720FBF79E
:10A8300073FB002211462820FBF77BFB2820FBF747
:10A840006BFB07B000BD0000303802400000024042
:10A850000008024000040240000C024000001110F9
:10A8600010B51048104908604FF48270486000210C
:10A870000D488160C160016141614FF400718161E7
:10A880000821C16100210162416281620A21C16225
:10A89000FBF748FF20B14FF4987104A005F0B4FF16
:10A8A00010BD00000030014068E500202E2E2F531F
:10A8B00072632F6D61696E2E6300000000B591B068
:10A8C00028482949086009204860002126488160FD
:10A8D0004FF43761C160002101614161FCF799FDCE
:10A8E00020B140F2451121A005F08EFF00200F900D
:10A8F00010900FA91C48FCF7B6FA20B14FF4A671CE
:10A900001AA005F081FF602008904FF4B76009900D
:10A9100000200A900C900D900E900C2208A912486D
:10A92000FCF7F3FC20B140F2571110A005F06CFFCA
:10A930000020019002900390049005904FF4005085
:10A9400006900020079001A90748FCF74DFA20B1B6
:10A9500040F2631105A005F057FF0348FCF7BAFC6D
:10A9600011B000BD00000140C0E500202E2E2F5385
:10A9700072632F6D61696E2E6300000000B587B0B1
:10A980001848194908604F20486000211648816026
:10A990004FF47A71C16000210161FCF7B8FA20B16F
:10A9A0004FF4BC7111A005F02FFF4FF480500390BD
:10A9B00003A90D48FCF729FB20B14FF4BF710BA090
:10A9C00005F022FF00200190029001A90648FCF743
:10A9D0004AFA20B140F2851104A005F015FF07B036
:10A9E00000BD000000040040FCE500202E2E2F5387
:10A9F00072632F6D61696E2E6300000010B50C4804
:10AA00000C4908604FF4E13048600021094881603A
:10AA1000C16001610C21416100218161C161FCF7CC
:10AA2000DDFE20B14FF4CC7103A005F0EDFE10BDAA
:10AA30000010014038E600202E2E2F5372632F6D38
:10AA400061696E2E6300000010B50C480C49086067
:10AA50004FF416404860002109488160C1600161DF
:10AA60000C21416100218161C161FCF7B7FE20B179
:10AA700040F2AB1103A005F0C7FE10BD004400403A
:10AA800078E600202E2E2F5372632F6D61696E2E93
:10AA90006300000010B50C480C4908604FF4E13029
:10AAA0004860002109488160C16001610C21416159
:10AAB00000218161C161FCF791FE20B14FF4DF718B
:10AAC00003A005F0A1FE10BD00140140B8E600206F
:10AAD0002E2E2F5372632F6D61696E2E630000005E
:10AAE00000BFFEE700487047108000200048704714
:10AAF000F07F002000487047008000200048704729
:10AB000025800020024604480260044801600120BC
:10AB1000034B1870002070474804002044040020B4
:10AB20004C0400200146034A505C0022014B5A5459
:10AB3000704700005E0400200146034A505C00227A
:10AB4000014B5A54704700006104002070B5044660
:10AB50000D460648006830B105482946026820467F
:10AB6000024B1B689847002070BD00005004002075
:10AB70005404002001460120024A50540020024A99
:10AB8000505470475E0400206104002001460120FB
:10AB9000024A50540020024A505470476104002079
:10ABA0005E04002010B5044614B94FF0FF3010BD0C
:10ABB000012004490870224680210348FEF78DFFDA
:10ABC0000020F4E764040020258000200249087872
:10ABD0000021014A117070476404002001460020E2
:10ABE0007047000070B505460C46152C07D222466A
:10ABF00029460448F5F72BFB0020024908550020A0
:10AC000070BD00001080002070B505460C46022C77
:10AC100002D24FF0FF3070BDA41E102C07D2224686
:10AC200029460448F5F713FB002002490855002087
:10AC3000F1E70000F07F002070B505460C46022CBD
:10AC400002D24FF0FF3070BDA41E102C07D2224656
:10AC500029460448F5F7FBFA002002490855002070
:10AC6000F1E700000080002002460348026003482C
:10AC700001600020704700005004002054040020B0
:10AC8000024908780021014A117070474C040020E5
:10AC900010B504460648006828B1064801682046F9
:10ACA000034A1268904704480460002010BD000069
:10ACB00048040020440400204004002070470000A5
:10ACC00008B50F48FEF754FC10B14FF0FF3008BD37
:10ACD0000C48FEF74DFC10B14FF0FF30F7E70020B5
:10ACE000094B42F210720121009006480068FEF7FD
:10ACF000CBFC002005490860F6F760FE0020E6E77F
:10AD0000340200203C020020D5180208380200203E
:10AD100070B504460E462046F5F7E5FA0546294685
:10AD2000204600F0D7F870BDF8B504460E4615462B
:10AD30001F46642C04D0652C03D0C82C29D117E001
:10AD400000BF16480068401C1449086008460068A7
:10AD500003280AD90020124B47F2305201460090D6
:10AD600010480068FEF790FC01E0F6F727FE11E0BE
:10AD700000200A4908602A463146022005F064FA9C
:10AD800010B109A0FDF78CFB29460DA0FDF788FB4B
:10AD900000E000BF00BF0020F8BD00003802002026
:10ADA00059E402083402002052544B20446174617B
:10ADB0002053656E64204572726F720D0A000000A8
:10ADC0002575422052544B20446174612053656EB6
:10ADD000740D0A002DE9F84F04460F4615461E462D
:10ADE000DDE90B8ADDF828904FF0000B1E48007853
:10ADF00018B14FF0FF30BDE8F88F24B1B8F1000F63
:10AE000001D005B116B94FF0FF30F4E722464021DA
:10AE10001648FEF762FE4A4620211548FEF75DFE01
:10AE20002B4614A2402115480096FEF756FE834695
:10AE30008023134A59461148FDF736FA1148076036
:10AE40001148C0F800801148C0F800A0012001F0AE
:10AE5000EDFB0C48008882B204490D48006802F0FE
:10AE600083FC0020C7E700005C050020D4C300205D
:10AE700054C4002025733A257300000014C4002038
:10AE8000B5C4002070050020680500206C05002076
:10AE90006005002010B500200A49087000230A4A06
:10AEA00001210A4802F086FC10B14FF0FF3010BDBE
:10AEB0000748FEF75DFB10B14FF0FF30F7E70020C9
:10AEC000F5E700005C050020F1D5020860050020D0
:10AED0006405002070B504460D4606480078052834
:10AEE00005D12A4621460448006802F089FE002068
:10AEF00070BD00005C05002060050020024800686D
:10AF0000C0F30220704700000CED00E010B50028EF
:10AF100007DA0A07140E054A00F00F031B1FD4546A
:10AF200003E00A07130E024A135410BD18ED00E0A7
:10AF300000E400E038B500250020009000BF5E4826
:10AF40000068C0F580525D485B4B1B68C1186B46BA
:10AF50005B48006802F098FD05460DB9009800B9FD
:10AF6000A7E055480068009908445349086008461E
:10AF70000068B0F5805F03D352A0FEF7C5FE98E0ED
:10AF800059480078052808D14B4801684B48FEF71E
:10AF9000E9FE0020484908608AE053480078032809
:10AFA0001BD152A14548009AFEF7F1FD50490860B7
:10AFB0000846006800287AD04E4B4FA23F480099BF
:10AFC000FEF798FC032803D04EA0FEF79DFE70E02C
:10AFD00000210846FEF7C6FE69E0434800780228D3
:10AFE00065D151480078002855D150A13348009AC6
:10AFF000FEF7CDFD3E49086008460068002856D09F
:10B00000002408460068001D08603A4B3AA22B480D
:10B010000099FEF76FFC032803D046A0FEF774FEEC
:10B0200047E04DA12548009AFEF7B1FD04466CB3F8
:10B03000103400E0641C20782028FBD01F48201A20
:10B04000009A111A494B4AA22046FEF753FC0128E8
:10B0500003D049A0FEF758FE2BE0254800681749A9
:10B06000401A4249096808444C49086001202E49A9
:10B070000870114800684949096888420AD33B486A
:10B0800001681B480068FEF76DFE12E044A0FEF761
:10B090003BFE0EE00BE00848006840490968884222
:10B0A00005D33248016812480068FEF75BFE00BF16
:10B0B00045E700BF002038BD7805002035C90020D5
:10B0C000600500202E2E5C464D4C5C496E74657206
:10B0D0006E65745C4E54524950436C69656E742EB3
:10B0E000633A3339350000005C0500200D0A00008A
:10B0F0008805002080050020252A20256420252A97
:10B100000D0A00002E2E5C464D4C5C496E74657233
:10B110006E65745C4E54524950436C69656E742E72
:10B12000633A3431330000005D0500200D0A0D0A3A
:10B13000000000002E2E5C464D4C5C496E7465721A
:10B140006E65745C4E54524950436C69656E742E42
:10B15000633A343334000000436F6E74656E742DAF
:10B160004C656E6774683A2000000000840500207A
:10B1700025640D0A000000002E2E5C464D4C5C49F3
:10B180006E7465726E65745C4E54524950436C69BE
:10B19000656E742E633A3435300000007C05002063
:10B1A0002E2E5C464D4C5C496E7465726E65745C07
:10B1B0004E54524950436C69656E742E633A34366E
:10B1C0003500000010B50446F6F756FBFFF70AF805
:10B1D00003480088401C0249088006F0EBFE10BDC1
:10B1E0000A00002010B501200549087000F09EF902
:10B1F000012211030348FAF7F9FD00F005F810BD2C
:10B20000160200200000024010B504F093FA01215C
:10B21000044806F055FC002006F098FC002006F0DB
:10B220001DFC10BD00D023247047000010B54FF462
:10B2300080511048FAF7D2FDD0B14FF47A7006F081
:10B24000BCF84FF480510B48FAF7C8FD80B10EE00E
:10B250004FF480510748FAF7C1FD40B9642006F069
:10B26000ACF800224FF480710348FAF7BFFDEFE716
:10B2700010BD0000000402400000024010B52DED9A
:10B28000028B4FF400719548FAF7A8FD002874D09E
:10B29000002093490880934908709348007850B97A
:10B2A0009248007838B9F6F747FB0320F6F7C2FC5E
:10B2B00001208D49087073E0FEF78AF98C4909680E
:10B2C000401A41F2707188422AD9FEF781F9884903
:10B2D000086083480088801D814908804FF48061A0
:10B2E0007E48FAF77BFD40B100F026F9BCEEC00ABB
:10B2F00010EE100A7F49087012E00122910277488F
:10B30000FAF774FD00F018F9BCEEC00A10EE100A4E
:10B310007849087000224FF480617048FAF766FDA2
:10B3200075480068F5F7DAF941EC180B9FED730BDF
:10B3300053EC102BF5F7FEF908D86A48007828B9C5
:10B340000120684908700020654908806A48006843
:10B35000F5F7C4F941EC180B9FED680B53EC102B7B
:10B36000F5F7E8F90AD85E480088B0F5E16F05DB2B
:10B370004FF408006349086004E01BE04FF4084004
:10B3800060490860642006F018F8F6F76DFBFEF7D8
:10B39000B3FF5C48002211460368104601F030F903
:10B3A0004FF400714D48FAF719FD18B1F6F71EFB7E
:10B3B000032881D00020544908704B480078C8B158
:10B3C0000020F6F737FC002047490870FFF70AFF16
:10B3D0004FF400714148FAF701FD58B9642005F0B7
:10B3E000ECFF00224FF480714848FAF7FFFC64201C
:10B3F00005F0E3FF4FF400713848FAF7EFFC10B99D
:10B4000000203A490870FEF7E3F84FF47A71B0FB78
:10B41000F1F201FB12000A281CD23D48007858BB0B
:10B42000344800780F2803DD88203649086003E09F
:10B430004FF408403349086001203549087031480D
:10B44000036834480268344801683448006801F0F1
:10B45000D7F811E02E48007870B100202C49087010
:10B4600028490860084603682A4802682A48016893
:10B470002A48006801F0C4F8FEF7AAF81C490968D8
:10B48000401A41F28831884225D9FEF7A1F81849BF
:10B4900008604FF480611148FAF7A0FC40B100F059
:10B4A0004BF8BCEEC00A10EE100A1249087012E008
:10B4B000012291020948FAF799FC00F03DF8BCEE30
:10B4C000C00A10EE100A0B49087000224FF4806188
:10B4D0000248FAF78BFCBDEC028B10BD0004024061
:10B4E0000C0000200E0000200F0000207E03002032
:10B4F000140000201E020020340600209A99999919
:10B5000099991040700600201000002000000240B1
:10B510002F0000206C060020680600206406002032
:10B5200010B50020FFF726FB002010BD10B500204D
:10B53000FFF72CFB002010BD10B52DED068B9FED05
:10B540003D0AB0EE408A9FED3B0AF0EE408A00F0E3
:10B5500081F8B0EE408A9FED380AB4EEC08AF1EE71
:10B5600010FA04D29FED330AF0EE408A19E0B1EEF2
:10B57000000AB4EEC08AF1EE10FA04DD9FED2F0A46
:10B58000F0EE408A0DE09FED2C0A38EE400A9FED68
:10B590002C1AC0EE010A9FED290A20EE800AF0EE77
:10B5A000408A284890ED000AB5EEC00AF1EE10FA84
:10B5B00006D2C0ED008AFEF70BF82349086033E09D
:10B5C000204890ED000A30EE680A10EE101A084686
:10B5D000F5F784F841EC1A0BB0EE4A0AF0EE6A0A6D
:10B5E00005F06AF9B0EE409AF0EE609A9FED170B05
:10B5F00053EC102B51EC190BF5F784F804D2FDF73E
:10B60000E7FF114908600FE0FDF7E2FF0E49096806
:10B61000401A4EF66021884206D90A48C0ED008AD9
:10B62000FDF7D6FF08490860064890ED000ABDEC1A
:10B63000068B10BD00000000333353400000C842A9
:10B640003333333F380600203C0600200000000062
:10B650000000E03F2DE9F0412DED0C8B0020F5F7C7
:10B66000D7FC85B200242846F5F70CF841EC1B0BFB
:10B670009FED500B53EC102BF4F795FF41EC1A0B98
:10B680009FED4E0B53EC102BF4F71BFF41EC190B05
:10B69000F5F768F808EE100AB0EE000A28EE000A86
:10B6A000B0EE408A2846F4F7EDFF41EC1B0B9FED0E
:10B6B000410B53EC102BF4F776FF41EC1A0B9FED86
:10B6C0003F0B53EC102BF4F7FCFE41EC190BF5F794
:10B6D00049F83C490860084690ED000AF0EE000A7F
:10B6E00020EE200A80ED000A0020F5F791FC87B2D9
:10B6F0000120F5F78DFC1FFA80F83348068838469C
:10B70000F4F7C0FF41EC1B0B3046F4F7BBFF41ECF4
:10B710001D0B9FED2A0B53EC102BF4F7D2FE41ECDE
:10B720001C0B53EC1B2BF4F7CCFE41EC1A0B9FEDDA
:10B73000270B53EC102BF4F7C4FE41EC190BF5F773
:10B7400011F800EE100AC8EB083000EE900AF8EE8F
:10B75000E00A80EE201AF0EE418A18EE900AF4F723
:10B76000BDFF41EC190B9FED150B53EC102BF4F7BB
:10B77000C9FF02D20120174908609FED170A38EE71
:10B78000C00A9FED161AC0EE010A9FED150A20EEC1
:10B79000800ABDEEC00A10EE104A642C00DD64245D
:10B7A000002C00DA0024B0EE480ABDEC0C8BBDE89A
:10B7B000F08100000000000000FEAF406666666693
:10B7C00066660A40340600202A7AFF1F0000000047
:10B7D000000000403006002033335340CDCC4C3FB6
:10B7E0000000C84210B500210248FFF73DFA0020D2
:10B7F00010BD0000F9B70208014B1A607047000045
:10B800007C0100201CB506F0CFFC40F20310BC49BF
:10B8100048800120BB490870B94890F84400BA49F3
:10B820000870012008700846007848B94FF47A7013
:10B83000B349C8800120C8870A204887002088872C
:10B84000AF48C088322802DA6420AD49C880AC48CD
:10B85000C088B0F57A7F03DD4FF47A70A849C880BC
:10B86000A748008F0A2802DD0220A5490887A448BE
:10B87000C08E432802DD4320A149C886A048C08E5F
:10B88000002802DA00209E49C8869D48808A4FF62B
:10B89000FF71884202D10A20994988829848808C99
:10B8A00042F21071884202DD002095498884944854
:10B8B00090F8360095490870914890F83E009449F8
:10B8C00008708F4890F83C00924908708C48807A44
:10B8D000914908708A4880889049086005209049FD
:10B8E00008808748C088098890FBF1F08D4908805E
:10B8F00083488088098890FBF1F201FB1200884997
:10B900000988484388490880084600888749088094
:10B910007B48C0884FF47A7191FBF0F0844908802D
:10B9200008460088C82191FBF0F082490880002079
:10B9300081490880552081490870AA2048707048C4
:10B94000408C000B4FF47A7110FB01F16C48408C75
:10B95000C0F3032000EBC00202EB001001EB8000FB
:10B96000674991F82210C1F3031101EB810100EB4B
:10B970004100634991F8221001F00F010844704919
:10B9800008805F48808C000B4FF47A7110FB01F047
:10B990005B49898CC1F3032101EBC10202EB011168
:10B9A00000EB8100564991F82410C1F3031101EB1B
:10B9B000810100EB4100524991F8241001F00F0180
:10B9C0000844604908804E48C08C000B4FF47A71DF
:10B9D00010FB01F14A48C08CC0F3032000EBC00209
:10B9E00002EB001001EB8000454991F82610C1F3ED
:10B9F000031101EB810100EB4100414991F8261050
:10BA000001F00F010844504908803D48008D000BAB
:10BA10004FF47A7110FB01F03949098DC1F303210C
:10BA200001EBC10202EB011100EB8100344991F8F6
:10BA30002810C1F3031101EB810100EB41003049F3
:10BA400091F8281001F00F010844404908802C4863
:10BA5000008B3F490880314801683EA004F0D6FEC3
:10BA600027488278408801123EA004F0CFFE384873
:10BA7000008836490988CDE90010334803883148E9
:10BA800002882F48018840A004F0C0FE1C48B0F88E
:10BA9000560001280DD11A48008B1949098DCDE9AE
:10BAA00000101748C38C828C418C3FA004F0AEFE7E
:10BAB00025E01348B0F85600022819D1454946A0A0
:10BAC00004F0A4FE0E48B0F8A01247A004F09EFEB9
:10BAD0004049223148A004F099FE3E4942314BA032
:10BAE00004F094FE3B4962314DA004F08FFE06E065
:10BAF0000348B0F8560010B94FA004F087FE1CBDF3
:10BB0000982400202D0000200C0200207506002043
:10BB1000F4010020F5010020D7010020CC01002015
:10BB2000E0010020E2010020DC010020EC01002007
:10BB3000EA010020000200200E020020641600200E
:10BB4000AC010020AE010020B0010020B2010020B5
:10BB5000B4010020C9E8B1B849443A202578202E24
:10BB60000D0A0000B9CCBCFEB0E6B1BE3A20555279
:10BB7000542D4D4BB0B2B0EEB3B5D4D82056256499
:10BB80002E25642E200D0A00B7FECEF1C6F7B5D8DB
:10BB9000D6B73A2025642E25642E25642E25643AD6
:10BBA00025642E0D0A0000005443505F5254434D4B
:10BBB000C4A3CABD2CB7FECEF1C6F7B5D8D6B73AE6
:10BBC0002025642E25642E25642E25643A25642EB6
:10BBD0000D0A0000182700204E74726970486F73B8
:10BBE000743A25732E0D0A004E74726970506F728C
:10BBF000743A25642E0D0A004E747269705573658F
:10BC0000726E616D653A25732E0D0A004E7472696D
:10BC10007050617373776F72643A25732E0D0A004A
:10BC20004E74726970536F757263656E616D653ABB
:10BC300025732E0D0A000000B5A5B5E3B6A8CEBB4E
:10BC4000C4A3CABDC4A3CABD2E200D0A00000000B3
:10BC500030B503460224144D2C70002007E0134C2D
:10BC600034F810409C4200D105E0441CE0B2104C76
:10BC70002478A042F3DB00BF0D4C2478A04209D108
:10BC80000B4C2478B4F5957F04DC094C2478641CB3
:10BC9000074D2C70054C24F81030064C24F8101079
:10BCA000054C225430BD00001A020020343E002012
:10BCB0001B0200208C400020E442002000B54FF41D
:10BCC0000000034908604FF4FA7006F0CBFB00BD9A
:10BCD0001804024030B50446002517230AE024FA70
:10BCE00003F000F0010515B100F01AF801E000F0D2
:10BCF00005F85B1E002BF2DA30BD000000B5802095
:10BD000006490860022006F0ADFB4FF4000003492D
:10BD100008600A2006F0A6FB00BD000018040240DF
:10BD200000B58020064908600B2006F09BFB4FF40D
:10BD3000000003490860022006F094FB00BD0000EB
:10BD40001804024038B504461CB9002000F010F871
:10BD500008E00020044B224601460090034800689A
:10BD6000FDF792FC38BD000071BD02082C060020D2
:10BD700072B60649064A116000BF00BF00BFBFF39C
:10BD80004F8F00BF00BF00BF704700000400FA05DE
:10BD90000CED00E000B585B014216846F4F770FAA8
:10BDA000642005F00AFB00224FF400411148FAF725
:10BDB0001DF84FF4004000900120019000200290F7
:10BDC000039069460B48F9F71FFF642005F0F5FA68
:10BDD0004FF4004000900320019000200290039057
:10BDE00069460448F9F710FF022005F0E6FA05B0AD
:10BDF00000BD00000004024010B50446204600F0DB
:10BE0000CCFA00B118E0204600F034F80022C72137
:10BE1000204600F039FA00B111E0204600F016F893
:10BE2000204600F0A9FA00B106E0204600F03CFAF6
:10BE300000B101E0002010BD4FF0FF30FBE72046CD
:10BE400000F004F84FF0FF30F5E7000010B50446AD
:10BE500004EB8402064B03EBC202118904EB84025B
:10BE600003EBC20250680122F9F7C0FF10BD0000C9
:10BE7000C87F002010B5044604EB8402064B03EB98
:10BE8000C202118904EB840203EBC2025068002253
:10BE9000F9F7ACFF10BD0000C87F00202DE9F0418C
:10BEA00007460C4615461E464FF0000807EB870074
:10BEB0001C4901EBC000406AA04211D985B160194C
:10BEC00007EB8701174A02EBC101496A884207D88C
:10BED000154850F82600401E204008B9032E03DB09
:10BEE0004FF0FF30BDE8F08164B907EB87000D49E2
:10BEF00001EBC000406AA84204D83846FFF77CFF37
:10BF00000020EFE709E004EB08013246384600F074
:10BF10006FF9054850F826008044A845F3D3002067
:10BF2000E0E70000C87F00200026030838B504467B
:10BF300003226946204600F011F910B14FF0FF309E
:10BF400038BD9DF80000FF2810D19DF80100FF28A2
:10BF50000CD19DF80200FF2808D103226946204633
:10BF600000F0FCF810B14FF0FF30E9E79DF8020057
:10BF7000152806D016280DD0172814D0182824D13B
:10BF80001AE04FF4800004EB8401164A02EBC10171
:10BF9000486223E04FF4800004EB8401114A02EB75
:10BFA000C10148621AE04FF4000004EB84010D4A1D
:10BFB00002EBC101486211E04FF0807004EB840194
:10BFC000084A02EBC101486208E04FF4800004EB2C
:10BFD0008401044A02EBC101486200BF00BF002097
:10BFE000AEE70000C87F00202DE9F04782460C46EE
:10BFF00090461D46DDF8209000260027E0B2C0F5EF
:10C000008077AF4200D92F46504600F04DF900B17D
:10C0100047E0504600F0C1F900B142E05046FFF75A
:10C0200029FF00220221504600F02EF900B13BE02A
:10C030000022C4F30741504600F026F900B133E076
:10C040000022C4F30721504600F01EF900B12BE096
:10C05000E1B20022504600F017F900B124E00026BA
:10C0600008E018F806100022504600F00DF900B163
:10C070001AE0761CBE42F4D35046FFF7E7FE504666
:10C0800000F07AF900B10CE0504600F00DF900B173
:10C0900007E0B9F1000F01D0C9F800700020BDE839
:10C0A000F0874FF0FF30FAE75046FFF7CFFE4FF032
:10C0B000FF30F4E730B500EB8004074D05EBC40416
:10C0C000241D44F8312000EB800405EBC404241D3A
:10C0D00004EBC104A38030BDC87F00202DE9F041EE
:10C0E00080460E4614461F4600254046FFF7C2FE16
:10C0F00000220321404600F0C7F800B128E00022EA
:10C10000C4F30741404600F0BFF800B120E0002230
:10C11000C4F30721404600F0B7F800B118E0E1B2DF
:10C120000022404600F0B0F800B111E0002507E021
:10C130007219FF21404600F0A7F800B108E06D1C1D
:10C14000BD42F5D34046FFF781FE0020BDE8F081F7
:10C150004046FFF77BFE4FF0FF30F7E72DE9F04157
:10C1600007460D46164600243846FFF783FE002298
:10C170009F21384600F088F800B111E0002407E064
:10C180002A19FF21384600F07FF800B108E0641C4E
:10C19000B442F5D33846FFF759FE0020BDE8F081E0
:10C1A0003846FFF753FE4FF0FF30F7E770B506460D
:10C1B0000C4600253046FFF75DFE00220521304683
:10C1C00000F062F805462DB92246FF21304600F006
:10C1D0005BF805463046FFF739FE284670BD000083
:10C1E00000EB8002014B03F832107047C87F00203B
:10C1F00070B506460C461546214850F82500401EED
:10C200008443304600F0C9F800B130E03046FFF713
:10C2100031FE1C48415D0022304600F035F800B187
:10C2200028E00022C4F30741304600F02DF800B1A9
:10C2300020E00022C4F30721304600F025F800B1C9
:10C2400018E0E1B20022304600F01EF800B111E023
:10C250003046FFF7FBFD304600F08EF800B106E0F7
:10C26000304600F021F800B101E0002070BD4FF031
:10C27000FF30FBE73046FFF7E9FD4FF0FF30F5E711
:10C28000002603080C26030837B50446154604EBC0
:10C290008401044A12F83100012301AA294600F062
:10C2A000A1F83EBDC87F002038B505460024002017
:10C2B000009000BF69462846FFF778FF044604B1A6
:10C2C00005E09DF8000000F001000028F2D100BF59
:10C2D000204638BD2DE9FC4104460D4617461E4652
:10C2E0004FF000080020019004EB8400214901EB8D
:10C2F000C000406AA84201D907B11EB94FF0FF3013
:10C30000BDE8FC8104EB84001A4901EBC000416ADE
:10C3100004EB8400174A02EBC000406A401E28402C
:10C32000081AB0420DD204EB8400114601EBC000A4
:10C33000416A04EB840002EBC000406A401E2840C2
:10C340000E1A13E001A833463A46294600902046CB
:10C35000FFF74AFE10B14FF0FF30D1E701980544D6
:10C36000019807440198361A01988044002EE9D1BB
:10C370000020C5E7C87F002070B504460025204690
:10C38000FFF778FD002204212046FFF77DFF0546D8
:10C390002046FFF75BFD284670BD70B504460025BA
:10C3A0002046FFF767FD002206212046FFF76CFFBD
:10C3B00005462046FFF74AFD284670BDF8B50446FD
:10C3C0000D4616462B46002280212046009600F09E
:10C3D0002DF828B1606D40F0200060650320F8BDA5
:10C3E0000020FCE7F8B506460D4617461C462DB959
:10C3F00022463946304600F06FF8F8BD642104FB50
:10C4000001F0A3B20449009051F826002A463946AB
:10C41000FAF79DFB0020F0E72406002002460248C0
:10C4200040F8221000207047240600202DE9F0413A
:10C4300004460E4617461D46DDF818803FE0681C8E
:10C44000E0B32DB1F9F7D8FCA0EB0800A84236D331
:10C450002068406820F0E000216848606068B0F51E
:10C46000827F0DD1A068B0F5004F03D0A068B0F571
:10C47000806F05D12068006820F0400021680860C6
:10C48000A06AB0F5005F0ED100BF206800684DF6CD
:10C49000FF710840216808602068006840F400507F
:10C4A0002168086000BF012084F8510000BF00200F
:10C4B00084F8500000BF0320BDE8F081FFE720684A
:10C4C00080683040B04201D1012000E00020B84235
:10C4D000B5D10020F0E7000070B505460E461446C1
:10C4E000642104FB01F3A2B2034951F8250031464F
:10C4F000FAF75AFA002070BD2406002070470000A9
:10C5000038B504460D460020009055201B490870A0
:10C51000AA20487003208870601DC870032008712D
:10C52000084645718471164800EB450122461348C0
:10C53000C01DF3F78CFE002008E0811C0F4A515CFF
:10C54000BDF80020114489B20091401C611D884251
:10C55000F3DB0A48801CF5F7C7F90090E01D074996
:10C560000844BDF8001001804FF47A7304F1090209
:10C5700002490448FBF7E3FB38BD00001C290020FA
:10C580009824002038E6002008B50948094B0A4ADB
:10C590004FF4806100900948FDF79FFA0849086050
:10C5A0000846064902680748006801F029FB08BDF3
:10C5B000B5C4002074C400208837030835C50020A6
:10C5C000740500206005002010B5084B084A4FF4A0
:10C5D00080610848FDF781FA074908600846054967
:10C5E00002680648006801F00BFB10BDB5C40020CE
:10C5F0000C37030835C500207405002060050020B5
:10C60000F0B507460C4615461E4672B6FFF756FBB8
:10C610003846FFF75FFB2046FFF75CFB2846FFF735
:10C6200059FB3046FFF756FB62B6F0BD10B5044625
:10C63000062C0BDA064850F82420064B1B7850F8DD
:10C64000231005A0FBF72CFF02480470002010BD4A
:10C650008C0500205C050020436C69656E74537482
:10C660006174652066726F6D205B25735D20636861
:10C67000616E676520746F205B25735D0D0A000095
:10C6800070B504460D46022C0FD0FCF70FFF50B1D9
:10C69000FCF70CFFD0F8900528B1FCF707FFD0F8A5
:10C6A000906504A0B047002070BD6868FEF77AFA74
:10C6B0000020F9E74552524F520D0A0070B5054669
:10C6C0000E460220FEF756FAFCF7F0FE50B1FCF7DA
:10C6D000EDFED0F8900528B1FCF7E8FED0F89045C3
:10C6E00001A0A047002070BD4F4B0D0A00000000C4
:10C6F0002DE9F04105460E46022D0DD0FCF7D6FE81
:10C7000050B1FCF7D3FED0F8900528B1FCF7CEFE6F
:10C71000D0F8907529A0B8477068F3F71EFE04465C
:10C720009CB90020F5F786FAFCF7C0FE002842D03D
:10C73000FCF7BCFED0F8900500283CD0FCF7B6FE14
:10C74000D0F8907520A0B84735E0012C11D1FCF746
:10C75000ADFE50B1FCF7AAFED0F8900528B1FCF769
:10C76000A5FED0F8907518A0B8470120F5F762FA39
:10C7700021E0022C11D1FCF799FE50B1FCF796FE96
:10C78000D0F8900528B1FCF791FED0F890750EA076
:10C79000B8470220F5F74EFA0DE0FCF787FE50B1DE
:10C7A000FCF784FED0F8900528B1FCF77FFED0F8A6
:10C7B000907503A0B8470020BDE8F0814172672062
:10C7C0004552524F520D0A004F4B0D0A0000000017
:10C7D0002DE9F04180460D466868F3F7BEFD04463A
:10C7E0004FF47A70B4FBF0F001036420B4FBF0F076
:10C7F0000A22B0FBF2F302FB130001EB0021B4FBB1
:10C80000F2F0B0FBF2F302FB130001EB0010114653
:10C81000B4FBF1F201FB124146180C498E80084628
:10C8200080880B49086005F07DFDFCF73FFE50B1A4
:10C83000FCF73CFED0F8900528B1FCF737FED0F8A5
:10C84000907504A0B8470020BDE8F081982400202E
:10C85000CC0100204F4B0D0A0000000070B50446CB
:10C860000E46022C10DAFCF721FE50B1FCF71EFE3A
:10C87000D0F8900528B1FCF719FED0F8905503A028
:10C88000A8474FF0FF3070BD0020FCE7646562757B
:10C89000675F6F666620666C61670D0A00000000C6
:10C8A00070B504460E46022C10DAFCF7FFFD50B1BD
:10C8B000FCF7FCFDD0F8900528B1FCF7F7FDD0F8A7
:10C8C000905503A0A8474FF0FF3070BD0020FCE753
:10C8D00064656275675F6F6E20666C61670D0A0044
:10C8E0002DE9F04105460E46022D0DD0FCF7DEFD88
:10C8F00050B1FCF7DBFDD0F8900528B1FCF7D6FD70
:10C90000D0F8907511A0B8477068F3F726FD04467B
:10C91000C4F30F201049A1F85200A1F8544005F0CB
:10C9200001FD2146022003F0F9FAFCF7BFFD50B1EA
:10C93000FCF7BCFDD0F8900528B1FCF7B7FDD0F8A6
:10C94000907506A0B8470020BDE8F08141726720CD
:10C950004552524F520D0A00982400204F4B0D0AA9
:10C96000000000002DE9F04106460F46FCF79EFD51
:10C9700058B1FCF79BFDD0F8900530B1FCF796FD5F
:10C980001EA1D0F8904520A0A047FCF78FFD70B104
:10C99000FCF78CFDD0F8900548B1FEF7A7F80546E6
:10C9A000FCF784FD2946D0F890451DA0A047FCF770
:10C9B0007DFD70B1FCF77AFDD0F8900548B1FEF727
:10C9C00091F80546FCF772FD2946D0F890451AA06B
:10C9D000A047FCF76BFD70B1FCF768FDD0F890053F
:10C9E00048B1FEF787F80546FCF760FD2946D0F808
:10C9F000904517A0A0470020BDE8F08156323032A4
:10CA0000313035313030300056657273696F6E3AAF
:10CA100020202020202020202025730D0A00000047
:10CA2000494D45493A202020202020202020202048
:10CA30002025730D0A000000434349443A2020207A
:10CA400020202020202020202025730D0A00000017
:10CA5000494D53493A20202020202020202020200A
:10CA60002025730D0A00000010B522210248FCF7B2
:10CA700097FC002010BD0000CC24030870B50446CC
:10CA80000E46022C10D0FCF711FD50B1FCF70EFD44
:10CA9000D0F8900528B1FCF709FDD0F890550AA010
:10CAA000A8474FF0FF3070BDFCF700FD50B1FCF718
:10CAB000FDFCD0F8900528B1FCF7F8FCD0F89055B3
:10CAC00006A0A8470020EEE775736167653A206C01
:10CAD0006F6720737472696E670D0A004F4B0D0A01
:10CAE0000000000070B505460E46FCF7DFFC50B1B3
:10CAF000FCF7DCFCD0F8900528B1FCF7D7FCD0F8A7
:10CB0000904502A0A047002070BD00004F4B0D0AC9
:10CB1000000000002DE9F04104460F460026032CDA
:10CB200011D0FCF7C3FC50B1FCF7C0FCD0F8900565
:10CB300028B1FCF7BBFCD0F8905504A0A8474FF0F3
:10CB4000FF30BDE8F0810020FBE7000075736167EE
:10CB5000653A206C6F675F7072696E7420617363F1
:10CB60005B302D315D20636E740D0A00024600209B
:10CB700070470000F8B505460C46022D10D0FCF7B2
:10CB800095FC50B1FCF792FCD0F8900528B1FCF769
:10CB90008DFCD0F890651AA0B0474FF0FF30F8BD7B
:10CBA0004CF6CC4000901BA0FBF77AFC002302223D
:10CBB0004FF488311846FFF771F902236A464FF4A3
:10CBC00088310020FFF786FB00234FF480724FF47A
:10CBD00090311846FFF762F96068F3F784FB461C52
:10CBE00033464FF4903100206268FFF773FB0A2050
:10CBF00004F0E3FB0020FFF7A5F80020CFE70000DA
:10CC000075736167653A206F74612075726C0D0AE7
:10CC100000000000676F746F206F74612061707096
:10CC20006C69636174696F6E0D0A000070B505462A
:10CC30000E460220FDF7AAFFFCF738FC50B1FCF7C6
:10CC400035FCD0F8900528B1FCF730FCD0F89045C1
:10CC500001A0A047002070BD4F4B0D0A000000004E
:10CC600070B505460E460020FDF784FFFCF71EFC5C
:10CC700050B1FCF71BFCD0F8900528B1FCF716FC6E
:10CC8000D0F8904501A0A047002070BD4F4B0D0A81
:10CC90000000000070B505460E460020FDF776FF47
:10CCA000FCF704FC50B1FCF701FCD0F8900528B16A
:10CCB000FCF7FCFBD0F8904501A0A047002070BD18
:10CCC0004F4B0D0A0000000070B504460E46022CC2
:10CCD00010D0FCF7EBFB50B1FCF7E8FBD0F8900567
:10CCE00028B1FCF7E3FBD0F890550AA0A8474FF015
:10CCF000FF3070BDFCF7DAFB50B1FCF7D7FBD0F882
:10CD0000900528B1FCF7D2FBD0F8905508A0A847B1
:10CD10000020EEE775736167653A207274635F7394
:10CD200065745F616C61726D207365630D0A00004C
:10CD30004F4B0D0A00000000024600207047000023
:10CD400070B504460E46072C10D0FCF7AFFB50B16F
:10CD5000FCF7ACFBD0F8900528B1FCF7A7FBD0F8A6
:10CD6000905503A0A8474FF0FF3070BD0020FCE7AE
:10CD700075736167653A207274635F7365742079B7
:10CD8000797979206D6D206464206868206D6D204C
:10CD900073730D0A0000000070B504460D460020B4
:10CDA000FEF7D0FF002070BD2DE9F04107460E468A
:10CDB000032F0DD0FCF77AFB50B1FCF777FBD0F8CE
:10CDC000900528B1FCF772FBD0F890851FA0C047F2
:10CDD0007068F3F7C2FA0446B068F3F7BEFA054686
:10CDE000142C22DC002C20DD322D1EDC002C1CDD5E
:10CDF0001949A1F870404FF47A7090FBF5F0C880A3
:10CE000005F090FAFCF752FB50B1FCF74FFBD0F85D
:10CE1000900528B1FCF74AFBD0F890850FA0C047D9
:10CE200001200D49A1F860000DE0FCF73FFB50B177
:10CE3000FCF73CFBD0F8900528B1FCF737FBD0F8A5
:10CE4000908502A0C0470020BDE8F08141726720B4
:10CE50004552524F520D0A00982400204F4B0D0AA4
:10CE60000000000070B505460C46062D10DAFCF7F0
:10CE70001DFB50B1FCF71AFBD0F8900528B1FCF768
:10CE800015FBD0F890651EA0B0474FF0FF3070BD85
:10CE90001DA220211D48636803F0C8FCA068FCF7B0
:10CEA00054FE1B49A1F8A00217A2202117482230E6
:10CEB000E36803F0BBFC14A220211448423023692C
:10CEC00003F0B4FC10A2202110486230636903F023
:10CED000ADFC05F027FAFCF7E9FA50B1FCF7E6FAE9
:10CEE000D0F8900528B1FCF7E1FAD0F8906509A0D8
:10CEF000B04701200649A1F860000020C7E7000004
:10CF00004552524F520D0A00257300001827002089
:10CF1000982400204F4B0D0A0000000070B5054614
:10CF20000C46052D10DAFCF7C1FA50B1FCF7BEFA39
:10CF3000D0F8900528B1FCF7B9FAD0F890651BA09D
:10CF4000B0474FF0FF3070BD1AA220211A48636825
:10CF500003F06CFC17A2202117482030A36803F0CF
:10CF600065FC14A2202114484030E36803F05EFC05
:10CF700010A2202110486030236903F057FC05F00F
:10CF8000D1F9FCF793FA50B1FCF790FAD0F890057C
:10CF900028B1FCF78BFAD0F8906508A0B0470120C3
:10CFA0000849A1F860000020CDE700004552524F2B
:10CFB000520D0A0025730000982600204F4B0D0AE1
:10CFC0000000000098240020F8B505460C46022D0C
:10CFD00010DAFCF76BFA50B1FCF768FAD0F890055C
:10CFE00028B1FCF763FAD0F8906516A0B0474FF06F
:10CFF000FF30F8BD69466068FCF732FC6068FCF7FA
:10D00000A4FD1249B1F85610884205D06068FCF7BB
:10D010009CFD0E49A1F8560005F084F9FCF746FA8C
:10D0200050B1FCF743FAD0F8900528B1FCF73EFA6E
:10D03000D0F8906506A0B04701200449A1F860002F
:10D040000020D6E74552524F520D0A009824002086
:10D050004F4B0D0A00000000F8B505460C46032DA5
:10D0600010DAFCF723FA50B1FCF720FAD0F890055B
:10D0700028B1FCF71BFAD0F8906528A0B0474FF014
:10D08000FF30F8BD69466068FCF7EAFB9DF80000D8
:10D090002449498C884211D19DF801002149898C8D
:10D0A00088420BD19DF802001E49C98C884205D1E7
:10D0B0009DF803001B49098D88420CD09DF80000A3
:10D0C000184948849DF8010088849DF80200C884AE
:10D0D0009DF803000885A068FCF737FD1149098B0E
:10D0E000884204D0A068FCF730FD0E49088305F0A3
:10D0F00019F9FCF7DBF950B1FCF7D8F9D0F8900535
:10D1000028B1FCF7D3F9D0F8906507A0B04701200B
:10D110000449A1F860000020B3E700004552524FD7
:10D12000520D0A00982400204F4B0D0A0000000009
:10D13000F8B505460C46032D10DAFCF7B7F950B1E7
:10D14000FCF7B4F9D0F8900528B1FCF7AFF9D0F8A6
:10D1500090652DA0B0474FF0FF30F8BD694660687C
:10D16000FCF77EFB9DF800002949B1F86610884263
:10D1700014D19DF801002649B1F8681088420DD1FC
:10D180009DF802002249B1F86A10884206D19DF844
:10D1900003001F49B1F86C10884210D09DF80000C0
:10D1A0001B49A1F866009DF80100A1F868009DF8F0
:10D1B0000200A1F86A009DF80300A1F86C00A068C5
:10D1C000FCF7C3FC1249B1F86E10884205D0A06884
:10D1D000FCF7BBFC0E49A1F86E0005F0A3F8012096
:10D1E0000B49A1F86000FCF761F950B1FCF75EF95A
:10D1F000D0F8900528B1FCF759F9D0F8906505A052
:10D20000B0470020A9E700004552524F520D0A00D6
:10D21000982400204F4B0D0A00000000F8B5054689
:10D220000C46022D10DAFCF741F950B1FCF73EF93B
:10D23000D0F8900528B1FCF739F9D0F8906516A020
:10D24000B0474FF0FF30F8BD69466068FCF708FB57
:10D250006068FCF77AFC1249B1F85810884205D092
:10D260006068FCF772FC0E49A1F8580005F05AF806
:10D27000FCF71CF950B1FCF719F9D0F8900528B16A
:10D28000FCF714F9D0F8906506A0B04701200449D6
:10D29000A1F860000020D6E74552524F520D0A0017
:10D2A000982400204F4B0D0A000000000246002089
:10D2B0007047000070B505460C461646214602A090
:10D2C000FBF7EEF870BD00004576656E743A257583
:10D2D0000D0A00002DE9F04104460D46022C0DD048
:10D2E000FCF7E4F850B1FCF7E1F8D0F8900528B16C
:10D2F000FCF7DCF8D0F8906514A0B0476868F3F745
:10D300002CF80746384600F0E7F970B9FCF7CEF87C
:10D31000C8B1FCF7CBF8D0F89005A0B1FCF7C6F87F
:10D32000D0F890650CA0B0470DE0FCF7BFF850B105
:10D33000FCF7BCF8D0F8900528B1FCF7B7F8D0F8A6
:10D34000906503A0B0470020BDE8F08141726720DE
:10D350004552524F520D0A004F4B0D0A000000007B
:10D360002DE9F04705460C46042D0DD0FCF79EF83C
:10D3700050B1FCF79BF8D0F8900528B1FCF796F86F
:10D38000D0F8908518A0C0476068F2F7E6FF8146A4
:10D39000A668E068F2F7E1FF87B23A4631464846B0
:10D3A00000F0E2F970B9FCF781F8C8B1FCF77EF83B
:10D3B000D0F89005A0B1FCF779F8D0F890850DA0D1
:10D3C000C0470DE0FCF772F850B1FCF76FF8D0F8E9
:10D3D000900528B1FCF76AF8D0F8908503A0C04703
:10D3E0000020BDE8F0870000417267204552524F8F
:10D3F000520D0A004F4B0D0A00000000F8B505461B
:10D400000E46002000900023194A0121684600F0D2
:10D41000D1F9E8B9FCF74AF858B1FCF747F8D0F869
:10D42000900530B1FCF742F8D0F8904511A0009972
:10D43000A047FCF73BF8C8B1FCF738F8D0F89005E6
:10D44000A0B1FCF733F8D0F890450DA0A0470DE04F
:10D45000FCF72CF850B1FCF729F8D0F8900528B16A
:10D46000FCF724F8D0F8904507A0A0470020F8BDAD
:10D47000B5D20208536F636B49443A25750D0A0013
:10D480004F4B0D0A000000004552524F520D0A004A
:10D490002DE9F04106460C46032E0DD0FCF706F8A8
:10D4A00050B1FCF703F8D0F8900528B1FBF7FEFF68
:10D4B000D0F8907518A0B8476068F2F74EFF804624
:10D4C000A5682846F2F70FFF07463A462946404628
:10D4D00000F096FB70B9FBF7E9FFC8B1FBF7E6FF78
:10D4E000D0F89005A0B1FBF7E1FFD0F890750DA042
:10D4F000B8470DE0FBF7DAFF50B1FBF7D7FFD0F8E4
:10D50000900528B1FBF7D2FFD0F8907503A0B8477B
:10D510000020BDE8F0810000417267204552524F63
:10D52000520D0A004F4B0D0A0000000070B5044672
:10D530000D46042102A000F029FF002070BD00006C
:10D54000B2E2CAD400000000F8B505460E464AF61D
:10D55000AA200090FBF7AAFF50B1FBF7A7FFD0F875
:10D56000900528B1FBF7A2FFD0F890450AA0A0478C
:10D57000002302224FF488311846FEF78FFC022365
:10D580006A464FF488310020FEF7A4FE01200549C9
:10D59000A1F860000020F8BD757064617465204FCB
:10D5A0004B0D0A009824002070B5B2B004460E4618
:10D5B000214608A0FAF774FF234606A2C821684650
:10D5C000FCF78BFAC5B22946684602F021F832B062
:10D5D00070BD00003447207369676E616C20696E0E
:10D5E00074656E736974792069732025750D0A005E
:10D5F000F8B505460C46164634B1012C15D0022C60
:10D6000044D0032C5AD156E02E480078012803D08C
:10D610002C480078042807D10020FFF707F80022E3
:10D6200011466420F4F770F949E0002026490860AB
:10D6300024480078012812D1FEF7C6FF00202349B4
:10D6400008700220FEF7F2FF0020214B47F2305213
:10D65000014600901F480068FCF716F815E01948CD
:10D660000078042811D1FEF78FFF002017490870B9
:10D670000320FEF7DBFF0020154B47F23052014636
:10D68000009014480068FBF7FFFF18E00D48007891
:10D69000042800D113E00F480068FBF753FF094846
:10D6A000007838B10020FEF7C1FF00221146652046
:10D6B000F4F72AF903E0FDF73DFC00E000BF00BFEE
:10D6C000F8BD00005C050020780500205D05002005
:10D6D0008DE40208640500200246C2EB8210C0EB14
:10D6E00000100A4B03EB8001002A02DB032A00DA58
:10D6F00011B94FF0FF307047087820B10878012841
:10D7000001D0052008700020F5E70000A880002067
:10D7100070B50025002400BF1FE0C5EB8510C0EBED
:10D720000010104901EB80042078032804D004285D
:10D7300003D006280ED101E000BF00BF0020A0707A
:10D7400001202070A06820B102212846D4E90232CD
:10D75000984700E000BF00BF6D1C032DDDDB0020FB
:10D7600070BD0000A88000202DE9F04104460E465F
:10D770001746C4EB8410C0EB00100C4901EB800588
:10D78000002C02DB032C00DA1DB94FF0FF30BDE89E
:10D79000F081334606A22A2105F11000FCF79DF91D
:10D7A0006F87032028700020F1E70000A880002088
:10D7B000257300002DE9F04707460E46904699462E
:10D7C0000025002400BF38E0C5EB8510C0EB001039
:10D7D0001C4901EB800474B3207860BB40F6C4613F
:10D7E0002046FBF7FDFF6560667002202070C4F8DC
:10D7F0000880C4F80C9010234FF4C06204F1C401F7
:10D8000004F13C00FCF756FA012E08D10123DA029C
:10D8100004F2C46104F1B000FAF7D7FC07E010236A
:10D82000DA0104F2C46104F16C00FCF743FA3D60D4
:10D830000020BDE8F087FFE76D1C032DC4DB4FF02F
:10D84000FF30F6E7A88000200146032908DAC1EB83
:10D850008110C0EB0010034A02EB800010307047CB
:10D8600001A0FCE7A8800020000000000146032979
:10D8700008DAC1EB8110C0EB0010034A02EB800014
:10D88000408F70470020FCE7A88000200146032954
:10D8900008DAC1EB8110C0EB0010034A02EB8000F4
:10D8A0003C3070470020FCE7A88000200146032997
:10D8B00007DAC1EB8110C0EB0010034A12F8200018
:10D8C00070470020FCE70000A880002001460329E3
:10D8D00008DAC1EB8110C0EB0010034A02EB8000B4
:10D8E000407870470020FCE7A8800020014603290B
:10D8F00008DAC1EB8110C0EB0010034A02EB800094
:10D90000807870470020FCE7A880002001460329AA
:10D910000ADA0120C1EB8112C2EB0212044B03EBC5
:10D9200082029070002070474FF0FF30FBE700004C
:10D93000A88000200146032909DA0020C1EB8112EA
:10D94000C2EB0212034B03EB8202907070474FF060
:10D95000FF30FBE7A880002070B50546C5EB8510B9
:10D96000C0EB00100D4901EB8004002D02DB032DFC
:10D9700000DA14B94FF0FF3070BD2078042801D1CF
:10D98000401FF9E701202070A06820B1022128463D
:10D99000D4E9023298470020EEE70000A88000207A
:10D9A00070B50546C5EB8510C0EB00100A4901EBC8
:10D9B0008004002D02DB032D00DA14B94FF0FF3094
:10D9C00070BD07202070A06820B100212846D4E94E
:10D9D000023298470020F3E7A880002070B5054682
:10D9E000C5EB8510C0EB0010184901EB8004002D39
:10D9F00002DB032D00DA14B94FF0FF3070BD0620B2
:10DA000020701023020204F1C40104F13C00FCF771
:10DA100051F96078012808D10123C20204F2C461DF
:10DA200004F1B000FAF7D1FB07E01023DA0104F2A9
:10DA3000C46104F16C00FCF73DF9A06820B101213C
:10DA40002846D4E9023298470020D7E7A880002072
:10DA500070B50446C4EB8410C0EB0010094901EB1B
:10DA60008005002C02DB032C00DA15B94FF0FF30E3
:10DA700070BDA86820B103212046D5E9023298473D
:10DA80000020F5E7A88000202DE9F84F07468846DA
:10DA900091461D464FF0FF3000900024C7EB8710E1
:10DAA000C0EB0010224901EB8006002F03DB032F9F
:10DAB00001DA06B11DB94FF0FF30BDE8F88F70787C
:10DAC00001281BD14FF0000A4FF0000B00BF0EE001
:10DAD00008EB0A0106F1B000FAF79EFB18B1C5F891
:10DAE00000B00020E9E70BF1010B0AF1010ACA4579
:10DAF000EED3C5F800B00020009016E006F16C00EF
:10DB0000FCF78DF8044684B16068484508D2404669
:10DB1000D4E90012F2F79BFB6068286000200090B7
:10DB2000214606F16C00FCF752F80098C5E70000AA
:10DB3000A88000202DE9F047044689461546C4EB2D
:10DB40008410C0EB0010254901EB80060027002C53
:10DB500002DB032C00DA1EB94FF0FF30BDE8F0877E
:10DB6000707801280FD100270AE009EB070106F1C0
:10DB7000B000FAF70DFB10B14FF0FF30EEE77F1C5D
:10DB8000AF42F2D328E000BFC4EB8411C1EB011116
:10DB9000124A02EB810101F16C002946FCF75EF8A4
:10DBA0008046B8F1000F12D02A464946D8F8000046
:10DBB000F2F74DFBC4EB8411C1EB0111074A02EBF4
:10DBC000810101F16C004146FCF715F803E02146A4
:10DBD00003A0FAF765FC00BF0020BFE7A880002083
:10DBE000536F636B65745B25755D205265637620AA
:10DBF0004275666665722046756C6C0D0A00000001
:10DC00002DE9F0410446884615460026C4EB8410F1
:10DC1000C0EB0010134901EB8007002C03DB032C41
:10DC200001DA07B11DB94FF0FF30BDE8F081294698
:10DC300007F13C00FCF712F8064636B921460AA067
:10DC4000FAF72EFC4FF0FF30EFE72A4641463068E6
:10DC5000F2F7FDFA314607F13C00FBF7CCFF00205C
:10DC6000E3E70000A8800020736F636B65745B2599
:10DC7000645D2073656E64206275662066756C6CE9
:10DC80000D0A00000246032A08DAC2EB8210C0EB3C
:10DC90000010044B03F82010002070474FF0FF30B5
:10DCA000FBE70000A880002001460020044A12681B
:10DCB00090B24FF6C77210400843014A1060704797
:10DCC0000030014010B5FBF711FDF8F79BF8F9F7AC
:10DCD0007CF810BD10B592B000BF002000902F4816
:10DCE000006840F080502D4908600846006800F048
:10DCF0008050009000BF00BF00BF00200090284867
:10DD0000006820F4404040F400402549086008467F
:10DD1000006800F44040009000BF00BF0120069062
:10DD20000004079002200C9041050D9108210E91EE
:10DD3000A0210F91022110910421119106A8F8F75A
:10DD4000A9FA18B1D22117A002F05EFD0F200190B0
:10DD500002200290002003904FF480500490002095
:10DD60000590022101A8F8F757F918B1E0210DA09C
:10DD700002F04AFDF8F710FA4FF47A71B0FBF1F4B3
:10DD80002046F9F708F80420F8F7F0FF00221146C2
:10DD9000501EF8F7CEF812B010BD00004038024017
:10DDA000007000402E2E2F5372632F6D61696E2E0E
:10DDB000630000001348006840F4700011490860D7
:10DDC0001148006840F001000F49086000200E492A
:10DDD000083108600C4800680C4908400A4908608E
:10DDE0000B48091D0860081F006820F48020091FE7
:10DDF0000860002004490C31086006480149803958
:10DE00000860704788ED00E000380240FFFFF6FE32
:10DE1000103000240000020870B505460C46FBF7E0
:10DE2000D7FB0949086044B122462946022002F086
:10DE30000BFA10B105A0FAF733FB214609A0FAF757
:10DE40002FFB002070BD00009001002052544B2099
:10DE5000446174612053656E64204572726F720D67
:10DE60000A0000002575422052544B204461746121
:10DE70002053656E740D0A0010B500200449087027
:10DE80000023044A01210448FFF794FC002010BD40
:10DE90008C0100205DDF0208880100203EB5FCF700
:10DEA00026FA01283FD1FBF793FB0446204800786F
:10DEB00040BB20480078D8B901201D4908701E4891
:10DEC000008D1D49C98C1C4A928CCDE9002102901D
:10DED0001948438C19A24FF480611B48FBF7FDFDE4
:10DEE0001548028B184919480068FFF73DFC19E0F6
:10DEF00017480068201A1749884213D900200D4995
:10DF000008700FE00A48007802280BD11248006818
:10DF1000201A42F21071884204D30F480460002096
:10DF20000349087002E000200149087000203EBD4E
:10DF30008C010020940100209824002025752E25B6
:10DF4000752E25752E25750080290020880100205A
:10DF50009801002080EE360090010020F8B50646BA
:10DF60000C46174634B1012C0CD0022C12D0032CD5
:10DF700026D113E014480078012802D1002012496C
:10DF800008701EE010480078012802D102200E49D6
:10DF9000087016E000200C49087012E000250020EF
:10DFA00000906B4640F2FF32084909480068FFF7CD
:10DFB0006BFD05461DB905480099FFF72DFF00E0F0
:10DFC00000BF00BFF8BD00008C01002080290020A8
:10DFD0008801002010B50248F9F7B1F810BD000023
:10DFE000FCE5002000220268234B98420BD0B0F1E0
:10DFF000804F08D0214B984205D0214B984202D047
:10E00000204B984201D1012300E000231BB122F0F4
:10E0100070024B681A43184B984214D0B0F1804FED
:10E0200011D0164B98420ED0154B98420BD0154B81
:10E03000984208D0144B984205D0144B984202D015
:10E04000134B984201D1012300E000231BB122F4BD
:10E050004072CB681A4302608B68C3620B688362AC
:10E06000054B984201D1012300E000230BB10B695D
:10E070000363012343617047000001400004004036
:10E0800000080040000C00400040014000440140F6
:10E090000048014030B50023012404FA01F3046A6A
:10E0A0009C430462046A02FA01F52C43046230BD09
:10E0B00030B50C460021816821F47F4142EA0325F6
:10E0C00025432943816030BD0A460021816821F043
:10E0D000700142F0070319438160704730B5002496
:10E0E00000220023056A25F001050562026A4368E3
:10E0F000846924F0700424F003040D682C4322F09A
:10E1000002028D682A430D4DA84201D1012500E08D
:10E1100000256DB122F00802CD682A4322F00402E6
:10E1200023F4807323F400734D692B438D692B43D3
:10E13000436084614D684563026230BD0000014068
:10E1400030B5002400220023056A25F01005056281
:10E15000026A4368846924F4E04424F440740D683E
:10E1600044EA052422F020028D6842EA05120F4D90
:10E17000A84201D1012500E0002585B122F08002EE
:10E18000CD6842EA051222F0400223F4806323F4B2
:10E1900000634D6943EA85038D6943EA8503436063
:10E1A00084614D688563026230BD0000000001405B
:10E1B00030B5002400220023056A25F4807505622D
:10E1C000026A4368C46924F0700424F003040D68F3
:10E1D0002C4322F400728D6842EA05220E4DA842BB
:10E1E00001D1012500E0002585B122F40062CD684F
:10E1F00042EA052222F4806223F4805323F4005380
:10E200004D6943EA05138D6943EA05134360C46110
:10E210004D68C563026230BD0000014030B5002288
:10E2200000230024056A25F480550562036A4468CA
:10E23000C26922F4E04222F440720D6842EA0522EB
:10E2400023F400538D6843EA0533094DA84201D1F8
:10E25000012500E0002525B124F480444D6944EAFD
:10E2600085144460C2614D680564036230BD0000DE
:10E270000000014030B50B46144600210022026A1E
:10E28000056A25F001050562816921F0F00141EA86
:10E29000041122F00A021A438161026230BD30B5D6
:10E2A0000B46144600210022056A25F01005056280
:10E2B0008169026A21F4704141EA043122F0A0022E
:10E2C00042EA03128161026230BD000010B50248CB
:10E2D000FBF7A5FC10BD000038DD002010B50423BD
:10E2E0001A0203490348FBF7E5FC002010BD0000BB
:10E2F00038D9002038DD002070B505460E460420D0
:10E300000D49086006B115B94FF0FF3070BD3146B8
:10E310000A48FBF7A3FC044614B94FF0FF30F5E7B9
:10E32000324629462068F1F792FF21460348FBF761
:10E3300062FC0020EAE70000180C024038DD0020F3
:10E3400010B50446FFF7C2FFA04204D1214603489E
:10E35000FBF73DFC10BD0020FCE7000038DD00208D
:10E3600010B50248FBF75BFC10BD000068E100201F
:10E3700010B504231A0203490348FBF79BFC002055
:10E3800010BD000068DD002068E1002070B5054682
:10E390000E4604211248F7F721FD38B90420104930
:10E3A000183108604FF4487003F007F806B115B94A
:10E3B0004FF0FF3070BD31460A48FBF74FFC044672
:10E3C00014B94FF0FF30F5E7324629462068F1F7DF
:10E3D0003EFF21460348FBF70EFC0020EAE7000061
:10E3E000000C024068E1002010B50446FFF7B8FFBA
:10E3F000A04204D121460348FBF7E9FB10BD0020F1
:10E40000FCE7000068E1002010B50021002016E0C4
:10E410000E4A135C125C521C0C4C2254052B0CDA75
:10E420000B4A32F810200A4B23F811202246145CC4
:10E430000A464B1C99B2054B9C54421C90B2054AAB
:10E4400012889042E4DB034A118010BD2052002064
:10E450009C4E00207602002010B5044604A0FAF776
:10E460001FF8002008490860F3F7A8FA10BD000063
:10E470004E5452495020417070205265636F6E6E49
:10E480006563740D0A0000003802002010B50446D0
:10E4900003A0FAF705F808A0FBF736FC10BD000052
:10E4A0004E5452495020436C69656E742074696DF6
:10E4B00065206F75740D0A002E2E5C464D4C5C492C
:10E4C0006E7465726E65745C4E54524950436C694B
:10E4D000656E742E633A31383800000070B5054619
:10E4E000AC6B0020E085E0842046F9F7CBF870BDE6
:10E4F00070B506460025B46B20684069C0F3C015AE
:10E5000094F83900212805D125B10020E084204667
:10E5100000F082F820684069C0F3801594F83A0052
:10E52000222805D125B10020E085204600F054F8CE
:10E53000E06B40F01000E0632046F9F7A3F870BDEF
:10E5400070B50546AC6B2868006800F48070B0B9FF
:10E550000020E0852068C06820F480702168C860D1
:10E560002068406920F00100216848612068406906
:10E5700020F0400021684861202084F83A002046BD
:10E58000F9F7D6FB70BD70B50446A56B2846F9F7C0
:10E59000D5FB70BD70B50546AC6B2868006800F40B
:10E5A000807070B90020E0842068406920F080000D
:10E5B000216848612068C06840F040002168C86058
:10E5C00002E02046F9F7A0FC70BD70B50446A56BCB
:10E5D0002846F9F79FFC70BD0168C96821F4907165
:10E5E0000268D1600168496921F001010268516146
:10E5F000202180F83A10704710B504462068C068A2
:10E6000020F040002168C860202084F839002046AE
:10E61000F9F77AFC002010BD0168C96821F0C0013B
:10E620000268D160202180F83910704770B5044627
:10E6300094F83A00222844D1A068B0F5805F13D145
:10E64000A56A206940B920684068C0F308002880A6
:10E65000A06A801CA06219E020684068C0B22880CF
:10E66000A06A401CA06211E0206938B920684068A7
:10E67000C1B2A26A501CA062117007E02068406815
:10E6800000F07F01A26A501CA0621170E08D401E54
:10E6900080B2E08598B92068C06820F49070216845
:10E6A000C8602068406920F001002168486120208E
:10E6B00084F83A002046F9F73BFB002070BD0020AB
:10E6C000FCE70220FAE700002DE9F04104460025AE
:10E6D0002068056925F44055E06805432068056118
:10E6E0002068C56849F20C6085432169A068084329
:10E6F00061690843E169084305432068C5602068F3
:10E70000456925F44075A069054320684561E069C5
:10E71000B0F5004F7ED1C4492068884203D0C34978
:10E72000206888425DD1F7F74DFD00EBC00101EB99
:10E73000001061684900B0FBF1F06421B0FBF1F01A
:10E740000601F7F73FFD00EBC00101EB0010616827
:10E750004900B0FBF1F7F7F735FD00EBC00101EB25
:10E76000001061684900B0FBF1F06421B0FBF1F0EA
:10E7700000EBC00101EB0010A7EB8000322101EBA0
:10E78000C0006421B0FBF1F000F0F80006EB400699
:10E79000F7F718FD00EBC00101EB001061684900BC
:10E7A000B0FBF1F7F7F70EFD00EBC00101EB001035
:10E7B00061684900B0FBF1F06421B0FBF1F000EBBF
:10E7C000C00101EB0010A7EB8000322101EBC0007B
:10E7D0006421B0FBF1F000F007003044216888604C
:10E7E00020E1F7F7DFFC00EBC00101EB00106168EE
:10E7F0004900B0FBF1F06421B0FBF1F00601F7F73E
:10E80000D1FC00EBC00101EB001061684900B0FBD6
:10E81000F1F700E045E0F7F7C5FC00EBC00101EBC4
:10E82000001061684900B0FBF1F06421B0FBF1F029
:10E8300000EBC00101EB0010A7EB8000322101EBDF
:10E84000C0006421B0FBF1F000F0F80006EB4006D8
:10E85000F7F7A8FC00EBC00101EB0010616849006C
:10E86000B0FBF1F7F7F79EFC00EBC00101EB0010E5
:10E8700061684900B0FBF1F06421B0FBF1F000EBFE
:10E88000C00101EB0010A7EB8000322101EBC000BA
:10E890006421B0FBF1F000F007003044216888608B
:10E8A000C0E061492068884203D0604920688842FE
:10E8B0005CD1F7F787FC00EBC00101EB0010616849
:10E8C0008900B0FBF1F6F7F77DFC00EBC00101EB2E
:10E8D000001061688900B0FBF1F06421B0FBF1F039
:10E8E00000EBC00101EB0010A6EB8000322101EB30
:10E8F00000106421B0FBF1F000F0F006F7F762FCC5
:10E9000000EBC00101EB001061688900B0FBF1F081
:10E910006421B0FBF1F006EB0016F7F753FC00EBB7
:10E92000C00101EB001061688900B0FBF1F7F7F757
:10E9300049FC00EBC00101EB001061688900B0FBED
:10E94000F1F06421B0FBF1F000EBC00101EB00102D
:10E95000A7EB8000322101EB00106421B0FBF1F045
:10E9600000F00F003044216888605BE0F7F71AFC84
:10E9700000EBC00101EB001061688900B0FBF1F60B
:10E98000F7F710FC00EBC00101EB00106168890093
:10E99000B0FBF1F06421B0FBF1F000EBC00101EB42
:10E9A0000010A6EB8000322101EB00106421B0FBC7
:10E9B000F1F000F0F006F7F7F5FB00EBC00101EB1A
:10E9C000001061688900B0FBF1F06421B0FBF1F048
:10E9D00006EB0016F7F7E6FB00EBC00101EB0010B9
:10E9E00061688900B0FBF1F7F7F7DCFB00EBC001D1
:10E9F00001EB001061688900B0FBF1F06421B0FB0D
:10EA0000F1F000EBC00101EB0010A7EB8000322118
:10EA100001EB00106421B0FBF1F000F00F00304476
:10EA200021688860BDE8F0810010014000140140B9
:10EA3000014691F8390021282CD18868B0F5805F13
:10EA40000FD10A6A1088C0F308000B685860086983
:10EA500018B9086A801C086209E0086A401C08624C
:10EA600005E00B6A581C086218780B685860C88C5F
:10EA7000401E80B2C88458B90868C06820F0800081
:10EA80000B68D8600868C06840F040000B68D86028
:10EA9000002070470220FCE72DE9F04104460D46B6
:10EAA00017469846069E21E0701CF8B12EB1F7F784
:10EAB000A3F9A0EB0800B04218D92068C06820F480
:10EAC000D0702168C8602068406920F0010021688A
:10EAD0004861202084F8390084F83A0000BF002003
:10EAE00084F8380000BF0320BDE8F081206800688A
:10EAF0002840A84201D1012000E00020B842D3D034
:10EB00000020F1E72DE9F04FBFB00746884600240A
:10EB100000203290FD49FEA0F9F7C2FC0822FEA1B8
:10EB20003846F1F70BFC002870D10C2333AA2C21B6
:10EB30003846FAF7E9FF0446052C04D24FF0FF30BF
:10EB40003FB0BDE8F08F3498FAF77BFEF54989882D
:10EB5000884259D1002500263598FAF7F6FF054678
:10EB6000F048B0F87000A84203D0EE49A1F8705008
:10EB7000012631A93698FAF773FE9DF8C400E949D9
:10EB8000B1F86610884214D19DF8C500E549B1F886
:10EB9000681088420DD19DF8C600E249B1F86A10AC
:10EBA000884206D19DF8C700DE49B1F86C10884252
:10EBB00014D001269DF8C400DA49A1F866009DF83A
:10EBC000C500A1F868009DF8C600A1F86A009DF88C
:10EBD000C700A1F86C000020D34908703798FAF7F5
:10EBE000B4FFD049B1F86E10884206D03798FAF7D2
:10EBF000ACFFCC49A1F86E0001262EB103F092FBC8
:10EC00000120C849A1F8600089E3FFE70822C7A1F5
:10EC10003846F1F793FB002846D10C2333AA2C2168
:10EC20003846FAF771FF0446042C02D24FF0FF3049
:10EC300086E73498FAF705FEBA4989888842E3D115
:10EC4000BDA13698F1F756FB0028DDDD4CF6CC402F
:10EC50003190BCA0F9F724FC002302224FF4883144
:10EC60001846FDF71BF9022331AA4FF48831002022
:10EC7000FDF730FB00234FF480724FF490311846BB
:10EC8000FDF70CF93598F1F72EFB451C2B464FF498
:10EC900090310020359AFDF71DFB0A2002F08DFB14
:10ECA0000020FDF74FF83AE30822ACA13846F1F70F
:10ECB00045FB78B90C2333AA2C213846FAF724FFF8
:10ECC0000446032C02D24FF0FF3039E73498FAF7AC
:10ECD000B8FD24E30922A4A13846F1F72FFB002850
:10ECE00053D10C2333AA2C213846FAF70DFF0446E2
:10ECF000032C02D24FF0FF3022E73498FAF7A1FD3F
:10ED0000884989888842CED19AA13598F1F7F2FADC
:10ED100020B93698FAF719FF9849088098A13598D4
:10ED2000F1F7E8FA20B93698FAF70FFF974908701B
:10ED300097A13598F1F7DEFA0028B4D13698F1F7AB
:10ED4000D2FA054629463698FFF720FB7548838896
:10ED500090A24FF480616D48FAF7BFFE32906B4984
:10ED60009148329A0068FEF74BFF6E48838889A26B
:10ED70004FF480616548FAF7B0FE329063498A48E3
:10ED8000329A0068FEF73CFFC9E20A2287A13846A2
:10ED9000F1F7D4FA40B9F2F729FE022899D15B497C
:10EDA0005BA0F9F7A3FBBAE2092283A13846F1F789
:10EDB000C5FA40BB30A82EAB82A24146009038462F
:10EDC000FAF798FD02281DD10020DDE92E128854A3
:10EDD0002E98FAF736FD53498988884212D1DDE929
:10EDE0003001FFF789FA4F4883886AA24FF48061A7
:10EDF0004648FAF772FE329044496B48329A0068EE
:10EE0000FEF7FEFE8BE2092273A13846F1F796FA6F
:10EE100060BB0C2333AA2C213846FAF775FE044652
:10EE20003498FAF70EFD3F49898888421DD1022C9B
:10EE300002D24FF0FF3083E63598FAF786FE85B2AE
:10EE40003698FAF782FE86B2102D02D14B48068022
:10EE50000BE0B5F5007F02DA324820F8156003F0C8
:10EE600061FA01202F49A1F8600058E20A225DA151
:10EE70003846F1F763FA002846D10C2333AA2C2137
:10EE80003846FAF741FE04463498FAF7DAFC254989
:10EE90008988884239D1022C02D24FF0FF304FE6E8
:10EEA0003598FAF752FE86B23698FAF74EFE1FFAF8
:10EEB00080FB4FA1684601F0D1FC85B219498A88D0
:10EEC0000DEB05004DA101F0C9FC1FFA80F905EB1F
:10EED000090085B2B24610E0124931F81A200DEB54
:10EEE000050047A101F0BAFC1FFA80F905EB090003
:10EEF00085B20AF101001FFA80FA0BEB06005045BB
:10EF0000EADC652228467DE09DE09BE0802D002024
:10EF100025730D0A0000000024636F6E6669672C7C
:10EF20000000000098240020A001002024757064D7
:10EF30006174652C000000005632303231303531BA
:10EF400030303000676F746F204F54412041707033
:10EF50006C69636174696F6E0D0A000024676574E3
:10EF60006C6F672C0000000024636F6E74726F6C0E
:10EF70002C000000626565706572000004000020CE
:10EF80007577625F656E61626C6500002D00002020
:10EF9000545453002452656365697665766F6963DE
:10EFA000652C25580D0A00009C010020247573650E
:10EFB00072646174612C000024736574746F6E65F3
:10EFC0002C00000024736574746F6E652C25702C02
:10EFD00025700D0A00000000247365747061726171
:10EFE0002C0000002472656164706172612C000065
:10EFF000247265706C79706172612C0025782C0028
:10F0000025642C00691C8DB20DF800206E22284664
:10F01000691C8DB20DF8002064222846691C8DB24F
:10F020000DF800200D222846691C8DB20DF8002035
:10F030000A222846691C8DB20DF800202946684630
:10F0400000F0E6FA6BE11222B6A13846F1F776F944
:10F0500000287BD10C2333AA2C213846FAF754FD23
:10F060000446062C02D24FF0FF3069E53498FAF7D7
:10F07000E8FB1FFA80FA3598FAF7E3FB80B231908B
:10F080003698FAF762FD85B23798FAF75EFD86B2D8
:10F090003898FAF75AFD1FFA80F9A748BDF8C4104E
:10F0A0000180A6488088504502D04FF0FF3047E5E8
:10F0B00000204EE000EB4001A14A02EB41014988EB
:10F0C0009D4A1288914205D000EB40019C4A12F8FB
:10F0D0001110C1B99849098800EB4002984B03EB25
:10F0E0004202518000EB400203EB4202567000EBFB
:10F0F000400203F8125000EB40011A4602EB4101B6
:10F10000A1F8049027E01D2821D18E490A780978BA
:10F11000491C8C4B19701E2A02DB00211A46117003
:10F12000884A127802EB4202854B03EB420256708A
:10F13000844A127802EB420203F8125000EB4001BD
:10F140001A4602EB4101A1F8049004E005E0411CDD
:10F15000C8B21E28AEDB00BFE1E011227AA138461A
:10F16000F1F7ECF8E8BB0C2333AA2C213846FAF768
:10F17000CBFC0446032C02D24FF0FF30E0E434987D
:10F18000FAF75FFB80B231903598FAF7DEFC85B272
:10F19000C8264FF064096848BDF8C41001800020FB
:10F1A0004FE000EB4001664A02EB41014988624AA8
:10F1B0001288914205D000EB4001614A12F811100B
:10F1C000D1B95D49098800EB40025D4B03EB420277
:10F1D000518000EB400203EB4202567000EB40020C
:10F1E00000E032E003F8125000EB40011A4602EB57
:10F1F0004101A1F8049026E01D2820D151490A7848
:10F200000978491C4F4B19701E2A02DB00211A464F
:10F2100011704C4A127802EB4202494B03EB420256
:10F220005670484A127802EB420203F8125000EB83
:10F2300040011A4602EB4101A1F8049003E0411C91
:10F24000C8B21E28ADDB00BF69E0142243A13846D6
:10F25000F1F774F8E8BB0C2333AA2C213846FAF7EF
:10F2600053FC0446042C02D24FF0FF3068E4F6F75A
:10F27000E1FB4FF400413F48F5F746F83598F1F7C8
:10F2800032F83190042231A93A48F5F7C1F9319AA0
:10F29000521C39483599F5F7BBF94CF6CC40309003
:10F2A000AFF26030F9F7FCF8002302224FF4883106
:10F2B0001846FCF7F3FD022330AA4FF488310020F2
:10F2C000FDF708F800234FF480724FF49031184690
:10F2D00000E008E0FCF7E2FD0A2002F06EF80020F2
:10F2E000FCF730FD1BE0172224A13846F1F726F881
:10F2F000A8B90C2333AA2C213846FAF705FC04469A
:10F30000022C02D24FF0FF301AE43498FAF799FA3F
:10F31000204908703498FAF794FA1F4908700020C1
:10F320000EE40000247772697465706172615F6138
:10F330006E63686F722C0000A801002098240020E2
:10F3400080310020AA01002024726561647061721E
:10F35000615F616E63686F722C00000024646F77D8
:10F360006E6C6F61645F616E63686F7262696E2C50
:10F37000000000000080000800810008247365740C
:10F380005F757064617465616E63686F725F6D6FE5
:10F3900064652C00AB0100207701002070B58AB0B5
:10F3A00000242B48007802284FD12A480078089082
:10F3B000294890ED000B8DED060B284890ED000BD1
:10F3C0008DED040B264827490968274A1278CDE9B4
:10F3D000002102902548838825A24FF4806130489F
:10F3E000FAF77BFB044600260BE02E4931F8162085
:10F3F0002B4908192CA101F031FA05462C44701C48
:10F4000086B2144800788642EFDB00260BE02749DD
:10F4100031F916202249081925A101F01FFA0546E5
:10F420002C44701C86B20B4800788642EFDB1C49E6
:10F43000081900221EA101F011FA05462C442246AB
:10F4400017491C480068FEF7DBFB00200AB070BDBE
:10F45000A00100201B020020F8030020F003002080
:10F46000B47D0020000400201E020020982400200B
:10F47000246D657373616765322C68656172742CE5
:10F48000253034782C2530327525252C25642C2503
:10F49000732C256C662C256C662C256400000000FE
:10F4A000802D0020343E00202C2578008C40002048
:10F4B0002C2564009C01002010B50023034A022182
:10F4C0000348FEF777F9002010BD000091F502080F
:10F4D0009C0100203EB5FAF70AFF012837D11E48EB
:10F4E0000078D8B901201C4908701C4800881C49C4
:10F4F00009881C4A1288CDE9002102901A48038825
:10F500001AA24FF480611C48FAF7E7FA1B480288F8
:10F5100019491B480068FEF727F91BE00E480078E0
:10F52000022817D1FAF754F8044616480068201A42
:10F5300042F21071884209D3002013490870114823
:10F540000460FFF72BFF00201049087002E0002044
:10F550000149087000203EBDA0010020B20100203A
:10F56000B0010020AE010020AC01002025752E2541
:10F57000752E25752E257500802D0020B4010020E4
:10F580009C010020A4010020B6010020B70100204A
:10F59000F8B506460C46174634B1012C0CD0022CA7
:10F5A00012D0032C2AD113E016480078012802D18A
:10F5B00000201449087022E012480078012802D186
:10F5C0000220104908701AE000200E49087016E069
:10F5D0000025002000906B4640F2FF320A490B489C
:10F5E0000068FEF751FA05463DB900200649009A29
:10F5F000885405480099FFF785FA00E000BF00BF76
:10F60000F8BD0000A0010020802D00209C010020FA
:10F6100070B505460C4614480078022821D11349DC
:10F62000134A1268881822462946F0F710FE10483F
:10F63000006820440E490860F9F7CAFF0D490968BF
:10F64000401AC8280DD3F9F7C3FF0A4908600848D3
:10F650000649026808480068FEF7D2FA002004490B
:10F660000860002070BD0000A0010020343600209A
:10F67000C4010020C80100209C01002010B5F6F74D
:10F68000D9F900224FF410410748F6F7AFFB0022EA
:10F6900004210648F6F7AAFB642001F08EFE002044
:10F6A000FCF750FB10BD00000000024000040240C7
:10F6B00010B50248F7F7ECFF10BD000038E6002057
:10F6C00010B50248F7F7E4FF10BD000078E600200F
:10F6D00010B50248F7F7DCFF10BD0000B8E60020C7
:10F6E00010B5F9F775FF0E490968401AB0F57A7F31
:10F6F00005D3F9F76DFF0A49086000F017F8F9F72C
:10F7000067FF08490968401A0749C988884205D334
:10F71000F9F75EFF0349086000F03AF810BD0000F9
:10F7200024020020280200209824002010B5FEF7B3
:10F730006BFE10BD70B54FF480100F49886140F624
:10F740008C2001F044FE10200B49886102F03AF948
:10F7500004460CE002F036F90446FAF775FD284637
:10F76000691CCDB2142802DD04A001F04FF807484F
:10F770008442EFD170BD0000000002404457204990
:10F7800044204552524F522E0D0A00003001CADE6D
:10F79000F8B5002138E000202EE06B4A32F9103035
:10F7A0001446421C34F91220934223DD674D35F88C
:10F7B0001020254635F81050ABB2654D2C5C634ED9
:10F7C000451C36F8155026F810505F4E451C36F88B
:10F7D000155026F810505E4E451C755D35545B4E35
:10F7E000451C26F815201EB2574F27F81560584EB5
:10F7F000745500BF421C90B2564A1278521E521ADB
:10F800008242CADC481C81B252480078401E8842BD
:10F81000C1DC50480078002809DD4F48006818B95D
:10F8200088204D49086002E000204B4908604B48A1
:10F8300003684B4802684B48016847480068FCF77A
:10F84000DFFE44480078142802DD14204149087086
:10F850001220454988703F48007800EB80000F3047
:10F86000C8700846414909888180414800783E496E
:10F8700088713F4801880088401C3D4A108008126A
:10F880003949C8713B48007808723B4800783B49C9
:10F89000097840EA41003A49097840EA810039494B
:10F8A000097840EA41103849097840EA81102E4928
:10F8B00048720020087348738873C873254800781D
:10F8C0000874244800784200204927481130F0F796
:10F8D000BEFC204909784A001E490978112303EB30
:10F8E0004101214BC8181849F0F7B1FC19490978B2
:10F8F000112202EB81011C4A881816490A78144922
:10F90000F0F7A5FC1348007800EB800000F10F0130
:10F910001548801CF1F7E8FF00900E48007800EBD6
:10F920008000113010490844BDF8001001800948DA
:10F93000007800EB800000F113010B48FAF70CFB94
:10F94000002004490870F8BD8C400020343E00209F
:10F95000E44200201B020020640600207006002004
:10F960006C0600206806002064160020CC010020F0
:10F97000180200201E0200202C0000200800002099
:10F980001A010020090000202E00002038B50020B8
:10F99000009000212D4802F093F800210F2001F083
:10F9A000F5FF2B4908600846008800F480400028D5
:10F9B0003AD04FF4804200210F2002F082F900215A
:10F9C000102001F0E3FFC4B200222146214802F0DA
:10F9D00031F82048B0F8010000901F48007850B17D
:10F9E0001C48407A302806D100201B490870BDF819
:10F9F00000001A490880BDF80000184909888842AB
:10FA000019D1022216491348401DF0F781FC90B924
:10FA10001048407A30280ED10120124908600D4864
:10FA2000807A1149087006E001F06AFE0F4A002151
:10FA30000F2002F046F90121044802F041F80020AD
:10FA400002F084F8002002F009F838BD00D0232429
:10FA50006C03002024650020AB0100207801002009
:10FA600070030020600300206B0300200090272417
:10FA70002DE9F04104460D464FF0FF360DB1032C41
:10FA800003DB4FF0FF30BDE8F08104EB4400C0EB36
:10FA90004410554901EB80008078002874D100BFE4
:10FAA00000BF04EB4402C2EB44120B4603EB82029C
:10FAB000926804EB4403C3EB44130F4607EB830344
:10FAC000DB681A4404EB4403C3EB441307EB8303E2
:10FAD0005B685B6B1B685B68D11A04EB4402C2EB8A
:10FAE00044123B4603EB8202D2680A4404EB44030F
:10FAF000C3EB441307EB83031B69D21A04EB4403E3
:10FB0000C3EB441307EB8303DB68B2FBF3F703FBA0
:10FB1000172001280DD84BD104EB4402C2EB44124C
:10FB2000314B03EB820252681268126802F0200225
:10FB30005ABB04EB4402C2EB44122B4B03EB820290
:10FB4000126912782A7004EB4402C2EB441203EBF0
:10FB50008202126904EB4403C3EB4413224F07EB08
:10FB600083035B699A4211D104EB4402C2EB441255
:10FB70003B4603EB8202926804EB4403C3EB44135D
:10FB800007EB83031A6112E013E011E004EB440277
:10FB9000C2EB4412144B03EB82021269521C04EBB9
:10FBA0004403C3EB4413104F07EB83031A61002691
:10FBB00017E004EB4400C0EB44100B4901EB80005C
:10FBC000807801280DD104EB4401C1EB4411064AB1
:10FBD00002EB810101F118002946F8F71DFB00B97D
:10FBE000002630464FE7000098E10020024609B1A8
:10FBF000032A02DB4FF0FF30704702EB4200C0EBFC
:10FC00004210034B03EB8000406808600020F3E7DC
:10FC100098E100202DE9F04105460C460CB1032D7A
:10FC200003DB4FF0FF30BDE8F08105EB4500C0EB92
:10FC30004510524901F82050207805EB4501C1EBF1
:10FC400045114E4A02EB81014870607805EB450191
:10FC5000C1EB451102EB8101887005EB4501C1EB59
:10FC6000451102EB81016068886005EB4501C1EB3D
:10FC7000451102EB8101A068C860607838BB05EBD4
:10FC80004500C0EB4510114601EB8000806805EB94
:10FC90004501C1EB451102EB8101086105EB45000F
:10FCA000C0EB4510114601EB8000806805EB450173
:10FCB000C1EB451102EB8101C9680844401E05EB08
:10FCC0004501C1EB451102EB8101486110E060780C
:10FCD00001280DD105EB4503C3EB4513274E06EB79
:10FCE000830303F118000123D4E90112F8F76DFA38
:10FCF00005EB4501C1EB4511204A02EB8101E068AB
:10FD0000C86205EB4501C1EB451102EB8101206999
:10FD1000086305EB4501C1EB451102EB8101A069C8
:10FD2000086705EB4501C1EB451102EB81016069F4
:10FD30004863207810B1207801280DD105EB4506E5
:10FD4000C6EB45160D4F07EB860606F13800D4E9E1
:10FD50000423E168F9F7AEFF607818B9284600F08F
:10FD60000FF808E06078012802D06078022802D1FC
:10FD7000284600F083F8002055E7000098E10020B5
:10FD80007CB5044628E004EB4400C0EB44103A493B
:10FD900001EB800040680068406880B20190BDF8C7
:10FDA0000400019000BF0020009004EB4400C0EB71
:10FDB000441001EB8000406800680068009004EB8C
:10FDC0004400C0EB441001EB8000406800684068CC
:10FDD000009000BF00BF00BF04EB4400C0EB441024
:10FDE000254901EB800040680068006800F00800C9
:10FDF0000028C8D104EB4400C0EB441001EB8000A4
:10FE0000806804EB4401C1EB44111B4A02EB810101
:10FE1000086104EB4400C0EB4410114601EB800084
:10FE2000806804EB4401C1EB441102EB8101C96815
:10FE30000844401E04EB4401C1EB441102EB810174
:10FE4000486104EB4403C3EB4413154605EB8303FD
:10FE50009B899AB204EB4403C3EB441305EB830381
:10FE6000996804EB4403C3EB441305EB8303586820
:10FE7000F7F7CAFE7CBD000098E100201CB50446DF
:10FE800028E004EB4400C0EB4410234901EB800060
:10FE900040680068406880B20190BDF8040001909D
:10FEA00000BF0020009004EB4400C0EB441001EBC5
:10FEB0008000406800680068009004EB4400C0EBDC
:10FEC000441001EB8000406800684068009000BF6B
:10FED00000BF00BF04EB4400C0EB44100E4901EB2F
:10FEE000800040680068006800F008000028C8D161
:10FEF00004EB4402C2EB44120B4603EB820202F114
:10FF0000680104EB4402C2EB441203EB8202506826
:10FF10000122F7F7DBFE1CBD98E1002070B5044616
:10FF20000D4604EB4401C1EB4411114A02EB81017F
:10FF30004868F7F790FB04EB4400C0EB44100C4911
:10FF400001EB80004068456004EB4401C1EB4411C3
:10FF5000074A02EB81014868F7F740FC10B14FF007
:10FF6000FF3070BD204600F005F80020F9E70000E2
:10FF700098E1002070B5044604EB4400C0EB441047
:10FF8000534901EB8000807838BB04EB4400C0EBA0
:10FF9000441001EB8000806804EB4401C1EB441184
:10FFA0004B4A02EB8101086104EB4400C0EB4410B2
:10FFB000114601EB8000806804EB4401C1EB441161
:10FFC00002EB8101C9680844401E04EB4401C1EB07
:10FFD000441102EB8101486123E004EB4400C0EBD3
:10FFE00044103B4901EB80008078012819D104EBD3
:10FFF0004403C3EB44130D4605EB8303DA6804EBBB
:020000040803EF
:100000004403C3EB441305EB8303996804EB4403F7
:10001000C3EB441305EB830303F118000123F8F746
:10002000D4F804EB4400C0EB4410294901EB8000F4
:10003000407840B104EB4400C0EB441001EB800079
:10004000407801281FD104EB4405C5EB4415204E30
:1000500006EB85056B6B04EB4405C5EB441506EB1D
:1000600085052A6B04EB4405C5EB441506EB8505B5
:10007000E96A04EB4405C5EB441506EB850505F17B
:100080003800F9F717FE04EB4400C0EB44101049A8
:1000900001EB8000807818B92046FFF771FE15E06B
:1000A00004EB4400C0EB4410094901EB8000807868
:1000B000012808D004EB4400C0EB441001EB8000A1
:1000C0008078022802D12046FFF7D8FE002070BDBC
:1000D00098E1002070B504460D460DB1032C02DBFB
:1000E0004FF0FF3070BD04EB4401C1EB4411084AEE
:1000F00002EB81007421F9F773FB04EB4400C0EBC1
:100100004410034901EB800045600020EAE700004D
:1001100098E1002070B50546002400BF2EE004EBF6
:100120004400C0EB4410174901EB80004068A8422E
:1001300022D104EB4400C0EB441001EB8000807836
:1001400018B92046FFF71CFE15E004EB4400C0EB95
:1001500044100C4901EB80008078012808D004EBA2
:100160004400C0EB441001EB80008078022802D1EB
:100170002046FFF783FE03E0601CC4B2032CCEDBF5
:1001800000BF70BD98E1002038B50546002400BFCF
:1001900054E004EB4400C0EB44102A4901EB80001A
:1001A0004068A84248D104EB4400C0EB441001EB86
:1001B00080008078012818D104EB4400C0EB441083
:1001C00001EB800090F86800009004EB4401C1EB63
:1001D00044111C4A02EB810101F118006946F7F74E
:1001E000D7FF2046FFF74AFE25E004EB4400C0EBB2
:1001F0004410144901EB8000807802281BD104EBE5
:100200004400C0EB441001EB8000006F80B104EBB0
:100210004402C2EB44120B4603EB820292F86800E0
:1002200004EB4402C2EB441203EB8202116F8847D5
:100230002046FFF723FE03E0601CC4B2032CA8DBBA
:1002400000BF38BD98E100202DE9F04104460F467B
:1002500015464FF0000817B10DB1032C03DB4FF02A
:10026000FF30BDE8F08104EB4400C0EB441060496E
:1002700001EB8000406810B94FF0FF30F1E704EB6C
:100280004400C0EB44105A4901EB80004078E8BBC1
:1002900000BFF9F757F804EB4401C1EB4411544A8D
:1002A00002EB810101F138002946F9F7D7FC064637
:1002B00026B9F9F72FFA4FF0FF382EE004EB44018E
:1002C000C1EB44114A4A02EB810101F13800314689
:1002D000F9F791FC2A4639463068EFF7B8FF04EB8E
:1002E0004401C1EB4411424A02EB810101F13800A3
:1002F000F9F795FC0646F9F70DFAB3889AB204EBC4
:100300004403C3EB4413DFF8E8C000E006E00CEB65
:10031000830331685868F7F77DFD66E004EB44001D
:10032000C0EB4410324901EB80004078012843D1F2
:1003300000BFF9F707F804EB4401C1EB44112C4A64
:1003400002EB810101F138002946F9F787FC0646E6
:1003500026B9F9F7DFF94FF0FF382CE004EB440140
:10036000C1EB4411224A02EB810101F13800314610
:10037000F9F741FC2A4639463068EFF768FF04EB8D
:100380004401C1EB44111A4A02EB810101F138002A
:10039000F9F745FC0646F9F7BDF9B3889AB204EBC4
:1003A0004403C3EB4413DFF848C00CEB830331680C
:1003B0005868F7F77DFD18E004EB4400C0EB4410EB
:1003C0000B4901EB8000407802280ED1642105FB27
:1003D00001F3AAB204EB4401C1EB4411044E06EB55
:1003E000810148683946F7F7AAFC404639E7000022
:1003F00098E100202DE9F0410646002400BF88E086
:1004000004EB4400C0EB4410454901EB8000406818
:10041000B0427CD104EB4400C0EB441001EB8000FF
:10042000407898BB00BF04EB4401C1EB44113C4A47
:1004300002EB810101F13800F9F7F1FB054604EB0D
:100440004401C1EB4411364A02EB810101F138004D
:100450002946F9F7BCFB04EB4401C1EB4411304AD7
:1004600002EB810101F13800F9F7D9FB054665B1CE
:10047000AB889AB204EB4403C3EB4413284F07EB59
:10048000830329685868F7F7C5FC3EE0FFE704EBF3
:100490004400C0EB4410224901EB80004078012861
:1004A00033D100BF04EB4401C1EB44111C4A02EB01
:1004B000810101F13800F9F7B2FB054604EB440174
:1004C000C1EB4411164A02EB810101F138002946C3
:1004D000F9F77DFB04EB4401C1EB4411104A02EB38
:1004E000810101F13800F9F79AFB054665B1AB8847
:1004F0009AB204EB4403C3EB4413094F07EB8303A5
:1005000029685868F7F7D4FC00BF05E0FFE7601CD6
:10051000C4B2032CFFF674AF00BFBDE8F081000049
:1005200098E1002038B50446622C0CD10020154912
:10053000A1F86200088001F0F5FE13A11AA000F0F6
:1005400065F9FFF79BF8642C1BD14AF6AA200090AE
:10055000002302224FF488311846FBF79FFC022348
:100560006A464FF488310020FBF7B4FE0A20F5F705
:10057000ABF911A10CA000F049F90020FBF7E2FB58
:1005800000BF38BD982400202E2E5C41504C5C7377
:10059000657269616C5F61745F636D645F617070E7
:1005A0002E633A35350000002573205552545265AC
:1005B00073746172740000002E2E5C41504C5C73A9
:1005C000657269616C5F61745F636D645F617070B7
:1005D0002E633A363700000000BFFEE770B50446D0
:1005E00000256448007808285AD100BF002004E0A4
:1005F0006149095C29448DB2401C60490978491F52
:100600008142F5DC5E480078284485B25B4800787A
:10061000284485B25B480078284485B25A4800785F
:10062000284485B259480078284485B26019C0B280
:10063000FF282BD15248007801281DD0022823D151
:1006400050480078FFF76EFF51494E4A12788818DB
:100650004D490A784849EFF7FAFD4A480078602882
:1006600003DB48480078642805DD01F05BFE0120CB
:100670004749A1F8600008E042480078411042482C
:100680000078FBF73DFF00E000BF00BF00203949C4
:1006900008703C490870394908703E49087067E0A5
:1006A00034480078072812D133483A49097844542D
:1006B00038480078401C3749087030480078401F9F
:1006C0000978884254D108202A49087050E0294806
:1006D0000078062805D12C480470072025490870A9
:1006E00046E024480078052805D1264804700620F5
:1006F000204908703CE01F480078042805D12048B4
:10070000047005201B49087032E01A48007803285D
:1007100008D11A48047000201A49087004201549AD
:10072000087025E01348007828B9552C03D1012022
:10073000104908701CE00F480078012805D1AA2C48
:1007400003D102200B49087012E00A480078022801
:1007500007D1032C05D10320064908700B4804700B
:1007600006E0002003490870064908700349087034
:1007700070BD000080010020B82800208201002008
:1007800085010020830100208101002084010020D8
:10079000982400208601002010B502211348F5F7A7
:1007A0001DFBC8B9F8F714FF11490968401A40F653
:1007B000B83188420DD902200E49088001200E4927
:1007C00008700E4908700E490870F8F701FF0849D3
:1007D0000860F8F7FDFE07E0F8F7FAFE0449086044
:1007E000F8F7F6FE0749086010BD0000000402405B
:1007F0002400002004000020B70100202C0000206D
:10080000B60100202800002000BFFEE70FB4054B12
:1008100010B503A9044A029800F028FA10BC5DF84C
:1008200014FB0000D91D03087C0900200FB41CB57F
:100830000246002007AC00290BD0491ECDE900215B
:10084000054B6A462146069800F010FA009A0021EE
:1008500011701CBC5DF814FB9B1303080FB4084B0C
:1008600010B504A902AA039800F000FA044602A9F0
:10087000002000F09DFD204610BC5DF814FB000038
:10088000B11303087CB5044600201D461646002916
:100890000BD0491ECDE90041044B6A46294630463B
:1008A00000F0E4F9009A002111707CBD9B1303084D
:1008B00000487047800900202DED020B019820F0C0
:1008C000004001909DED000B02B070470000000059
:1008D00000B583B09FED060B0A4601468DED000B77
:1008E0006846EFF7AEFF9DED000B03B000BD0000C2
:1008F000000000000000000002E008C8121F08C14C
:10090000002AFAD170477047002001E001C1121F90
:10091000002AFBD1704708B5002000906B460122E9
:1009200002212C2001F0E5F9022000906B46012203
:1009300002212C2001F0DDF908BD38B504466D20F8
:1009400000906B46012240F606012E2001F0D1F9FD
:100950003CB140F2076241F606012E2001F09EF9FB
:1009600006E041F2076241F606012E2001F096F9F9
:1009700038BD38B504466B4602220021362001F00E
:1009800027F80E2C57D2DFE804F011071A565656F6
:1009900056233256563F464D00208DF800009DF8F4
:1009A000010000F0FE008DF8010045E09DF8000018
:1009B00000F0FC0040F001008DF800003CE09DF8E4
:1009C000000000F0FC0040F002008DF8000033E071
:1009D0009DF8000000F0B30040F048008DF80000E2
:1009E0009DF8010040F080008DF8010024E09DF8A2
:1009F000000000F0B3008DF800009DF8010000F049
:100A00007F008DF8010017E09DF8010040F0020022
:100A10008DF8010010E09DF8010000F0FD008DF858
:100A2000010009E09DF8000000F0CF0040F0200038
:100A30008DF8000000E000BF00BF6B4601220021DE
:100A4000362001F056F90DF101030122114636203E
:100A500001F04FF938BD08B503208DF801000120E1
:100A60008DF800006B4602220021362001F041F98A
:100A70004FF4004206212D2001F010F9012000F072
:100A80009CFC0120FFF775FF08BD38B50446200A1D
:100A90008DF80100E0B28DF800006B4602220421BF
:100AA0002D2001F026F903208DF800006B4601226D
:100AB00006212D2001F01DF900208DF800006B4665
:100AC000012206212D2001F014F90A212D2000F029
:100AD0005DFF0546284638BD2DE9FF5F82B0002145
:100AE000DDE90430020DDDF840B0034318D044F6D0
:100AF0001050A2F2FF3242431514119801281FD062
:100B0000A5EB0B00401C5FEA000A4FF000064E4FB9
:100B1000DFF83891B046504615D5CAF1000413E00D
:100B2000119801244AA3012801D16FEA0B01029810
:100B3000119AC0E90031C0E9024206B0BDE8F09F59
:100B4000CBF10000DFE704460021404A491842EBA0
:100B50000450CDE9001012E0E00707D032463B46D2
:100B600040464946EFF7ADFC8046894632463B4653
:100B700010461946EFF7A5FC06460F466410002CF8
:100B8000EAD1DDE90401DDE90023BAF1000F06DA5C
:100B9000EFF797FC42464B46EFF793FC05E0EFF783
:100BA00002FD42464B46EFF7FEFC04460E4600228D
:100BB000284BEFF7BFFD03D84FF0FF30014607E0A9
:100BC0000022254B20463146EFF7D4FBEFF738FFE4
:100BD000102409E0002C0ADB0A220023EFF7F6FAC2
:100BE000039B30321A55641E50EA0102F2D1641C94
:100BF000039AC4F111031444119A012A03D001226B
:100C000008430DD10AE0084304D000204FF0110B37
:100C1000119072E7A3EB0B056D1E0DE05B4504DD43
:100C20004FF0000205F1010504E003DA4FF0000285
:100C3000A5F10105002AECD002981199C0E9023112
:100C4000C0E9004579E70000000014400000F03FD3
:100C5000300000000000F0430000E03F30380A2878
:100C600001D2012070470020704700002DE9FF4F9E
:100C700095B09B468946064600250FE2252877D188
:100C800000242746F84A0121059400E0044316F8A1
:100C9000013F203B01FA03F01042F7D130782A28B7
:100CA00011D06FF02F033078A0F13002092A16D846
:100CB000059A44F0020402EB820203EB4202104464
:100CC000761C0590EFE759F8042B0592002A03DA09
:100CD000504244F40054059044F00204761C3078ED
:100CE0002E2816D116F8010F44F004042A280DD03E
:100CF0006FF02F023078A0F13003092B09D807EBF1
:100D0000870302EB4303C718761CF3E759F8047B0B
:100D1000761C30786C280FD006DC4C2817D0682859
:100D20000DD06A2814D104E0742810D07A280FD18D
:100D30000DE044F400140AE044F4801401E044F4AB
:100D400040147278824202D104F58014761C761C1D
:100D5000307866280BD013DC582877D009DC0028BF
:100D600075D04528F6D04628F4D047281AD19DE101
:100D700018E0632835D0642879D0652812D195E130
:100D8000702873D008DC6728F1D069286FD06E28EE
:100D90000DD06F2806D1B5E073282CD0752875D0FA
:100DA000782874D05A46179990476D1C75E1C4F3A2
:100DB0000250022809D003280DD0D9F800100428C9
:100DC0000DD00D6009F1040967E1D9F80010EA17A8
:100DD000C1E90052F6E7D9F800100D80F2E70D7076
:100DE000F0E719F8041B8DF8001000208DF80100C1
:100DF000EA46012003E059F804AB4FF0FF306107E9
:100E00004FF0000102D40DE008F101018846B9421B
:100E10000FDA8045F8DB1AF808100029F4D108E051
:100E200008F1010188468142FADB1AF8081000290E
:100E3000F6D105985B46A0EB080721463846179A7D
:100E400000F094FA284400EB080507E04DE029E1A2
:100E50000DE01AF8010B5A4617999047B8F10108AE
:100E6000F7D25B4621463846179A13E142E00A2240
:100E70000092C4F302524FF0000A022A08D059F837
:100E800004CB032A4FEAEC710AD00DE029E02AE0F6
:100E900009F1070121F00702F2E802C1914609E0D9
:100EA0000FFA8CFC4FEAEC71042A03D14FFA8CFC48
:100EB0004FEAEC71002907DA0A460021DCF1000C48
:100EC00061EB02012D2202E0220504D52B228DF8D0
:100ED0000420012203E0E20701D02022F7E7904638
:100EE00059E00A2102E010220DE010214FF0000A23
:100EF00000910BE010224FF0000A44F00404082790
:100F0000009203E008224FF0000A0092C4F302525C
:100F1000022A05D059F804CB0021032A08D009E0A1
:100F200009F1070121F00702F2E802C1914605E04C
:100F30001FFA8CFC042A01D10CF0FF0C4FF00008C2
:100F4000220728D5702806D0009B83F0100353EAAF
:100F50000A0305D00EE040228DF80420012208E0AB
:100F60005CEA010206D030228DF804208DF80500DD
:100F700002229046009B83F0080353EA0A030AD139
:100F80005CEA010201D1620705D530228DF8042008
:100F90004FF001087F1E582804D034A003900EA8FB
:100FA00002900DE036A0F9E753466046009AEFF74D
:100FB0000DF984460398825C0298401E02900270EC
:100FC0005CEA0100F0D1029806A9081A00F1200A93
:100FD000600702D524F4803400E00127574502DD84
:100FE000A7EB0A0000E0002000EB0A010090059842
:100FF0004144401A0590E00306D45B462146179A07
:10100000059800F0B3F90544002706E001A85A4608
:10101000C05D179990476D1C7F1C4745F6DBE003C8
:101020000CD55B462146179A059800F09FF90544B8
:1010300004E030205A46179990476D1C0099481ECD
:1010400000900029F5DC08E0029802995A460078E1
:10105000491C0291179990476D1CBAF10001AAF141
:10106000010AF1DC65E1000009280100303132336A
:1010700034353637383961626364656600000000D4
:1010800030313233343536373839414243444546BE
:101090000000000000F058F90544761C3078002864
:1010A0007FF4ECAD19B02846BDE8F08F620700D49C
:1010B000062709F1070222F0070CFCE80223E146AB
:1010C00003F000485FEA080C02D00FF2702C0DE02C
:1010D0005FEA045C02D50FF2682C07E05FEAC47C8B
:1010E00002D00FF2602C01E0AFF2700C4FF0FF382D
:1010F00023F00043CDF850C065280CD006DC45280D
:1011000009D046281DD047283DD13DE0662818D09B
:1011100067287ED138E00021112F01DB112000E08B
:10112000781CCDE9000106A90EA8FFF7D5FCDDE982
:101130000F010E9A03910021009207F1010A049118
:101140004DE04FF000400097CDE9011006A90EA830
:10115000FFF7C2FCDDE90F0203920E9B11990022FA
:10116000DDF80CA00093049211B9791C00EB010A80
:10117000B7EB0A0004D4C0F1FF3007F1010A049074
:10118000AAEB0700019044E0012F00DA01270021BB
:10119000112F01DD112000E03846CDE9000106A93C
:1011A0000EA8FFF799FCDDE90F010E9A03910021CB
:1011B00004910092BA4621070CD40399514500DAF4
:1011C0008A46BAF1010F05DD009AAAF10101515CCE
:1011D000302908D0B84202DA10F1040F06DA0121F2
:1011E000CDE9011015E0AAF10101E9E7002805DCCD
:1011F000049901440491AAEB000102E0411C51450D
:1012000000DD8A460499401A401C01904FF00040CE
:101210000290200704D40198504501DBCDF80480EA
:1012200000208DF84F0002980DF14F07B0F1004FEC
:1012300025D02B200E9002984FF0020800280CDADF
:10124000404202902D200E9007E00A210298EFF70D
:10125000A5FA3031029007F8011DB8F10001A8F19C
:101260000108F2DC02980028EFD1791E0E98087070
:10127000307800F0200040F0450007F8020D12A879
:10128000C01B00F107081498007800B1012000EBA2
:101290000A01019801EBE07105984144401A401E93
:1012A0000590E00306D45B462146179A059800F0A6
:1012B0005DF805441498007818B15A46179990477C
:1012C0006D1CE00324D55B462146179A059800F073
:1012D0004DF805441CE00498002807DBDDE9030114
:1012E000884203DD0098405C179901E0179930208F
:1012F0005A469047049805F10105401C0490019856
:10130000401E019004D12E205A46179990476D1C1B
:10131000BAF10001AAF1010ADDDC05E017F8010BC2
:101320005A46179990476D1CB8F10001A8F10108C1
:10133000F4DC5B462146179A0598ABE62D000000C9
:101340002B000000200000002DE9F041044600259C
:101350001E461746880404D405E039462020B047CD
:101360006D1C641EF9D52846BDE8F0812DE9F041D9
:10137000044600251E469046C80301D5302700E0EC
:101380002027880404D505E041463846B0476D1C47
:10139000641EF9D52846BDE8F0814A68002A06D0C7
:1013A0000A68531C0B6010704868401E4860704704
:1013B0000A68531C0B601070704710B503464FF459
:1013C0007A7003FB00F4204600F001F810BD002104
:1013D00000BF40E000BF00BF00BF00BF00BF00BFB4
:1013E00000BF00BF00BF00BF00BF00BF00BF00BF05
:1013F00000BF00BF00BF00BF00BF00BF00BF00BFF5
:1014000000BF00BF00BF00BF00BF00BF00BF00BFE4
:1014100000BF00BF00BF00BF00BF00BF00BF00BFD4
:1014200000BF00BF00BF00BF00BF00BF00BF00BFC4
:1014300000BF00BF00BF00BF00BF00BF00BF00BFB4
:1014400000BF00BF00BF00BF00BF00BF00BF00BFA4
:1014500000BF00BF491C8142BCD370472DE9F84F43
:1014600004464FF00009CA4625786079824931F870
:1014700010806078401E8149C6B20863042D01D0F7
:10148000072D01D1012000E00020834620787B4910
:101490000873E07938B90846806940F480008861B3
:1014A0004FEAE80805E07548806920F48000734938
:1014B0008861207A7149487308468069217A4FF41F
:1014C000403202EA014108436C4988610846002124
:1014D0008269042000F0F5FB424642F604012E200A
:1014E00000F0DCFB3046FFF728FA6548405D00EB72
:1014F000800064494318052207212B2000F0F9FBE6
:10150000614800EB0B0301220B21282000F0F1FBC6
:101510005B48405D5D4951F820200C21282000F0F7
:10152000D0FBE0795A4901EB8000A17930F8112015
:101530000221272000F0B2FB564830F81620042183
:10154000272000F0ABFBE07928B964220621272090
:1015500000F0A4FB1EE0A07804280DD1102000901C
:1015600010220621272000F099FB6B46012226213C
:10157000272000F0BEFB0DE028200090202206214D
:10158000272000F08BFB6B4601222621272000F04C
:10159000B0FB00BF404800EB0610E17850F8212076
:1015A0000821272000F08DFBB4F8090018B941F29A
:1015B0004100A4F80900B4F809202021272000F0F8
:1015C0006DFB36480C210268232000F07AFB33487B
:1015D000001D30F816200421232000F05FFBA079C5
:1015E00058B1E0792E49431801220021212000F052
:1015F00080FB4FF003094FF0010A05F00F00F021C6
:1016000001EA0511084361784FF4402202EA814162
:101610000843910001EA095108434FF4003101EAFF
:101620004A41084321794FF0F86202EA81510843A8
:101630006179520102EAC16140EA01073A4600219C
:101640001F2000F03EFBA0786178084300040B499E
:10165000086108460069E1794FF4004242EA4131ED
:10166000084306490861084600210269082000F085
:1016700028FB0020BDE8F88FC42A030884E400207A
:101680006C2A0308800600209E060020742A0308A6
:10169000942A0308A02A0308A42A03088C2A030812
:1016A000A006002038B504460D460848808B044348
:1016B000224600212C2000F0F1FA00956B46012211
:1016C00006212C2000F015FB38BD000084E400202A
:1016D00010B5FFF720F910BD70B50546042136207E
:1016E00000F054F9044615B144F4006401E024F418
:1016F000006422460421362000F0E3FA70BD0000A9
:1017000038B54020009000210E2000F03FF904463B
:10171000002211460E2000F0D4FA6B46012200216F
:101720000D2000F0E6FA084A00210F2000F0C9FA67
:1017300000F098FA224600210E2000F0C2FA0020A4
:10174000024981F82C0038BDF8FF272484E40020EA
:101750002DE9FC4105460420019000264FF00008C9
:1017600000207849487508630021764880F82510E4
:101770000020744981F82C0088834863886300F056
:1017800021F9704908600EE04FF480106E498861BD
:1017900040F2A460FFF71BFE10206B49886100F047
:1017A00011F968490860674800686849884204D0B0
:1017B0003846791CCFB20A28E6DB0A2F03DD002069
:1017C0006349A1F858000020FFF7D3F800F0FAF8B9
:1017D0005C4908605F480078242805DD5D48007892
:1017E00024385D49086011E05A480078062190FBD2
:1017F000F1F201FB120057490978062291FBF2F140
:10180000C1F1060140EA411053490860524800788E
:1018100000065149098840EA01404F49096840EAF9
:1018200001204D49096808434C49086008460021D9
:1018300002681E2000F045FA00F0C4F84149086033
:1018400001AB01220021242000F053FA1E20FFF7F3
:101850001CF986B2300A3B4988730420FFF715F95A
:10186000804600F0AFF83749086008F0FF0070B11B
:10187000022000906B46012212212D2000F039FA3F
:101880003048808B40F480502E49888300BF00F0A0
:1018900099F82C4908600620FFF7F7F829494860B5
:1018A0000720FFF7F2F82749886006F01F00087547
:1018B0000846007D08B9102008752249087D00F00F
:1018C00071FA05F0010040B1FFF7C5F81D48808BA3
:1018D00040F400601B4988830DE00521362000F0AC
:1018E0003FF804464FF6FF500440224605213620BB
:1018F00000F0D4F900BF0120FFF73BF800210420DD
:1019000000F044F80F498861012000F0EBF8002155
:10191000262000F03BF8044644F4A03444F4A0240C
:1019200022460021262000F0CCF900222621362074
:1019300000F0B4F900F046F8024908600020BDE864
:10194000FC81000084E40020000002403001CADE77
:101950009824002075060020780600207C060020D0
:10196000F8B504460D464FF6FF76A9B2A0B26B4615
:10197000022200F02DF8074637B99DF800009DF8C7
:10198000011000EB012086B23046F8BD2DE9F84386
:1019900005460E464FF0FF37B1B2A8B26B4604229F
:1019A00000F016F88046B8F1000F08D1032404E0D7
:1019B0001DF8040000EB0727641E002CF8DA3846F7
:1019C000BDE8F88310B500210846FFF7DFFF10BD22
:1019D0002DE9F84306460C461746984600252CB9D3
:1019E000F2B228466D1C0DF800201BE0F0B240F06A
:1019F000400228466D1C0DF800207F2C05DCE2B269
:101A000028466D1C0DF800200CE0E0B240F080028A
:101A100028466D1C0DF80020C4F3C71228466D1C23
:101A20000DF80020A8B243463A46694600F03EFC55
:101A3000BDE8F88370B504460D46164623462A468F
:101A400031461120FFF7C4FF70BD10B50446234690
:101A5000052200211520FFF7BBFF10BD38B5044655
:101A60000020009000F0FEF84FF480750CB145F4B2
:101A700000752A4600210D2000F010F9B4B16B4624
:101A8000012203210F20FFF7A3FF9DF8000000F0C3
:101A9000080058B1FFF734FE4FF480752A46002144
:101AA0000D2000F0FBF84FF0FF3038BD0020FCE7C0
:101AB00010B50446224601210A2000F002F910BDAB
:101AC00070B504460E4600210E20FFF75FFF054665
:101AD0000EB1254300E0A5432A4600210E2000F068
:101AE000F0F870BD70B5054600212620FFF74EFFC7
:101AF000044624F47C2405F0010008B144F4802459
:101B000005F0020008B144F4A0342246002126204A
:101B100000F0D7F870BD70B5054600211A20FFF718
:101B200035FF04466FF31304C5F313000443224644
:101B300000211A2000F0C5F870BD10B504462246F9
:101B400041F604012E2000F0A9F810BD38B5044676
:101B50006B46012203210420FFF73AFF002C16DD1B
:101B6000224600210C2000F099F89DF8000040F07A
:101B7000100000900F48806940F080500D49886146
:101B80006B4601220321042000F0B3F810E09DF819
:101B9000000020F0100000900648806920F080507E
:101BA000044988616B4601220321042000F0A1F85A
:101BB00038BD000084E4002010B504462246002110
:101BC000182000F06BF810BDF8B504460025002081
:101BD0000090002604F0020058B1802000906B466F
:101BE000012200210D2000F084F801201C4981F819
:101BF0002C0004F0010028B39DF8000040F006001E
